:020000040800F2
:1060000000FC0020119F00088D9F000819A00008C7
:1060100085A0000887A0000889A0000800000000F3
:106020000000000000000000000000008BA000083D
:106030008DA00008000000008FA000088FA00008BD
:10604000619F0008619F0008ADA00008619F0008E3
:10605000619F0008619F000803A1000809A10008D2
:106060000FA1000815A100081BA10008B9A0000895
:10607000C5A00008D1A00008DDA00008619F0008AD
:10608000619F0008619F0008619F0008619F0008F0
:10609000619F0008619F000821A10008619F00081E
:1060A000619F0008619F0008619F0008619F0008D0
:1060B000619F0008619F0008619F0008619F0008C0
:1060C0007969020885690208619F0008619F0008DC
:1060D000E9A0000801A10008B5A10008619F00081F
:1060E000619F000861A1000895A00008619F000859
:1060F000619F0008619F0008619F0008619F000880
:10610000619F0008619F0008A1A00008CDA10008C0
:10611000619F0008619F0008619F0008619F00085F
:10612000619F0008619F0008619F0008619F00084F
:08613000619F0008619F000857
:1061400010B5054C237833B9044B13B10448AFF3B1
:1061500000800123237010BD300E002000000000DD
:1061600068DA020808B5034B1BB103490348AFF3D3
:10617000008008BD00000000340E002068DA02082C
:10618000034613F8012B002AFBD1181A0138704777
:1061900001F0FF01102A2BDB10F0070F08D010F8D8
:1061A000013B013A8B422DD010F0070F42B3F6D1DC
:1061B000F0B441EA012141EA014122F007047FF0F5
:1061C00000070023F0E80256083C85EA010586EA4C
:1061D000010685FA47F5A3FA87F586FA47F6A5FA88
:1061E00087F68EB9EED1F0BC01F0FF0102F0070294
:1061F00032B110F8013B013A83EA010313B1F8D13F
:106200000020704701387047002D06BF354603381F
:10621000073815F0010F07D1013015F4807F02BF58
:10622000013015F4C03F0130F0BC0138704700BFA9
:1062300010F8012B11F8013B012A28BF9A42F7D030
:10624000D01A704781F0004102E000BF83F00043A4
:1062500030B54FEA41044FEA430594EA050F08BF01
:1062600090EA020F1FBF54EA000C55EA020C7FEAC5
:10627000645C7FEA655C00F0E2804FEA5454D4EB42
:106280005555B8BF6D420CDD2C4480EA020281EA0C
:10629000030382EA000083EA010180EA020281EA44
:1062A0000303362D88BF30BD11F0004F4FEA013196
:1062B0004FF4801C4CEA113102D0404261EB4101A5
:1062C00013F0004F4FEA03334CEA133302D052422B
:1062D00063EB430394EA050F00F0A780A4F10104E7
:1062E000D5F1200E0DDB02FA0EFC22FA05F2801821
:1062F00041F1000103FA0EF2801843FA05F3594107
:106300000EE0A5F120050EF1200E012A03FA0EFC85
:1063100028BF4CF0020C43FA05F3C01851EBE371AF
:1063200001F0004507D54FF0000EDCF1000C7EEBCC
:1063300000006EEB0101B1F5801F1BD3B1F5001F0A
:106340000CD349085FEA30004FEA3C0C04F1010429
:106350004FEA445212F5800F80F09A80BCF1004F52
:1063600008BF5FEA500C50F1000041EB045141EAD4
:10637000050130BD5FEA4C0C404141EB0101013C9D
:1063800028BFB1F5801FE9D291F0000F04BF01468C
:106390000020B1FA81F308BF2033A3F10B03B3F15E
:1063A00020020CDA0C3208DD02F1140CC2F10C02EE
:1063B00001FA0CF021FA02F10CE002F11402D8BF4C
:1063C000C2F1200C01FA02F120FA0CFCDCBF41EA18
:1063D0000C019040E41AA2BF01EB0451294330BDE7
:1063E0006FEA04041F3C1CDA0C340EDC04F11404C4
:1063F000C4F1200220FA04F001FA02F340EA03009B
:1064000021FA04F345EA030130BDC4F10C04C4F1E0
:10641000200220FA02F001FA04F340EA03002946C0
:1064200030BD21FA04F0294630BD94F0000F83F40A
:10643000801306BF81F480110134013D4EE77FEAED
:10644000645C18BF7FEA655C29D094EA050F08BF39
:1064500090EA020F05D054EA000C04BF194610461A
:1064600030BD91EA030F1EBF0021002030BD5FEA5E
:10647000545C05D14000494128BF41F0004130BD86
:1064800014F580043CBF01F5801130BD01F00045DA
:1064900045F0FE4141F470014FF0000030BD7FEA4D
:1064A000645C1ABF194610467FEA655C1CBF0B4648
:1064B000024650EA013406BF52EA033591EA030F5F
:1064C00041F4002130BD00BF90F0000F04BF002157
:1064D000704730B54FF4806404F132044FF000058A
:1064E0004FF0000150E700BF90F0000F04BF002103
:1064F000704730B54FF4806404F1320410F0004569
:1065000048BF40424FF000013EE700BF42004FEA63
:10651000E2014FEA31014FEA02701FBF12F07F43E0
:1065200093F07F4F81F06051704732F07F4208BF97
:10653000704793F07F4F04BF41F40021704730B59E
:106540004FF4607401F0004521F000411CE700BFEA
:1065500050EA010208BF704730B54FF000050AE06D
:1065600050EA010208BF704730B511F0004502D56E
:10657000404261EB41014FF4806404F132045FEA70
:10658000915C3FF4D8AE4FF003025FEADC0C18BF19
:1065900003325FEADC0C18BF033202EBDC02C2F10B
:1065A000200300FA03FC20FA02F001FA03FE40EA9D
:1065B0000E0021FA02F11444BDE600BF70B54FF0A1
:1065C000FF0C4CF4E06C1CEA11541DBF1CEA13557F
:1065D00094EA0C0F95EA0C0F00F0DEF82C4481EAE7
:1065E000030621EA4C5123EA4C5350EA013518BF07
:1065F00052EA033541F4801143F4801338D0A0FBF4
:1066000002CE4FF00005E1FB02E506F00042E0FBA0
:1066100003E54FF00006E1FB03569CF0000F18BFA6
:106620004EF0010EA4F1FF04B6F5007F64F540744E
:1066300004D25FEA4E0E6D4146EB060642EAC621E1
:1066400041EA55514FEAC52040EA5E504FEACE2E4E
:10665000B4F1FD0C88BFBCF5E06F1ED8BEF1004F51
:1066600008BF5FEA500E50F1000041EB045170BDCD
:1066700006F0004646EA010140EA020081EA030111
:10668000B4EB5C04C2BFD4EB0C0541EA045170BD0D
:1066900041F480114FF0000E013C00F3AB8014F187
:1066A000360FDEBF002001F0004170BDC4F10004D0
:1066B000203C35DA0C341BDC04F11404C4F1200551
:1066C00000FA05F320FA04F001FA05F240EA0200AC
:1066D00001F0004221F0004110EBD37021FA04F6E2
:1066E00042EB06015EEA430E08BF20EAD37070BD9C
:1066F000C4F10C04C4F1200500FA04F320FA05F0FB
:1067000001FA04F240EA020001F0004110EBD370FC
:1067100041F100015EEA430E08BF20EAD37070BD6C
:10672000C4F1200500FA05F24EEA020E20FA04F345
:1067300001FA05F243EA020321FA04F001F00041F4
:1067400021FA04F220EA020000EBD3705EEA430E65
:1067500008BF20EAD37070BD94F0000F0FD101F094
:106760000046400041EB010111F4801F08BF013CCD
:10677000F7D041EA060195F0000F18BF704703F00B
:106780000046520043EB030313F4801F08BF013D92
:10679000F7D043EA0603704794EA0C0F0CEA13554E
:1067A00018BF95EA0C0F0CD050EA410618BF52EA08
:1067B0004306D1D181EA030101F000414FF000000E
:1067C00070BD50EA410606BF1046194652EA43061C
:1067D00019D094EA0C0F02D150EA013613D195EA90
:1067E0000C0F05D152EA03361CBF104619460AD1D8
:1067F00081EA030101F0004141F0FE4141F47001E2
:106800004FF0000070BD41F0FE4141F4780170BDD1
:1068100070B54FF0FF0C4CF4E06C1CEA11541DBF36
:106820001CEA135594EA0C0F95EA0C0F00F0A7F838
:10683000A4EB050481EA030E52EA03354FEA013165
:1068400000F088804FEA03334FF0805545EA131378
:1068500043EA12634FEA022245EA111545EA106540
:106860004FEA00260EF000419D4208BF964244F1D7
:10687000FD0404F5407402D25B084FEA3202B61AF6
:1068800065EB03055B084FEA32024FF480104FF4CA
:10689000002CB6EB020E75EB030E22BFB61A75463E
:1068A00040EA0C005B084FEA3202B6EB020E75EBD1
:1068B000030E22BFB61A754640EA5C005B084FEA39
:1068C0003202B6EB020E75EB030E22BFB61A754606
:1068D00040EA9C005B084FEA3202B6EB020E75EB11
:1068E000030E22BFB61A754640EADC0055EA060ED2
:1068F00018D04FEA051545EA16754FEA06164FEA15
:10690000C30343EA52734FEAC2025FEA1C1CC0D1C0
:1069100011F4801F0BD141EA00014FF000004FF04D
:10692000004CB6E711F4801F04BF01430020B4F10E
:10693000FD0C88BFBCF5E06F3FF6AFAEB5EB030CC6
:1069400004BFB6EB020C5FEA500C50F1000041EBC3
:10695000045170BD0EF0004E4EEA113114EB5C0490
:10696000C2BFD4EB0C0541EA045170BD41F4801163
:106970004FF0000E013C90E645EA060E8DE60CEA6B
:10698000135594EA0C0F08BF95EA0C0F3FF43BAF88
:1069900094EA0C0F0AD150EA01347FF434AF95EA3F
:1069A0000C0F7FF425AF104619462CE795EA0C0F23
:1069B00006D152EA03353FF4FDAE1046194622E7F0
:1069C00050EA410618BF52EA43067FF4C5AE50EACA
:1069D00041047FF40DAF52EA43057FF4EBAE12E7BA
:1069E0004FF0FF3C06E000BF4FF0010C02E000BF9B
:1069F0004FF0010C4DF804CD4FEA410C7FEA6C5C7E
:106A00004FEA430C18BF7FEA6C5C1BD001B050EA20
:106A1000410C0CBF52EA430C91EA030F02BF90EA0B
:106A2000020F0020704710F1000F91EA030F58BFCA
:106A3000994208BF90422CBFD8176FEAE37040F02C
:106A4000010070474FEA410C7FEA6C5C02D150EACA
:106A5000013C07D14FEA430C7FEA6C5CD6D152EA85
:106A6000033CD3D05DF8040B704700BF844610464A
:106A700062468C461946634600E000BF01B5FFF749
:106A8000B7FF002848BF10F1000F01BD4DF808ED19
:106A9000FFF7F4FF0CBF012000205DF808FB00BFEA
:106AA0004DF808EDFFF7EAFF34BF012000205DF844
:106AB00008FB00BF4DF808EDFFF7E0FF94BF012091
:106AC00000205DF808FB00BF4DF808EDFFF7CEFF92
:106AD00094BF012000205DF808FB00BF4DF808EDD1
:106AE000FFF7C4FF34BF012000205DF808FB00BFA2
:106AF0004FEA410C7FEA6C5C02D150EA013C0AD1BA
:106B00004FEA430C7FEA6C5C02D152EA033C02D1AB
:106B10004FF0000070474FF0010070474FEA41020C
:106B200012F5001215D211D56FF47873B3EB6252DF
:106B300012D94FEAC12343F0004343EA505311F006
:106B4000004F23FA02F018BF404270474FF0000098
:106B5000704750EA013005D111F0004008BF6FF0D6
:106B6000004070474FF00000704700BF4A0011D24C
:106B700012F5001211D20DD56FF47873B3EB625297
:106B80000ED44FEAC12343F0004343EA505323FAA3
:106B900002F070474FF00000704750EA013002D118
:106BA0004FF0FF3070474FF0000070474FEA41024E
:106BB000B2F1E04324BFB3F5001CDCF1FE5C0DD95B
:106BC00001F0004C4FEAC0024CEA5070B2F1004FA5
:106BD00040EB830008BF20F00100704711F0804FA8
:106BE00021D113F13872BCBF01F00040704741F46D
:106BF00080114FEA5252C2F11802C2F1200C10FA71
:106C00000CF320FA02F018BF40F001004FEAC12354
:106C10004FEAD32303FA0CFC40EA0C0023FA02F3F8
:106C20004FEA4303CCE77FEA625307D150EA0133CE
:106C30001EBF4FF0FE4040F44000704701F000409E
:106C400040F0FE4040F40000704700BF80F000407C
:106C500002E000BF81F0004142001FBF5FEA410334
:106C600092EA030F7FEA226C7FEA236C6AD04FEA34
:106C70001262D2EB1363C1BFD21841404840414079
:106C8000B8BF5B42192B88BF704710F0004F40F42B
:106C9000000020F07F4018BF404211F0004F41F447
:106CA000000121F07F4118BF494292EA030F3FD013
:106CB000A2F1010241FA03FC10EB0C00C3F1200326
:106CC00001FA03F100F0004302D5494260EB4000B5
:106CD000B0F5000F13D3B0F1807F06D340084FEA20
:106CE000310102F10102FE2A51D2B1F1004F40EB15
:106CF000C25008BF20F0010040EA0300704749007D
:106D000040EB0000013A28BFB0F5000FEDD2B0FA19
:106D100080FCACF1080CB2EB0C0200FA0CF0AABF3C
:106D200000EBC25052421843BCBFD04018437047DA
:106D300092F0000F81F4000106BF80F400000132E0
:106D4000013BB5E74FEA41037FEA226C18BF7FEAB7
:106D5000236C21D092EA030F04D092F0000F08BFF9
:106D60000846704790EA010F1CBF0020704712F0E0
:106D70007F4F04D1400028BF40F00040704712F11F
:106D800000723CBF00F50000704700F0004343F084
:106D9000FE4040F4000070477FEA226216BF0846BA
:106DA0007FEA23630146420206BF5FEA412390EA7D
:106DB000010F40F4800070474FF0000304E000BF73
:106DC00010F0004348BF40425FEA000C08BF704724
:106DD00043F0964301464FF000001CE050EA0102E8
:106DE00008BF70474FF000030AE000BF50EA0102FD
:106DF00008BF704711F0004302D5404261EB4101EA
:106E00005FEA010C02BF84460146002043F0B6430E
:106E100008BFA3F18053A3F50003BCFA8CF2083A33
:106E2000A3EBC25310DB01FA02FC634400FA02FC3C
:106E3000C2F12002BCF1004F20FA02F243EB020043
:106E400008BF20F00100704702F1200201FA02FCA5
:106E5000C2F1200250EA4C0021FA02F243EB020098
:106E600008BF20EADC7070474FF0FF0C1CEAD052DC
:106E70001EBF1CEAD15392EA0C0F93EA0C0F6FD09D
:106E80001A4480EA010C400218BF5FEA41211ED07B
:106E90004FF0006343EA501043EA5111A0FB013167
:106EA0000CF00040B1F5000F3EBF490041EAD3713C
:106EB0005B0040EA010062F17F02FD2A1DD8B3F1B8
:106EC000004F40EBC25008BF20F00100704790F027
:106ED000000F0CF0004C08BF49024CEA502040EA79
:106EE00051207F3AC2BFD2F1FF0340EAC25070473F
:106EF00040F400004FF00003013A5DDC12F1190F7D
:106F0000DCBF00F000407047C2F10002410021FAEE
:106F100002F1C2F1200200FA02FC5FEA310040F106
:106F2000000053EA4C0308BF20EADC70704792F07F
:106F3000000F00F0004C02BF400010F4000F013AB7
:106F4000F9D040EA0C0093F0000F01F0004C02BFB2
:106F5000490011F4000F013BF9D041EA0C018FE721
:106F60000CEAD15392EA0C0F18BF93EA0C0F0AD027
:106F700030F0004C18BF31F0004CD8D180EA01004D
:106F800000F00040704790F0000F17BF90F0004FE6
:106F9000084691F0000F91F0004F14D092EA0C0FC8
:106FA00001D142020FD193EA0C0F03D14B0218BF5B
:106FB000084608D180EA010000F0004040F0FE40A1
:106FC00040F40000704740F0FE4040F4400070473D
:106FD0004FF0FF0C1CEAD0521EBF1CEAD15392EABC
:106FE0000C0F93EA0C0F69D0A2EB030280EA010CAC
:106FF00049024FEA402037D04FF0805343EA111145
:1070000043EA10130CF000408B4238BF5B0042F1A2
:107010007D024FF4000C8B4224BF5B1A40EA0C0047
:10702000B3EB510F24BFA3EB510340EA5C00B3EB79
:10703000910F24BFA3EB910340EA9C00B3EBD10F67
:1070400024BFA3EBD10340EADC001B0118BF5FEAB9
:107050001C1CE0D1FD2A3FF650AF8B4240EBC250E2
:1070600008BF20F0010070470CF0004C4CEA5020A3
:107070007F32C2BFD2F1FF0340EAC250704740F4F2
:1070800000004FF00003013A37E792F0000F00F0E4
:10709000004C02BF400010F4000F013AF9D040EA62
:1070A0000C0093F0000F01F0004C02BF490011F4F6
:1070B000000F013BF9D041EA0C0195E70CEAD153EE
:1070C00092EA0C0F08D142027FF47DAF93EA0C0FD5
:1070D0007FF470AF084676E793EA0C0F04D14B02B9
:1070E0003FF44CAF08466EE730F0004C18BF31F06B
:1070F000004CCAD130F000427FF45CAF31F0004365
:107100007FF43CAF5FE700BF4FF0FF3C06E000BFFD
:107110004FF0010C02E000BF4FF0010C4DF804CD20
:107120004FEA40024FEA41037FEA226C18BF7FEA30
:10713000236C11D001B052EA530C18BF90EA010F32
:1071400058BFB2EB030088BFC81738BF6FEAE170C1
:1071500018BF40F0010070477FEA226C02D15FEA5D
:10716000402C05D17FEA236CE4D15FEA412CE1D0C9
:107170005DF8040B704700BF844608466146FFE790
:107180000FB5FFF7C9FF002848BF10F1000F0FBD72
:107190004DF808EDFFF7F4FF0CBF012000205DF86B
:1071A00008FB00BF4DF808EDFFF7EAFF34BF0120F0
:1071B00000205DF808FB00BF4DF808EDFFF7E0FF89
:1071C00094BF012000205DF808FB00BF4DF808EDDA
:1071D000FFF7D2FF94BF012000205DF808FB00BF3D
:1071E0004DF808EDFFF7C8FF34BF012000205DF81F
:1071F00008FB00BF53B94AB9002908BF00281CBFCB
:107200004FF0FF314FF0FF3000F06CB9ADF1080CDA
:107210006DE904CE00F006F8DDF804E0DDE90223B4
:1072200004B070472DE9F047089E0D4604468E468F
:10723000002B40F082808A42174646D9B2FA82F289
:107240004AB1C2F1200105FA02F320FA01F1974098
:1072500041EA030E94404FEA1748230CBEFBF8FCAA
:10726000B9B208FB1CEE43EA0E430CFB01F0984256
:107270000AD9FB180CF1FF3580F01681984240F2D4
:107280001381ACF1020C3B441B1AA4B2B3FBF8F01F
:1072900008FB103344EA034400FB01F1A14209D981
:1072A0003C1900F1FF3380F00181A14240F2FE80E1
:1072B00002383C44641A40EA0C4000211EB1D4401C
:1072C0000023C6E90043BDE8F08702B9FFDEB2FA49
:1072D00082F2002A4FD1CB1B4FEA174E1FFA87F8D4
:1072E0000121B3FBFEFC250C0EFB1C3345EA0345D4
:1072F00008FB0CF3AB4207D97D190CF1FF3002D229
:10730000AB4200F2E7808446ED1AA3B2B5FBFEF073
:107310000EFB105543EA054408FB00F8A04507D9C9
:107320003C1900F1FF3302D2A04500F2D780184685
:10733000A4EB080440EA0C40C0E78B4208D9002EB9
:1073400000F0AF800021C6E900050846BDE8F087DF
:10735000B3FA83F100294BD1AB4202D3824200F24F
:10736000B780841A65EB030301209E46002EAAD045
:10737000C6E9004EA7E7C2F1200C01FA02F39740DC
:1073800020FA0CF04FEA174E21FA0CFC1843BCFB14
:10739000FEF1050C0EFB11CC1FFA87F845EA0C45EF
:1073A00001FB08F3AB4204FA02F409D97D1901F19B
:1073B000FF3C80F08B80AB4240F2888002393D4434
:1073C000EB1A85B2B3FBFEF00EFB103345EA034522
:1073D00000FB08F3AB4207D97D1900F1FF3C71D2E5
:1073E000AB426FD902383D44EB1A40EA014178E7DD
:1073F000C1F1200C8B4022FA0CF71F4320FA0CF449
:1074000005FA01F34FEA174E25FA0CF51C43230C3D
:10741000B5FBFEF91FFA87F80EFB195543EA05453F
:1074200009FB08FAAA4502FA01F200FA01F308D9A9
:107430007D1909F1FF3047D2AA4545D9A9F10209C2
:107440003D44A5EB0A05A4B2B5FBFEF00EFB1055BA
:1074500044EA054400FB08F8A04507D93C1900F1AF
:10746000FF352DD2A0452BD902383C4440EA0940D3
:10747000A4EB0804A0FB02894C45C6464D4619D32F
:1074800016D05EB1B3EB0E0264EB050404FA0CFCFB
:10749000CA404CEA0202CC40C6E900240021BDE803
:1074A000F087314630460EE7AC46EDE6184601E778
:1074B0004345E6D2B8EB020E69EB07050138E0E779
:1074C0002846D3E760468FE78146BAE7614677E70B
:1074D00008464BE7ACF1020C3D4415E702383C444A
:1074E00026E700BF704700BF10B5062286B0022312
:1074F00047484FF4E13104F0BFF90121084604F098
:1075000094FC0121002004F090FC0021012004F0F3
:10751000A3FC0021084604F09FFC41F288300AF0E9
:10752000F9FB3C493A4804F049FB3B4802A904F006
:10753000E9FA024618B13949354804F049FB9DF88B
:1075400016309DF814203649009331489DF81530C7
:1075500004F03EFB049B334900932D48DDE90223F0
:1075600004F036FB01220A210C2000F0F7F8002875
:1075700049D12D4926482D4C04F020FB00F034FA67
:107580002B490246224804F023FB0C21204600F040
:107590000BFA024690B127491D4804F019FB00F090
:1075A00023FA254902461A4804F012FB234B2449CA
:1075B0001A68174804F00CFB06B010BD21491448A6
:1075C00004F0FCFA2049124804F0E1FA0A2221688A
:1075D0000F4804F06DFB1D490D4804F0D8FA6068AF
:1075E000FEF794FF0B46022102460091084804F082
:1075F0000FFC1749064804F0CAFA217A04480A2207
:1076000004F056FBCBE71349014804F0D7FAC6E76C
:10761000841C0020B6DB0208D81C0020CFDB020847
:10762000F6DB020814DC02084BDC0208500E0020D6
:107630005EDC02086EDC0208FBDC0208600E002043
:1076400010DD020885DC020897DC0208ACDC0208C9
:10765000BFDC0208D6DC0208374B186870B5374C1F
:10766000013018602060FEF73FFF31A3D3E900230B
:10767000FEF7A4FFFFF79AFA0126606032460C215C
:107680002046267200F002F9054668B300F0ACF916
:107690002B4903462A462B4804F09AFA31463046D5
:1076A00004F0DAFB25480C2100F07EF9054600289D
:1076B00030D100F099F924490246224804F088FAB2
:1076C000226822491F4804F083FA6068FEF71EFF13
:1076D00002460B461B481E4904F07AFABDE870408A
:1076E00044F620600AF016BB00F07EF91949024604
:1076F000144804F06DFA22681449124804F068FA3C
:107700006068FEF703FF02460B460E48104904F07E
:107710005FFAC7E700F068F90F4903462A460948AF
:1077200004F056FA0121002004F096FBD6E700BFD2
:107730007B14AE47E17A843F4C0E0020500E0020AF
:1077400028DD0208841C002083DD020863DD0208B6
:1077500074DD020848DD0208A3DD02082DE9F04FC0
:1077600089B0044689463A4804A9164604F0CAF985
:10777000024640B13749384804F02AFA4FF0FF304A
:1077800009B0BDE8F08F354A354F049B3B600234A9
:107790001460B3FBF4F4334BDFF8ECA0DFF8B8B0BF
:1077A0004C4528BF4C46DFF8A8901C609046013C31
:1077B000D8F800106143022303AA0239484604F0B6
:1077C0007FF9054630B102462749234804F000FA04
:1077D0000320D5E79DF80D309DF80C20009451460C
:1077E000584604F0F5F99DF80C30AA2B0DD19DF800
:1077F0000D30A34209D122461C49174804F0E8F98C
:107800001B4B01341C602846BAE7E4B919491248F9
:1078100004F0DEF9164B184A1C60184B18490E4844
:10782000002E08BF1A4604F0D3F976B115490A486C
:1078300004F0C4F93A680648214604F070F920B112
:107840006FF004009CE7013CB2E7012098E700BF1D
:10785000D81C0020CDDD0208841C00205C0E002016
:10786000640E0020600E0020E5DD02081BDE020829
:10787000680E002032DE0208C2DD0208C7DD020801
:107880004ADE020879DE0208FBDD02082DE9FF4727
:107890003E4C3F4F23683F4E15463A6801339342B2
:1078A00084BF00232360236888463168814659439A
:1078B00008F10202384804F032F9306821684A467B
:1078C00041434346344804F00CF9024640B1334981
:1078D000334804F07DF96FF0010004B0BDE8F08793
:1078E000EDB1DFF8B4A0054645452168306816D0F3
:1078F00001236A4600FB0151504604F0E1F89DF86F
:10790000002019F805309A4207D0264924482A4613
:1079100004F05EF96FF00300DFE70135E4E70023D0
:10792000ADF800302368316823B3013B5943023975
:10793000022319486A4604F0D4F821684B1E3168C6
:10794000154859436A460223023904F0B9F8AA23BC
:1079500031688DF8003023688DF8013059430E48A6
:1079600002236A46023904F0BCF82368013323601D
:107970000020B2E73B680848013B59436A460223AE
:10798000023904F0AEF83B68013BD8E7680E0020EE
:10799000600E00205C0E0020D81C002087DE02084C
:1079A000841C00209FDE02080B460A4910B50C68B3
:1079B000024604B1013C084908480968614304F0E3
:1079C0007FF8024628B10649064804F001F96FF035
:1079D000020010BD680E00205C0E0020D81C0020A4
:1079E0006EDC0208841C0020024B186800B10138CC
:1079F000704700BF680E002003F072B903F075B93C
:107A000070470000BFF34F8F0549064BCA6802F468
:107A1000E0621343CB60BFF34F8F00BFFDE700BFB1
:107A200000ED00E00400FA0570B5002386B0CDE952
:107A300004334FF0B0420F4DD16C41F00201D164DC
:107A4000D26C039302F002024FF48056009201A917
:107A50002846CDE90163009A0CF060FD31462846C6
:107A60000CF07CFE3146044628460CF003FE20460E
:107A700006B070BD000400480D2070474FF0B043C1
:107A800082B0DA6C0243DA64DB6C18400190019B2F
:107A900002B070472DE9F04186B01422002101A800
:107AA00000F040FB0220FFF7E9FF144D144F0420C3
:107AB000FFF7E4FF4FF4807601230024CDE9016352
:107AC00001A903232846CDE903434FF400580CF0E5
:107AD00025FD01A93846CDF804800CF01FFD224693
:107AE000414638460CF040FE2846224631460CF00E
:107AF0003BFE204606B0BDE8F08100BF0004004810
:107B000000080048032810B50ED8012810D868B91D
:107B100002460B484FF480710CF026FE0022094803
:107B20004FF400510CF020FE002010BD0122F0E7C0
:107B3000012203484FF480710CF016FE0122EEE79B
:107B400000040048000800480220704701207047E8
:107B50000120704710B59AB04822002108A800F013
:107B6000E1FA1822002102A800F0DCFA0CF00EFE67
:107B70004FF0B0420024D2F8903023F01803C2F83E
:107B80009030D2F8003423F4C06343F40073C2F899
:107B90000034D2F80034119403F4C06301934FF41D
:107BA0008072019B0C922E234022089381230B9319
:107BB0000D920123B02208A8CDE90E341093129241
:107BC00013940CF035FF08B103F0DEF94F230221C6
:107BD00002A8CDE90234CDE90444CDE906440DF014
:107BE000C7F908B103F0D0F91AB010BD13B5037886
:107BF000082B00F29880DFE803F0128287968E8EC1
:107C0000059692000479204608F040FE204608F0D0
:107C1000E7FD0021204608F041FE02B010BD002023
:107C200008F034FE012839D1012008F02FFE012888
:107C300004D001200AF028FD00283DDC022008F0D5
:107C400025FE0128E9D002200AF01EFD0028E4DD0F
:107C5000012201A902200AF0E1FB022008F016FE31
:107C60000028F0D102200AF0EDFC00283FD19DF859
:107C70000410022008F020FDE5E7012201A9002000
:107C80000AF0CCFB002008F001FE044630B90AF0EF
:107C9000D9FC48B99DF8041008F00EFD00200AF048
:107CA000F3FC0028E9DCBFE70128F7D19DF80410B8
:107CB00020460AF01FFCF1E7012201A910460AF054
:107CC000ADFB012008F0E2FD0028B2D101200AF04E
:107CD000B9FC28B99DF80410012008F0EDFCA8E7D4
:107CE0000128A6D19DF804100AF004FCA1E70128A0
:107CF000A9D19DF8041002200AF0FCFBA3E714F0C0
:107D000043FA04F0E5F888E70A4B1B68002B84D09F
:107D10004068984781E740680AF052FD7DE7406877
:107D20000AF000FA79E7044B1B6E002B3FF475AFA5
:107D3000984772E7006F002014F2020830B52E4B0E
:107D40002E4A9A6085B00AF06FFDFFF703FF4FF0EF
:107D5000B0430B209A6C42F004029A649A6C02F0D1
:107D600004020392039A9A6C42F001029A649B6C9B
:107D7000002203F0010311460293029B0BF0BCF9B1
:107D80000B200BF0EBF90AF00FFD09F075FF08F07E
:107D90004FFE002401460546234603220120CDE97B
:107DA00000440AF07DFA2346032229460220CDE949
:107DB00000440AF075FA09F0C5FF08F033FD08F039
:107DC000E5FE06F04BF8E5B2284608F05FFD10B975
:107DD000284608F005FD0134032CF4D10AF0C8FC54
:107DE00009F0F4FB012804D105B0BDE8304006F0ED
:107DF000A9BB05B030BD00BF00ED00E00060000889
:107E000008B50AF0C3FCBDE8084004F061B8000002
:107E100013B5FFF793FF4FF0B043DA6C42F0020264
:107E2000DA64DB6C03F002030193019B02F06CF84F
:107E3000FFF7FAFDF0B1164804F013F8154B164899
:107E40001A68164B196804F00CF815480AF0AAFADB
:107E500004F04EFB01280FD002280FD010B91148B2
:107E60000AF0A0FA104CFFF7CBFF237843B902F0D9
:107E70004DF8F8E70D48DFE70D48F1E70D48EFE76B
:107E800008F04AFD0028EED000200AF0D3F9EAE716
:107E9000BFDE020870000020D7DE02088800002044
:107EA000E7DE0208FBDE02086C0E0020CBDE0208D3
:107EB00007DF020812DF0208054808B5082303603F
:107EC0000EF006F918B1BDE8084003F05DB808BD32
:107ED000E86700204FF0B04307B55A6E42F0010248
:107EE0005A665B6E002203F00103019311463220B3
:107EF000019B0BF001F9322003B05DF804EB0BF0AD
:107F00002DB90000024B9868024BC04318607047BF
:107F100000280040700E0020014B1868704700BF19
:107F2000700E0020034B044A9B681068DB43181A4C
:107F3000704700BF00280040700E0020034B1878E7
:107F400010B1034B9868C043704700BF6D0E00200E
:107F5000002800400320704708B501464FF47A72AC
:107F60000023C003490CFFF745F908BD4FF47A72AE
:107F7000A0FB0223D00B40EA4340704710B5074BEB
:107F8000074C0122DA654FF4807120460DF0EEF8BF
:107F90004FF0FF332363002010BD00BF00280040D6
:107FA000346A00200246002101480DF0F4BA00BFF7
:107FB000346A00200246012101480DF0ECBA00BFEE
:107FC000346A002010B58CB02C220021044601A890
:107FD00000F0A8F8FFF7D2FF0C4B18680023044408
:107FE000089306934FF00053E44307930848029424
:107FF0004FF48073012201A90B930DF0CDF908B164
:1080000002F0C2FF00200CB010BD00BF700E0020B7
:10801000346A00200C4B70B59C68064602210B4860
:108020000DF0C0FAE44300221219C2F30E044FF41B
:108030007A71A4FB014540F10003E40BD00B3480BE
:1080400040EA434070BD00BF00280040346A002071
:10805000014800210DF0A6BA346A00200148012130
:108060000DF0A0BA346A0020F8B5114E3578E5B9A4
:10807000104C2A4629464FF0FF372846276302F066
:1080800099FDFFF77BFF4FF4807120460DF06EF8ED
:10809000204627630DF02AFA2A46022120460DF0D9
:1080A0007AFAFFF72FFF012333700020F8BD00BFDD
:1080B0006D0E0020346A002011F08EBA10B5064C07
:1080C000022120460DF06EFA0221421C2046BDE836
:1080D00010400DF060BA00BF346A002070B50D4D3D
:1080E0000D4C641BA4100026A64209D10B4D0C4C6C
:1080F00025F0BAFC641BA4100026A64205D170BD71
:1081000055F8043B98470136EEE755F8043B98478D
:108110000136F2E778150308781503087815030887
:108120008415030802440346934200D1704703F8C4
:10813000011BF9E72DE9F04788B0002B1F461446D4
:10814000B8BF03F10043129A109DDDF84CA0B6BFF2
:108150001F4600232D231370149B23F02008B8F131
:10816000460F05D0B8F1450F00D10135022300E0DC
:10817000032307AA049206AACDE902A2CDE900359D
:1081800022463B4600F0C0FCB8F1470F064602D13C
:10819000119BDB0722D5B8F1460F06EB050910D17C
:1081A0003378302B0AD10022002320463946FEF7CF
:1081B0006DFC18B9C5F10105CAF80050DAF80030B5
:1081C00099440022002320463946FEF75FFC08B19F
:1081D000CDF81C903022079B4B4507D3079B159A7F
:1081E0009B1B3046136008B0BDE8F087591C07910F
:1081F0001A70F0E7F7B503460029B8BF494203F803
:10820000022BB4BF2D222B22092942702ADD0DF149
:108210000704A4460A27A6460A4691FBF7F607FB81
:1082200016153035632A04F1FF340EF8015C31462F
:10823000F1DC3031AEF1020504F8011C441C294682
:1082400061450AD30DF10902A2EB0E02654588BF14
:1082500000221344181A03B0F0BD11F8012B04F8E2
:10826000012FEDE7302330318370C170031DF1E73A
:108270002DE9F04F91B00C46DDF8688016461F4698
:10828000054601F013FA036809931846FDF778FFD5
:1082900000230E93D8F800300A90073323F0070329
:1082A00003F1080294F81890D4F800B0C8F8002040
:1082B000D3E90023C4E91223D4E9128A2AF0004347
:1082C0000B930B999C4B4FF0FF324046FEF710FC8E
:1082D00070BB994B0B994FF0FF324046FEF7EAFB1B
:1082E00030BB0022002340465146FEF7D9FB10B1B7
:1082F0002D2384F84330914B9148B9F1470F94BF37
:1083000098468046032323612BF0040323604FF03B
:10831000000A009733460FAA2146284600F0D2F9FA
:10832000013040F08F804FF0FF3011B0BDE8F08F8A
:108330004246534640465146FEF7DAFB40B1BAF199
:10834000000FBCBF2D2384F843307E487E4BD4E71A
:1083500063685A1C09F0DF0142D1062363600022E2
:1083600006920EAACDE904920DAA4BF48063039203
:108370000DF13302CDE90132236063680093424678
:10838000534628460B91FFF7D5FE0B9947298046A7
:108390000D9908D1C81C02DB6368994240DDA9F140
:1083A00002095FFA89F9B9F1650F1FD801394A4608
:1083B00004F150000D91FFF71DFF0E9A1318012ACA
:1083C0008246236102DC2268D20701D50133236192
:1083D0009DF83330002B9CD02D2384F8433098E750
:1083E0004729BCD1002BBAD10123B7E7B9F1660FF9
:1083F00018D1002963680BDD216113B92268D00709
:1084000002D501330B442361A1654FF0000ADFE779
:1084100013B92268D20701D50233F4E70123F2E74A
:108420004FF067090E9B994205DB23682161D8074D
:10843000EAD54B1CE7E70029D4BFC1F102020122B3
:108440001344E0E723685A0507D4236942463146BE
:108450002846B84701302BD165E7B9F1650F40F2E6
:10846000DC80D4E9120100220023FEF70FFB002874
:1084700033D0364A012331462846B84701303FF40D
:1084800052AFDDE90D239A4202DB2368D8070FD5EE
:10849000DDE9092331462846B84701303FF443AFB0
:1084A0004FF0000804F11A090E9B013B434509DC1B
:1084B00023689B0700F10181E0680F9B9842B8BFD9
:1084C000184632E701234A4631462846B84701306C
:1084D0003FF429AF08F10108E6E70D9B002B37DCDC
:1084E0001A4A012331462846B84701303FF41BAFF2
:1084F000DDE90D23134302D12368D907D8D5DDE97F
:10850000092331462846B84701303FF40CAF4FF0FD
:10851000000904F11A0A0D9B5B424B4501DC0E9BDE
:1085200094E70123524631462846B84701303FF4CC
:10853000FAAE09F10109EEE7FFFFEF7F69E00208FB
:108540006DE0020875E0020871E002080AF1020815
:108550000E9AA36D9A42A8BF1A46002A914637DCAC
:108560004FF0000B29EAE97904F11A02D4F858A077
:10857000AAEB09035B4533DCDDE90D239A423BDBC3
:108580002368DA0738D40E9A0D99A2EB0A03A2EBFE
:1085900001099945A8BF9946B9F1000F34DC4FF0A5
:1085A000000829EAE97904F11A0ADDE90D239B1A8A
:1085B000A3EB090343457FF77BAF012352463146C6
:1085C0002846B84701303FF4AEAE08F10108ECE7A9
:1085D0001346314642462846B8470130C0D1A2E68C
:1085E0000123314628460B92B84701303FF49BAE39
:1085F0000B9A0BF1010BB9E7DDE909233146284657
:10860000B8470130BFD18EE64B4608EB0A0231462F
:108610002846B8470130C2D185E60E9A012A01DC0E
:10862000DB0737D50123424631462846B84701309B
:108630003FF479AEDDE9092331462846B8470130D9
:108640003FF471AED4E9120100220023FEF71EFAB6
:10865000D8B90E9B08F10102013B31462846B847C4
:1086600001300ED15FE601234A4631462846B8471D
:1086700001303FF458AE08F101080E9B013B434521
:10868000F1DC534604F15002E1E64FF0000804F13A
:108690001A09F2E701234246DFE701234A46314641
:1086A0002846B84701303FF43EAE08F10108E368C0
:1086B0000F995B1A4345F0DCFEE64FF0000804F129
:1086C0001909F4E72DE9F047164699468A680B69BF
:1086D000DDF820809342B8BF1346336091F8432001
:1086E00007460C460AB1013333602368990642BF3E
:1086F000336802333360256815F0060506D104F1AE
:10870000190AE36832689B1AAB4226DC94F84320CE
:10871000131E226818BF012392062BD404F14302D2
:1087200049463846C04701301ED02368E5683268A4
:1087300003F00603042B08BFAD1AA36822690CBF1F
:1087400025EAE57500259342C4BF9B1AED18002663
:108750001A34B5421AD1002008E001235246494696
:108760003846C047013003D14FF0FF30BDE8F087F5
:108770000135C6E7E1185A1C302081F84300224435
:1087800094F8451082F843100233C7E701232246CC
:1087900049463846C0470130E6D00136D9E70000E7
:1087A0002DE9FF470C469146277E0C99782F80468D
:1087B0009A4604F1430207D8622F0AD8002F00F02E
:1087C000D880582F00F0A38004F1420684F842704C
:1087D0003AE0A7F16303152BF6D801A050F823F077
:1087E000398800084D880008C9870008C987000833
:1087F000C9870008C98700084D880008C987000894
:10880000C9870008C9870008C98700085989000876
:108810007D8800083B890008C9870008C9870008CF
:108820007B890008C98700087D880008C98700087F
:10883000C9870008438900080B681A1D1B680A6075
:1088400004F1420684F842300123A3E02568086859
:108850002E0600F104030AD505680B60002D03DA2B
:108860002D236D4284F843305E480A2319E015F049
:10887000400F05680B6018BF2DB2EFE70B68256845
:10888000181D0860280601D51D6802E06906FBD5A1
:108890001D8854486F2F0CBF08230A23002184F839
:1088A00043106668A660002EA2BF216821F0040173
:1088B00021600DB9002E4DD01646B5FBF3F103FB38
:1088C0001157C75D06F8017D2F46BB420D46F4D90E
:1088D000082B0BD12368DF0708D52369616899420B
:1088E000DEBF302306F8013C06F1FF36921B226101
:1088F000CDF800A04B4603AA21464046FFF7E2FE12
:1089000001304CD14FF0FF3004B0BDE8F08735485E
:1089100084F8457023680E681F0656F8045B0E60E5
:1089200014D5D90744BF43F0200323601DB9236841
:1089300023F0200323601023B0E7236843F02003D3
:1089400023607823284884F84530E3E75E0648BF73
:10895000ADB2E6E71646BBE70B68266860691D1DE9
:108960000D6035061B6801D5186002E07106FBD565
:108970001880002323611646BAE70B681A1D0A60A7
:108980001E68626800213046FDF702FC08B1801BBA
:10899000606063682361002384F84330A8E723699B
:1089A000324649464046D0470130ABD023689B074A
:1089B00013D4E068039B9842B8BF1846A4E701238C
:1089C000324649464046D04701309BD00135E368E6
:1089D00003995B1AAB42F2DCEBE7002504F11906C0
:1089E000F5E700BF79E002088AE002082DE9F74FB9
:1089F00003690C69A3420746C0F28180013C01F182
:108A0000140800F1140505EB8403019358F8243091
:108A100055F8242001339A424FEA840B08EB84096D
:108A2000B2FBF3F631D34FF0000E4046AC46F246AF
:108A300050F8042B93B206FB03E34FEA134E9BB2AC
:108A4000AAEB0303120CDCF800A006FB02E213FA07
:108A50008AF34FEA124E1FFA82FADCF80020CAEBC2
:108A6000124202EB23429BB243EA024381454CF897
:108A7000043B4FEA224ADBD255F80B302BB9019B5D
:108A8000043B9D421A462ED33C61384601F059F80A
:108A9000002824DB013628464FF0000C58F8042B40
:108AA000D0F800E093B2ACEB0303120C13FA8EF390
:108AB000C2EB1E4202EB23429BB243EA0243C14592
:108AC00040F8043B4FEA224CE8D255F8242005EB4D
:108AD000840322B9043B9D421A460AD33C613046C6
:108AE00003B0BDE8F08F1268043B002ACCD1013CF2
:108AF000C7E71268043B002AF0D1013CEBE70020F5
:108B0000EEE70000000000002DE9F04F446A99B044
:108B100016461F46CDE90467DDF8948005463CB94A
:108B2000102000F0C7FDC0E9014468620460C46021
:108B30006B6A196851B15A684A60012393408B608F
:108B4000284600F009FE6B6A00221A603B1EB9BF7E
:108B500023F0004305930023C8F80030DDF814909B
:108B6000A74BBCBF0122C8F8002033EA090319D182
:108B7000249A42F20F731360C9F31303334300F0D6
:108B80006D85269B53B99F4B23E09F4B039308337E
:108B9000269A1360039819B0BDE8F08F994B0393A0
:108BA0000333F5E7DDE90434CDE90C34DDE90C01EC
:108BB00000220023FDF76AFF804660B1249A01235A
:108BC0001360269B002B00F04685904B269A13607D
:108BD000013B0393DEE716AB019317AB00932846E6
:108BE000DDE90C2301F03EF8C9F30A548346002C5A
:108BF0007ED00D9BCDF84C80C3F31303DDE90C014F
:108C000043F07F5141F44011A4F2FF34804B002225
:108C1000FDF71CFB74A3D3E90023FDF7CFFC74A37D
:108C2000D3E90023FDF714FB064620460F46FDF767
:108C30005BFC71A3D3E90023FDF7C0FC02460B46A1
:108C400030463946FDF704FB06460F46FDF766FF42
:108C500000228246002330463946FDF721FF48B105
:108C60005046FDF741FC32463B46FDF70FFF08B981
:108C70000AF1FF3ABAF1160F57D8664B03EBCA0355
:108C8000D3E90023DDE90C01FDF70AFF00284ED0EF
:108C90000AF1FF3A00230F93169B1C1B631E0993D6
:108CA00045BFC4F101030693002300234CBF099381
:108CB0000693BAF1000F3CDB099BCDF838A0534472
:108CC000099300230A93229B092B00F2B580052B00
:108CD000C4BF043B2293229BA3F10203CCBF002418
:108CE0000124032B00F2B480DFE803F02D987AA46E
:108CF000DDE916431C4404F23243202BC3BFC3F109
:108D0000400304F2124009FA03F3C3F12003C6BF83
:108D100026FA00F0184306FA03F0FDF7D5FB01230D
:108D2000A1F1F871013C139370E70123B3E70F90B1
:108D3000B2E7069BA3EB0A030693CAF100030A936A
:108D400000230E93BFE700230B93239B002B00F31C
:108D500082804FF00109CDF820904B46CDF88C90E1
:108D60006E6A00227260042202F114009842716857
:108D700077D9284600F0BCFC6B6A30601B6803930F
:108D8000089B0E2B00F2EE80002C00F0EB80BAF175
:108D9000000F7ADD1F4A0AF00F0302EBC303D3E989
:108DA00000341AF4807FCDE910344FEA2A145CD0E5
:108DB000194BDDE90C01D3E90823FDF729FDCDE9C5
:108DC000040104F00F040327134E002C4FD1DDE9FA
:108DD0001023DDE90401FDF71BFDCDE904016EE080
:108DE0000123B1E7AFF3008061436F63A787D23FF0
:108DF000B3C8608B288AC63FFB799F501344D33F8A
:108E00000000F07FA4E002089BE002080BF10208DA
:108E10000000F83FD0E00208A8E0020800230B930E
:108E2000239B0AEB030909F10103012B0893B8BF47
:108E3000012395E70123F2E70124002322930B94F9
:108E40004FF0FF390022CDF820901223239287E7BC
:108E500001230B93F4E7DDF88C90CDF820904B467E
:108E60007EE70131716052007EE70227ACE7E1073F
:108E700008D5DDE91001D6E90023FDF79FFBCDE918
:108E800010010137641008369FE700F0A580CAF191
:108E90000004A44BA44E04F00F0203EBC203D3E979
:108EA0000023DDE90C01FDF789FBCDE90401241164
:108EB00000230227002C40F08480002B8DD10F9BD3
:108EC000002B00F08B80DDE90434CDE91034DDE9BE
:108ED0001001964B0022FDF7E3FD00287ED0089B91
:108EE000002B7BD0B9F1000F38DDDDE91001904B8C
:108EF0000022FDF763FBCDE904010AF1FF380137D9
:108F00004C463846FDF7F0FADDE90423FDF756FB41
:108F1000884B0022FDF79CF9A1F15076CDE91001B4
:108F20001196002C5DD1DDE90401834B0022FDF791
:108F30008DF902460B46CDE90423109A3346FDF71E
:108F4000CDFD002840F09782DDE90401109A06F17A
:108F50000043FDF7A5FD002840F08B82DDE90C34CD
:108F6000CDE90434179B002BC0F25181BAF10E0FEA
:108F700000F34D816B4B03EBCA03D3E90034CDE919
:108F80000634239B002B80F2DB80089B002B00F330
:108F9000D78040F06D82684B0022DDE90601FDF7C5
:108FA0000DFBDDE90423FDF78FFD089C2646002814
:108FB00040F04382039F312307F8013B0AF1010A85
:108FC0003FE2E20705D5D6E90023FDF7F7FA0137BE
:108FD0000123641008366DE7022770E7089CD0462D
:108FE0008FE703994F4B214412910B9903EBC40374
:108FF000DDE9106753E90223002946D04F490020DC
:10900000FDF706FC3B463246FDF720F9CDE910019D
:10901000039FDDE90401FDF781FD0446FDF764FAD5
:1090200002460B46DDE90401FDF710F93034024633
:109030000B46CDE9042307F8014BDDE91023FDF7CA
:109040002FFD002865D1DDE9042338490020FDF714
:10905000FDF8DDE91023FDF723FD002840F0B68080
:10906000129B9F423FF47AAFDDE91001304B0022A2
:10907000FDF7A4FA2E4BCDE910010022DDE9040131
:10908000FDF79CFACDE90401C3E730463946FDF708
:1090900095FACDE91001129B039C1493DDE90401BC
:1090A000FDF73CFD1590FDF71FFA02460B46DDE982
:1090B0000401FDF7CBF8159B303304F8013B129BFC
:1090C0009C4206460F464FF0000224D11B4BDDE9BF
:1090D0001001FDF7BDF802460B4630463946FDF754
:1090E000FDFC002871D1DDE9102314490020FDF7B3
:1090F000ADF802460B4630463946FDF7D1FC002854
:109100003FF42CAF149F7B1E149317F8013C302BB7
:10911000F8D0C24649E0064BFDF750FACDE904010C
:10912000BCE700BFD0E00208A8E002080000F03F62
:109130000000244000001C40000014400000E03FFC
:10914000DDE90489039FDDE9062340464946FDF732
:109150005FFBFDF7E3FC0446FDF7C6F9DDE90623F6
:10916000FDF72CFA04F130060B460246494640460C
:10917000FDF76CF807F8016B039E089BBE1BB3421A
:1091800038D102460B46FDF763F8DDE90623804639
:109190008946FDF7A3FC58BBDDE906234046494656
:1091A000FDF774FC08B1E10722D42846594600F0C7
:1091B000D3FA00233B70249B0AF101001860269B20
:1091C000002B3FF4E7AC1F60E4E427463B461F4614
:1091D00013F8012D392A07D1039A9A42F7D103993E
:1091E000302208F101080A701A7801321A7090E7EB
:1091F000D046EBE7A14B0022FDF7E0F90022002367
:1092000080468946FDF742FC00289CD0CDE70B9AAA
:10921000002A00F0CD80229A012A00F3AF80139A31
:10922000002A00F0A78003F233430A9C069F069AA7
:109230001A440692099A01211A442846099200F01C
:109240002EFB0646002F0CDD099B002B09DDBB42DF
:10925000069AA8BF3B46D21A0692099AFF1AD31A59
:1092600009930A9BF3B10B9B002B00F0A580002C07
:1092700010DD31462246284600F0B6FB5A4601462C
:109280000646284600F014FB59468046284600F062
:1092900063FAC3460A9B1A1B04D05946284600F0BD
:1092A000A3FB83460121284600F0F9FA0E9B002B10
:1092B000044640F383801A460146284600F094FB9A
:1092C000229B012B04467CDD4FF00008236904EB50
:1092D0008303186900F095FAC0F12000099B184437
:1092E00010F01F0000F08E80C0F12003042B40F32B
:1092F0008780C0F11C00069B03440693099B03442E
:1093000007440993069B002B05DD59461A4628465B
:1093100000F0B8FB8346099B002B05DD21461A4669
:10932000284600F0AFFB04460F9B002B6CD0214673
:10933000584600F006FC002866DA002359460A2247
:10934000284600F020FA0B9B0AF1FF3A8346002BD7
:1093500000F08B81314600230A22284600F013FAE0
:10936000B9F1000F064600F39180229B022B40F3D7
:109370008D8051E0169BC3F1360356E7089B5C1EB7
:109380000A9BA342BFBF0A9B0A94E21A0E9BB6BF78
:109390009B181C1B0E93089BB8BF0024002BB9BF61
:1093A000069B089A069F089BBCBF9F1A00233EE7B6
:1093B0000A9C069F0B9E45E70A9A6EE7229B012BAB
:1093C00019DC049BBBB9059BC3F313039BB9059B35
:1093D00023F000431B0D1B0583B1069B013306934D
:1093E000099B013309934FF001080E9B002B7FF47A
:1093F0006DAF012072E74FF00008F6E79846F4E7FA
:1094000080D018461C3076E7089B002B38DC229B66
:10941000022B35DDDDF82090B9F1000F0DD121468A
:109420004B460522284600F0AEF901460446584650
:1094300000F087FB00283FF7BDAD239B039F6FEA39
:10944000030A4FF000082146284600F085F9002E57
:109450003FF4ABAEB8F1000F05D0B04503D04146A4
:10946000284600F079F93146284600F075F99CE667
:1094700000242646E1E7C24626469BE5000024403C
:109480000B9BDDF82090002B00F0F680002F05DD0F
:1094900031463A46284600F0F5FA0646B8F1000F84
:1094A00055D07168284600F023F932690232074628
:1094B000920006F10C010C3000F00CF90122394643
:1094C000284600F0DFFA039B01330893039B4B44CB
:1094D0000A93049B03F00103B04609930646089BD8
:1094E0002146013B58460493FFF780FA0346303388
:1094F0000690414658460B9300F023FB32468146C6
:109500002146284600F038FBC2680B9B074602BB89
:109510000146584600F015FB0B9B0246394628468B
:10952000CDE90B3200F018F9229B0C9A089F43EA10
:109530000201099B0B430B9B0DD1392B29D0B9F1AB
:10954000000F01DD069B3133049A13707BE7304630
:10955000B9E70122E2E7B9F1000F06DB229941EAFF
:109560000909099959EA010120D1002AECDD59467F
:1095700001222846089300F085FA2146834600F030
:10958000E0FA0028089B02DCDED1DA07DCD5392BB3
:10959000D8D1049A392313703B461F46013B17F874
:1095A000012C392A50D001321A704CE7002A03DD11
:1095B000392BEED00133C7E7089A0A9902F8013C2B
:1095C0008A422AD0594600230A22284600F0DBF8B6
:1095D000B04583464FF000034FF00A02414628464B
:1095E00007D100F0D0F880460646089B0133089367
:1095F00075E700F0C8F83146804600230A22284665
:1096000000F0C1F80646F0E7B9F1000F039ACCBFAD
:109610004F46012717444FF00008594601222846BB
:10962000089300F02FFA2146834600F08AFA0028BA
:10963000B2DC02D1089BDB07AED43B461F4613F8D1
:10964000012D302AFAD0FEE6039A9A42A5D10AF1FA
:10965000010A312379E7134BFFF7BBBA269B002B96
:109660007FF493AA104BFFF7B4BAB9F1000F03DCF3
:10967000229B022B3FF7D0AE039F21465846FFF7AF
:10968000B5F900F1300307F8013B039ABA1A914586
:10969000BADD594600230A22284600F074F88346B2
:1096A000EBE700BF0AF102089BE0020800487047A0
:1096B000E0010020024B0146186800F07FBB00BFAC
:1096C0008C000020024B0146186800F029BB00BF47
:1096D0008C0000200A44914200F1FF3300D1704712
:1096E00010B511F8014B03F8014F9142F9D110BDAB
:1096F00070B5466A04460D463EB91020FFF7DAFF02
:10970000C0E9016660620660C660666AF36883B19C
:10971000636ADB6853F82500B8B9012101FA05F640
:10972000721D9200204600F0ECFA60B1C0E90156CB
:109730000EE021220421204600F0E3FA636AF06083
:10974000DB68002BE4D1002070BD026843F82520BF
:109750000023C0E90333F7E770B5466A05460C46B7
:109760003EB91020FFF7A6FFC0E9016668620660F7
:10977000C6603CB16B6A6268DB6853F822102160F6
:1097800043F8224070BD2DE9F0410E690746984626
:109790000C4601F1140000230568A9B202FB018107
:1097A0004FEA114C2D0C02FB05C589B2013301EBC8
:1097B00005419E4240F8041B4FEA1548ECDCB8F125
:1097C000000F1BD0A368B34212DC61683846013138
:1097D000FFF78EFF2269023204F10C010546920068
:1097E0000C30FFF777FF21463846FFF7B5FF2C46D0
:1097F00004EB86030136C3F8148026612046BDE8D9
:10980000F081020C12040346CAB90304102013F0BD
:109810007F4F04BF1B02083013F0704F04BF1B01C1
:10982000043013F0404F04BF9B000230002B05DBD7
:1098300013F0804F00F1010008BF20207047002086
:10984000E5E70368024613F007000BD0D90722D4DE
:10985000980749BF5B089B08012013605CBF136039
:109860000220704799B209B91B0C102013F0FF0FAA
:1098700004BF1B0A0830190704BF1B0904309907ED
:1098800004BF9B080230D90703D45B0800F1010034
:1098900003D013607047002070472020704710B538
:1098A0000C460121FFF724FF01224461026110BD33
:1098B0002DE9F04F15460A692B699A42B8BF0B464D
:1098C0000C46BCBF2C461D462769D5F81090A368EE
:1098D000616807EB0906B342B8BF013185B0FFF7F5
:1098E00007FF00F1140101EB86080B4600224345F7
:1098F0001DD304F1140305F1140203EB870702EBF7
:10990000890302933B1B153B23F00303043304F14B
:109910001505AF4238BF04230193029B0392934283
:1099200008D8002E5ADC066105B0BDE8F08F43F878
:10993000042BDCE7B2F800A0BAF1000F24D004F148
:10994000140E89464FF0000C5EF8045BD9F800B0A5
:10995000ABB21FFA8BFB0AFB03B34FEA154BD9F8E6
:10996000005063444FEA154C0AFB0BC505EB134549
:109970009BB243EA0543774549F8043B4FEA154C4F
:10998000E2D8019B41F803C0039BB3F80290043274
:10999000B9F1000F20D00B6804F1140C8E464FF083
:1099A000000ABCF80050BEF802B009FB05B5AA4495
:1099B0009BB243EA0A434EF8043B5CF8043BBEF812
:1099C00000501B0C09FB035303EB1A4367454FEA96
:1099D000134AE6D8019D4B5104319EE758F8043DE7
:1099E000002BA0D1013E9CE72DE9F843154612F06B
:1099F000030206460F4607D0214C013A002354F8D3
:109A00002220FFF7C0FE0746AD1035D0746A3CB97E
:109A10001020FFF74FFEC0E9014470620460C4608B
:109A2000D6F82480D8F808404CB940F2712130466D
:109A3000FFF735FF0023C8F80800044603604FF025
:109A40000009EB070AD5394622463046FFF730FFBA
:109A5000394680463046FFF77FFE47466D100BD0F3
:109A6000206838B9224621463046FFF721FF2060A2
:109A7000C0F800900446E4E73846BDE8F88300BF2C
:109A800098E102082DE9F0470C464968236903EB89
:109A90006218A368074691464FEA621A08F1010668
:109AA000B3423FDB3846FFF723FE0023054600F1B3
:109AB000140100F110021846534536DB20692AEAEA
:109AC000EA7A04F1140319F01F0901EB8A0103EB90
:109AD000800C2ED0C9F1200E8A460022186800FAA8
:109AE00009F002434AF8042B53F8042B9C4522FA50
:109AF0000EF2F3D8ACEB0403153B23F0030304335D
:109B000004F11500604588BF0423CA500AB108F16A
:109B10000206013E38462E612146FFF71DFE28460B
:109B2000BDE8F08701315B00BAE742F8040F01336A
:109B3000C2E7043953F8042B41F8042F9C45F9D8A7
:109B4000E7E70A6903460069801A30B50DD114337E
:109B5000143103EB820401EB820154F8045D51F8E7
:109B6000042D954202D004D3012030BDA342F4D38A
:109B7000FBE74FF0FF30F8E72DE9F84F0C460646BB
:109B8000114620461746FFF7DCFF051E08D129467F
:109B90003046FFF7ADFD0123C0E90435BDE8F88F7D
:109BA000A4BF3B46274630467968A6BF1C46002521
:109BB0000125FFF79DFD3E69C560256907F1140188
:109BC00004F1140900F1140E07F1100201EB860CE8
:109BD00009EB8505F246002759F8043B52F804BF0B
:109BE0001FFA83F817FA8BF71B0CA7EB0808C3EBD7
:109BF0001B4303EB28431FFA88F81F144D4548EA1E
:109C000003434AF8043BE7D82B1B153B23F003031F
:109C100004331534A54238BF0423194473449E46C7
:109C20000D4665450ED30CF10302521A22F00302D1
:109C300003398C4538BF00221A4452F8043D7BB1E9
:109C40000661ABE755F8048B17FA88F4221402EB8F
:109C50001842A4B244EA02444EF8044B1714E0E759
:109C6000013EEAE72DE9F34101211C46DDE90865E3
:109C70009046FFF73DFDC4F31303C4F30A540746AF
:109C80002CBB0193B8F1000326D068460093FFF780
:109C9000D8FD0099F0B1019AC0F1200302FA03F354
:109CA0000B43C2407B610192019BBB61002B14BF3F
:109CB000022101213961C4B1A4F233440444C0F14A
:109CC000350034602860384602B0BDE8F08143F4C6
:109CD0008013D6E77961E7E701A8FFF7B2FD019BA2
:109CE0007B61012139612030E5E707EB8103A0F2B8
:109CF000324030601869FFF784FDC0EB41112960E4
:109D0000E1E738B502FB01F5294600F057F80446B3
:109D100018B12A460021FEF705FA204638BD00009A
:109D200038B50546002945D051F8043C0C1F002BDE
:109D3000B8BFE41800F0BEF81F4A1368104633B9E4
:109D4000636014602846BDE8384000F0B9B8A3420B
:109D50000BD921686218934204BF1A685B6863607C
:109D600004BF521822600460ECE71A465B680BB12E
:109D7000A342FAD911685018A0420BD120680144BF
:109D8000501883421160DDD118685B68536001444C
:109D90001160D7E702D90C232B60D3E72068211884
:109DA0008B4204BF19685B68636004BF09182160B7
:109DB0005460C7E738BD00BF740E0020F8B5CD1C55
:109DC00025F0030508350C2D38BF0C25002D06465F
:109DD00001DBA94203D90C2333600020F8BD00F059
:109DE00069F821490A6814469CB9204F3B6823B999
:109DF0002146304600F03CF838602946304600F0F5
:109E000037F8431C23D10C233360304600F058F858
:109E1000E3E723685B1B17D40B2B03D923601C4497
:109E2000256004E06368A2420CBF0B6053603046BB
:109E300000F046F804F10B00231D20F00700C21AC1
:109E4000CCD01B1AA350C9E722466468CCE7C41CD7
:109E500024F00304A042E3D0211A304600F008F8B1
:109E60000130DDD1CFE700BF740E0020780E002056
:109E700038B5064D0023044608462B6000F036F83E
:109E8000431C02D12B6803B1236038BDF467002066
:109E900082B001B901A942B14BB113780B601278BD
:109EA000101E18BF012002B070471046FBE76FF08C
:109EB0000100F8E7014800F016B800BFFC67002079
:109EC000014800F011B800BFFC67002003460846B7
:109ED00041B1FF2A04D98A221A604FF0FF3070473F
:109EE0000A7001207047704770470000044A054916
:109EF0001368002B08BF0B461844106018467047C3
:109F00007C0E002068850020FDF7EEBAFDF7A4BBAB
:109F10000D4885461BF01EFF0C480D490D4A0023D5
:109F200002E0D458C4500433C4188C42F9D30A4A0E
:109F30000A4C002301E013600432A242FBD3FEF777
:109F4000CDF8FDF765FFFEE700FC002000000020D3
:109F5000300E002090150308300E00206885002088
:109F600000F05AB80368074A934206D1DA69D2066C
:109F700006D510221A6201F08FBA034A9342F5D037
:109F8000704700BF00800040003801404FF0B043F0
:109F90004FF0FF319A6B9963DA6BD9639A6B0022A9
:109FA0009A63D86BDA63186C1964186C1A64586C6D
:109FB0005964586C5A64986A9962986A9A62D86A25
:109FC000D962D86ADA62186B1963196B1A635A6C12
:109FD00042F001025A645A6C22F001025A64D3F82A
:109FE000902042F48032C3F89020D3F8902022F4DD
:109FF0008032C3F89020BFF34F8F0549054BCA68E4
:10A0000002F4E0621343CB60BFF34F8F00BFFDE764
:10A0100000ED00E00400FA054FF0B0434FF0FF31CF
:10A020009A6B9963DA6BD9639A6B00229A63D86B47
:10A03000DA63186C1964186C1A64586C5964586C9B
:10A040005A64986A9962986A9A62D86AD962D86A98
:10A05000DA62186B1963196B1A635A6C42F00102C9
:10A060005A645A6C22F001025A64D3F8902042F4E8
:10A070008032C3F89020D3F8902022F48032C3F8C5
:10A080009020FEE7FEE7FEE7FEE77047704708F026
:10A09000E1BB000001480BF0A5B800BF346A002006
:10A0A00001480CF060BA00BFE867002001480BF0DF
:10A0B00061BA00BF346A002001480AF0D3B900BF7A
:10A0C0001C6E002001480AF0CDB900BF6C6A002068
:10A0D00001480AF0C7B900BFCC6A002001480AF065
:10A0E000C1B900BF2C6D002010B5044C20460CF007
:10A0F00065FB2046BDE81040FFF734BF8C6D0020A3
:10A10000704701200AF036BB02200AF033BB04205E
:10A110000AF030BB08200AF02DBB10200AF02ABB41
:10A120000E4BDA68920602D520200AF023BBDA68CB
:10A13000500601D54020F8E7DA68110601D58020E5
:10A14000F3E7DA68D20502D54FF48070EDE7DB68FB
:10A150009B0502D54FF40070E7E7704700080058F0
:10A16000134BDA68510503D54FF480600AF002BB47
:10A17000DA68120502D54FF40060F7E7DA68D00418
:10A1800002D54FF48050F1E7DA68910402D54FF41C
:10A190000050EBE7DA68520402D54FF48040E5E75F
:10A1A000DB681B0402D54FF40040DFE7704700BFB7
:10A1B0000008005810B5044C20460CF0FFFA204669
:10A1C000BDE81040FFF7CEBE9C6C0020014809F0AE
:10A1D00015BD00BF286900204FF0B04382B0DA6C93
:10A1E0000243DA64DB6C18400190019B02B07047B7
:10A1F0001FB514284FF00003CDE902330C460CD8EC
:10A20000092812D90A380A280FD8DFE800F07B0E97
:10A210000E0E0E820E0E74116D00FE2800F083806B
:10A22000FF2800F08280FD287AD06FF0030059E00B
:10A230003F4A404B0193137843F0010313703E48AB
:10A240003E4A4FF00043C0E900233D4B04221B6807
:10A250008360426100230122C2614FF480510622D3
:10A260000383C0E90333C0E90933C0E90C128376E4
:10A2700080F8203080F82C30836380F83C30C36451
:10A2800008F034FB08B100F07FFE2B4808F0D6FE42
:10A2900008B100F079FE0023274801A9CDE9023377
:10A2A00008F0A6FC08B100F06FFE234808F0FAFDA4
:10A2B00008B100F069FE0A211F4808F03BFC1E4867
:10A2C00008F09EFE1C4808F090FC1E4B019A80B2DC
:10A2D0009A42208004BF00EB40002080164808F01E
:10A2E00043FE002004B010BD114A174B01931378B0
:10A2F00043F00203A2E70E4A144B0193137843F094
:10A3000004039BE70A4A124B0193137843F00803B6
:10A3100094E7074A0F4B0193137843F010038DE73E
:10A320000D4B01938BE70D4BFBE7064BF9E700BFA5
:10A33000800E002004000008046800200024014072
:10A340005C020020004000B80800000C1000001063
:10A35000400000180008002C001000B0002000B4DD
:10A3600070477047014B1878704700BF61020020AA
:10A37000014B1878704700BF6002002010B50446FA
:10A3800086B01422002101A8FDF7CCFE22685E4BA6
:10A390009A4240F08E804FF0B0435C4C1A6E42F40B
:10A3A00000721A661B6E03F400730093009B2378FF
:10A3B000DA0708D5132000F079FAB0F1904F7AD17E
:10A3C0000120FFF709FF23789B0708D5142000F030
:10A3D0006DFAB0F1904F76D10120FFF7FDFE2378A2
:10A3E000580708D5122000F061FAB0F1904F72D1F1
:10A3F0000120FFF7F1FE2378190708D50A2000F0A5
:10A4000055FAB0F1904F6ED10120FFF7E5FE2378A9
:10A41000DA0608D50F2000F049FAB0F1904F6AD162
:10A420000120FFF7D9FE00234FF0030CCDE902C352
:10A430002378DB0709D5132000F03DFA01901320A3
:10A4400000F034FA01A90AF069F82378980709D5D1
:10A45000142000F030FA0190142000F027FA01A92E
:10A460000AF05CF82378590709D5122000F023FA86
:10A470000190122000F01AFA01A90AF04FF823788F
:10A480001A0709D50A2000F016FA01900A2000F0F8
:10A490000DFA01A90AF042F82378DB0609D50F204E
:10A4A00000F009FA01900F2000F000FA01A90AF06B
:10A4B00035F806B010BD132000F0F8F9144B98429F
:10A4C00081D102207DE7142000F0F0F9104B984272
:10A4D00085D1022081E7122000F0E8F90C4B984268
:10A4E00089D1022085E70A2000F0E0F9084B984264
:10A4F0008DD1022089E70F2000F0D8F9044B984253
:10A5000091D102208DE700BF00240140800E002081
:10A510000004004838B50268324B9A4260D14FF0CF
:10A52000B042314C136E23F4007313662378DD07B9
:10A530000ED5132000F0BAF90546132000F0BBF940
:10A54000014628460AF096F8237823F00103237089
:10A55000237898070ED5142000F0A8F9054614209A
:10A5600000F0A9F9014628460AF084F8237823F080
:10A5700002032370237859070ED5122000F096F9B4
:10A580000546122000F097F9014628460AF072F8B5
:10A59000237823F00403237023781A070ED50A20AA
:10A5A00000F084F905460A2000F085F901462846A6
:10A5B0000AF060F8237823F0080323702378DB0681
:10A5C0000ED50F2000F072F905460F2000F073F948
:10A5D000014628460AF04EF8237823F01003237032
:10A5E00038BD00BF00240140800E00200A4B00F15E
:10A5F0001002C1781970817859704178997010F8FB
:10A60000041BD970904203F10403F2D1034B1022D2
:10A610001A800020704700BF840E002062020020D4
:10A620002DE9F04F3B4EDFF8F4C085B002AF044691
:10A6300090469A46384AF26000233046C6E900C385
:10A64000C6E909333D8ED7F834B0B36089467361EB
:10A65000F36208F0FBFE304A7A6008B100F094FC27
:10A660002C4808F016FF08B100F08EFC2B4804229D
:10A67000C6E900020022B260002C39D174610022C8
:10A680007B682448F3600121C6E90912F26208F0F0
:10A69000DDFE08B100F078FC2B071DBF25F00F048C
:10A6A0001034A4B22C46A300073323F00703ADEB0C
:10A6B000030D02AE224600213046FDF733FD2A4647
:10A6C00051463046FFF706F8FF23009311485B46DA
:10A6D00022463146B9F1000F14D109F031F970B9B1
:10A6E0000C4808F0D6FE80B90C37BD46BDE8F08FA7
:10A6F000012C0CBF20224022C6E90482BFE76FF084
:10A700000600F1E709F0AAF9E9E700F03DFC0020B6
:10A71000EAE700BF28690020940E002000180058C6
:10A7200021F00803102B01D0202911D10A4B00F190
:10A730001002C1781970817859704178997010F8B9
:10A74000041BD970904203F10403F2D1002070473A
:10A750006FF01F00704700BF940E002007B5CDE9D1
:10A7600000120022034611461046FFF759FF03B0BE
:10A770005DF804FB70B586B004460D461646002110
:10A78000102202A8FDF7CEFC074B08491A8802A840
:10A79000FEF7A0FFCDE90056234602AA00210120C2
:10A7A000FFF73EFF06B070BD62020020840E00205D
:10A7B00070B586B004460D4616460021102202A848
:10A7C000FDF7B0FC074B08491A8802A8FEF782FF84
:10A7D0000121CDE90056234602AA0846FFF720FFD3
:10A7E00006B070BD62020020840E002008B5FFF79D
:10A7F00097FFC0B208BD08B510230A461946FFF7F7
:10A80000ADFFC0B208BD70B51446054618460E46E9
:10A81000FFF7ECFE23019BB2324619462846FFF7AC
:10A82000A9FFC0B270BD70B51446054618460E4665
:10A83000FFF7DCFE23019BB2324619462846FFF79C
:10A84000B7FFC0B270BD0000034B00221A70034B6B
:10A8500001221A70704700BF9C7D0020207E0020DE
:10A86000024B53F8203003B118477047A41600205C
:10A87000002201230342D1B202F101020DD02F299F
:10A880000ED8084B084800221A70082300F831300F
:10A8900000EBC100416007F073BF5B009BB2E9E7CA
:10A8A000704700BF9C7D002024160020000900F5A1
:10A8B00090108002704700F00F030120984080B292
:10A8C000704700002F2870B503461CD81424444359
:10A8D0000D4A03F00F060125B54015511019022548
:10A8E00000240129C0E9024501D1416001E00029AD
:10A8F000FBD01846FFF7DAFF1421BDE8704001FBDA
:10A90000032109F00BBE70BDA40E00202F2870B5E6
:10A9100004460D4624D8FFF7C9FF012304F00F01B8
:10A9200003FA01F1064609F0A5FE0E4A142325B9E3
:10A9300003FB04230221996004E0012D0AD103FBEB
:10A9400004239D60142101FB04213046BDE87040C2
:10A9500009F0E4BD022DF5D103FB04230021EAE751
:10A9600070BD00BFA40E00202F2808B50A4603467C
:10A9700015D851B9FFF79AFF012103F00F03994051
:10A9800089B2BDE8084009F0EFBE012907D1FFF701
:10A990008DFF03F00F0301FA03F399B2F1E708BD4D
:10A9A0002F28F8B5054600F28280414E142242431A
:10A9B00000F00F040123B018A340B35003294FF057
:10A9C0000202C2602DD801292ED94FF488124260AC
:10A9D0002846FFF76BFFC76893FAA3F2B2FA82F238
:10A9E000510003228A403A4093FAA3F3B3FA83F367
:10A9F0005B0022FA03F3012B4FF014021ED0022B4E
:10AA00001CD0142101FB056109F088FDD4B9062092
:10AA10002246022108F070FB0620BDE8F84008F04D
:10AA20009DBB0439012906D9142202FB05624FF4AB
:10AA300044115160CCE74FF40412C8E702FB0562F1
:10AA40009360DEE7012C06D107200022022108F0E6
:10AA500053FB0720E1E7022C06D108200022214603
:10AA600008F04AFB0820D8E7032C06D10920002271
:10AA7000022108F041FB0920CFE7042C06D10A206F
:10AA80000022022108F038FB0A20C6E7053C042C0E
:10AA90004FF000024FF0020104D8162008F02CFB02
:10AAA0001620BAE7292008F027FB2920B5E7F8BDD2
:10AAB000A40E0020044B00F00F0053F820200AB928
:10AAC00043F8201000207047A41600202DE9F84319
:10AAD000184E194D194FDFF86C80DFF86C90002488
:10AAE0000F2C07DDA4F11103152B19D829FA03F354
:10AAF000DB0715D557F8243093B973682B60B3681A
:10AB00006B60F368AB603369EB602B7C43B198F802
:10AB100000102046FFF744FF09492046FFF7CAFF0F
:10AB20000134302C06F1140605F11405D8D1BDE826
:10AB3000F88300BFA40E002064120020A416002099
:10AB400049A80008640200207F7C38002DE9F0410C
:10AB5000144E154D154FDFF8588000240F2C07DDDB
:10AB6000A4F11103152B14D828FA03F3DB0710D531
:10AB700057F824306BB933686B607368AB60B368A7
:10AB8000EB602046F3682B61FFF790FE294609F041
:10AB9000C5FC0134302C06F1140605F11405DDD195
:10ABA000BDE8F08164120020A40E0020A41600204D
:10ABB0007F7C380000B58DB02C22002101A8FDF764
:10ABC000B1FA1748174B03604FF080420023C0E9E9
:10ABD0000433C0E90723836083614FF480734362C9
:10ABE0000AF07EFB08B100F0CFF90D480AF09CFC9A
:10ABF00008B100F0C9F94FF07C53002207930848D0
:10AC000008924FF4807301A9029206920B930AF006
:10AC1000C3FB08B100F0B8F900200DB05DF804FBEB
:10AC2000346A00200028004007B5074B0DF10600EC
:10AC30001B699847BDF806304FF47A7202FB00306A
:10AC4000002103B05DF804FB1CDF02087047704769
:10AC500008B50A480AF0D8FD002211460C2008F079
:10AC60004BFA0C2008F07AFA00220D20114608F069
:10AC700043FABDE808400D2008F070BA68020020D1
:10AC80007047000038B5054D002415F8013B0BB1A5
:10AC9000FFF7DEFF0134042CF7D138BD6417002024
:10ACA00070B50D461446064607F00AFE306007F000
:10ACB0000DFE286007F010FE206070BDBFF34F8FBF
:10ACC0000549064BCA6802F4E0621343CB60BFF348
:10ACD0004F8F00BFFDE700BF00ED00E00400FA0564
:10ACE00072B6EFF3108303607047036883F3108834
:10ACF00062B670477047000008B504480EF0CAFB02
:10AD0000002814BF6FF00600002008BD681700205F
:10AD1000084A0346002108481170042200F8332035
:10AD2000064A00EBC3000C2101FB0323436007F03C
:10AD300027BD00BF9C7D0020A81700200C18002014
:10AD4000084A0346002108481170052200F8332004
:10AD5000064A00EBC3000C2101FB0323436007F00C
:10AD60000FBD00BF9C7D002080170020D017002061
:10AD700083680BB1406818477047003818BF01203E
:10AD800070470EF01BBB000037B503460C2410467D
:10AD90000E4A5C431519042B135598BF0C4AA96041
:10ADA00094BF52F823400024FFF7E7FF4FF0FF3134
:10ADB000024600932046074B0EF00AFB002814BF02
:10ADC0006FF00600002003B030BD00BF0C1800205B
:10ADD000ACE2020811AD0008042898BF0D4B70B515
:10ADE00098BF53F820400C4D4FF00C0303FB00F3C9
:10ADF00005EB030688BF0024E854726020460EF07D
:10AE0000D3FB18B920460EF095FB08B16FF0060091
:10AE100070BD00BFACE202080C180020042898BFE7
:10AE20000B4A08B5034698BF52F82000094A4FF074
:10AE30000C0101FB03234FF0000288BF00205A6081
:10AE40000EF028FB002814BF6FF00600002008BD9C
:10AE5000ACE202080C18002037B503460C2410465B
:10AE60000E4A5C431519042B135598BF0C4AA96070
:10AE700094BF52F823400024FFF77FFF4FF0FF31CB
:10AE8000024600932046074B0EF0A2FA002814BF9A
:10AE90006FF00600002003B030BD00BFD0170020C7
:10AEA000C0E2020841AD0008042898BF0D4B70B500
:10AEB00098BF53F820400C4D4FF00C0303FB00F3F8
:10AEC00005EB030688BF0024E854726020460EF0AC
:10AED0006BFB18B920460EF02DFB08B16FF0060091
:10AEE00070BD00BFC0E20208D0170020042898BF40
:10AEF0000B4A08B5034698BF52F82000094A4FF0A4
:10AF00000C0101FB03234FF0000288BF00205A60B0
:10AF10000EF0C0FA002814BF6FF00600002008BD34
:10AF2000C0E20208D0170020BFF34F8F0549064B3F
:10AF3000CA6802F4E0621343CB60BFF34F8F00BFD7
:10AF4000FDE700BF00ED00E00400FA054FF0B0435C
:10AF500082B09A6C02439A649B6C18400190019BEA
:10AF600002B0704710B5064C0649802220460CF00E
:10AF700051F92268136843F01003136010BD00BF3D
:10AF80009C6C00201C6C002008B5FFF7CDFF000072
:10AF9000012810B50BD1094C0949802220460CF03C
:10AFA00039F92268136843F01003136010BD0228BA
:10AFB000FCD1BDE81040FFF7D5BF00BF8C6D00206D
:10AFC0007D6E00202DE9F04385B0012B9DF83050B7
:10AFD0009DF8348014BF00274FF40057012D04461C
:10AFE0000E463DD0032D3ED0002D3FD00025013A26
:10AFF000D2B2022A3CD8614B53F82290012C69D17D
:10B000000420FFF7A3FF2046FFF7A0FF0022114610
:10B010000E2008F071F80E2008F0A0F8584B59489F
:10B0200083F80180584B0561C0E900360C240023E9
:10B03000C0E90297C0E90543C0E907334362B8F1AC
:10B04000000F1BD0B8F1020F01BF082383624FF439
:10B05000004383634B480CF057F8A0B1FFF764FF3F
:10B060004FF4C065C3E74FF48065C0E7022A02D001
:10B070004FF00009C2E74FF08059BFE7C0F82880C1
:10B080000CF012F8E9E700213E480CF09FF9014668
:10B090000028E3D13B480CF0BDF90028DED1394847
:10B0A0000CF079F90028D9D10120FFF771FF4FF496
:10B0B0004013019A3348009319460CF0F9F8002820
:10B0C000CCD14FF0B042936843F40043936005B095
:10B0D000BDE8F083022CFAD1294B2C4C83F8028076
:10B0E0000420FFF733FF0120FFF730FF0022114655
:10B0F0000B2008F001F80B2008F030F8244B2561F4
:10B10000C4E900360C2200232046C4E90297C4E9B2
:10B110000523C4E90833A36263660BF0C5FF01464B
:10B1200000289BD120460CF051F90146002895D10A
:10B1300020460CF06FF9002890D120460CF02BF936
:10B1400000288BD1FFF70EFF4FF44013029304AB9E
:10B1500013E9060020460CF0ABF800287FF47EAF20
:10B160000C4AD2F8803043F08053C2F88030226815
:10B17000936843F480039360A3E700BFD4E202081E
:10B18000801C00208C6D0020003801409C6C002049
:10B1900000800040000800582DE9F7439DF82890F2
:10B1A0009DF82C40CDE9009416461D4680460F467A
:10B1B0000C24FFF707FF074B04FB08F01C180122C3
:10B1C0001A5467602672657284F80A9003B0BDE86D
:10B1D000F08300BF5C1C0020022810B5044605D196
:10B1E00007480BF051FA28B1FFF79EFE012801D164
:10B1F0000448F6E70C20044B444300221A5510BDC6
:10B200009C6C00208C6D00205C1C00200128F8B58F
:10B2100005460E461F462BD194B2184A5278013A81
:10B22000012A17D816480BF090FC224614483B46DA
:10B2300031460BF0A9FE044611480BF0ACFC84B972
:10B24000104B1B680BB90020F8BD214628469847D3
:10B250002046F9E70A4822460BF096FE04460028ED
:10B26000F6D0022C14BF6FF006006FF00500EBE77C
:10B270000228E8D1044892B2EEE700BF801C00200B
:10B280008C6D00204C1800209C6C0020012802D1FD
:10B29000044800F05DBA022801D10348F9E76FF0D5
:10B2A00006007047CC020020E0020020012807B50C
:10B2B0000AD10A480DF1070100F087FA50B16FF08A
:10B2C000060003B05DF804FB0228F8D104480DF134
:10B2D0000701F1E79DF80700F3E700BFCC0200206B
:10B2E000E002002070470000012802D1044800F06D
:10B2F000D3B9022801D10348F9E76FF0060070477F
:10B30000CC020020E0020020F8B5224D224F00249C
:10B310000C23224A63439B5CCBB1022C1BD1204EF1
:10B320003368DA69D103FCD4DA695202FCD51C48CF
:10B330000CF005F833681A4810221A621A6822F0D5
:10B3400010021A600BF0BEF9F06F08F081FF0134B3
:10B35000032CDDD1F8BD012CF9D108232B624FF469
:10B3600080132B6255E8003F43F0020345E80032AA
:10B37000002AF7D157E8003F43F4800347E8003242
:10B38000002AF7D1074AD2F8803043F08063C2F830
:10B390008030DCE700380140083801405C1C0020A8
:10B3A0009C6C00200008005873B50B4C0B4E4FF0FE
:10B3B000FF35012D0BD923784BB133780193A37A54
:10B3C0000093227A637A61680020FFF7FBFD013564
:10B3D000022DEED102B070BD5C1C0020801C00204C
:10B3E00002681D4B9A4270B5044615D10BF06AF9FC
:10B3F0001A4E002516F8011B0220013507F058F9F6
:10B40000802DF7D1154916482A4600F054F9134902
:10B410002A4620460BF0FEFE2268124B9A4216D1B5
:10B4200020460BF04FF9104E002516F8011B0120A5
:10B43000013507F03DF9802DF7D10B490B482A461D
:10B4400000F039F908492A4620460BF0E3FEBDE832
:10B450007040074807F094B9008000401C6C002041
:10B46000E0020020003801407D6E0020CC02002068
:10B47000541C00200268054B9A4205D1044B1B68FE
:10B4800013B1012108461847704700BF003801403A
:10B490004C18002070470000F8B502682E4B9A4205
:10B4A00004461DD10BF00EF92C4B2D4F1B685D6827
:10B4B000C5F18005ADB20026B5423FDC28492948D8
:10B4C0002A4600F0F8F88022254920460BF0A2FE1B
:10B4D000254B1A78012A03D100221A7006F0A2FE29
:10B4E0002268224B9A4224D120460BF0EBF8204BE5
:10B4F000204F1B685D68C5F18005ADB20026B542DE
:10B5000023DC1C491C482A4600F0D5F88022194942
:10B5100020460BF07FFE144B1A78012A03D100223B
:10B520001A7006F07FFE154B1B6813B10121084607
:10B530009847BDE8F840124807F022B917F8011BF8
:10B54000022007F0B5F80136B6E717F8011B012015
:10B5500007F0AEF80136D2E7008000401C6E0020F4
:10B560001C6C0020E0020020481800200038014038
:10B570002C6D00207D6E0020CC0200204C18002095
:10B58000541C002073B5314B00261E7003685A6AA4
:10B590008DF807202E4A9342054619D12D482E4C8E
:10B5A0000BF0E3FE2D4926621523C4E90013204663
:10B5B0008023C4E90266C4E90436C4E9066608F0DB
:10B5C000D5FD08B1FFF7B0FCEC67A562FFF7CAFC38
:10B5D0002A68234B9A421AD12248234C0BF0C5FE0D
:10B5E000224A1123C4E90023204600238022C4E913
:10B5F0000233C4E90423C4E90633236208F0B6FD2C
:10B600000028DFD1EC670120A562FFF7C1FC2C68A0
:10B610000F4B9C420DD19DF80710022007F048F80F
:10B620002B68A34205D1124801220DF1070100F059
:10B6300042F8104807F0A4F80F4B1A781AB9012203
:10B640001A7006F0E7FD02B070BD00BF9C7D0020BF
:10B65000008000409C6C00201C6E0020080002400E
:10B66000003801408C6D00202C6D00204400024009
:10B67000E0020020541C00204818002008B5026891
:10B68000044B9A4205D10BF0ACFABDE80840FFF735
:10B6900069BC08BD00800040C26803699A4282BF4D
:10B6A00040681B180133981A704708B54168FFF7C6
:10B6B000F3FF081A08BD2DE9F743044601A8164612
:10B6C000884607F067F82046FFF7EFFF864228BF5D
:10B6D00006462046FFF7E9FFE3682569A268AB420A
:10B6E0009CBF636801335D1B814623682069AE42BD
:10B6F00002FB003013D872434146FDF7EBFF23698C
:10B7000062683344934296BF236900239B192361E7
:10B7100001A807F041F8304603B0BDE8F08305FB0F
:10B7200002F73A464146FDF7D5FFA2682068751B2F
:10B730006A4308EB0701FDF7CDFF4E452561E7D9C8
:10B7400023696268934234BF01330023E360DFE77B
:10B750002DE9F341044601A81646884607F01AF879
:10B760002046FFF799FFE768E5682369A26821682A
:10B77000864228BF06469D4284BF636801335D1B35
:10B78000AE4202FB071110D872434046FDF7A2FFFC
:10B7900062683744974288BF0027E76001A806F037
:10B7A000FBFF304602B0BDE8F08105FB02F73A46E8
:10B7B0004046FDF78FFFA2682168751B6A4308EBBE
:10B7C0000700FDF787FFE560E8E703460846D9680C
:10B7D0001A69914210B523D09A68DC681968531E23
:10B7E000072B18D8DFE803F00408170C17171710F9
:10B7F0000B5D0370002010BD31F814300380F9E7B1
:10B8000051F824300360F5E701EBC401D1E90023CE
:10B81000C0E90023EEE704FB0211FDF75BFFE9E757
:10B820006FF00E00E7E707B503688DF807105B6857
:10B8300001220DF10701984703B05DF804FB007C7D
:10B8400006F054BD007C06F01FBF07B5007C012246
:10B8500001A906F0E3FD20B19DF8040003B05DF8F6
:10B8600004FB4FF0FF30F9E7007C06F0EFBD007CF1
:10B8700006F0FCBD05F0DCB8F7B5054608461646EF
:10B880000F461C4605F0DAF8287C06F0E1FE3E2E55
:10B8900022D8194B19499A5D194B895D9B5D287C0B
:10B8A0000026CDE90016394606F0FAFC012C02D03C
:10B8B000022C15D0ECB9287C04F0E8FF844218D0A3
:10B8C000287C214604F0EAFF98B994B9287C03B09B
:10B8D000BDE8F04004F084BF00210B460322DEE700
:10B8E0002B7C012B03D9022B03D13446E3E701243F
:10B8F000E1E703B0F0BD00BFE0E202085EE302084A
:10B900001FE302080A490B4A0023022010B54B60CE
:10B910000A6008740849C1E900230B74074901242F
:10B92000C1E900230C740649C1E90023087410BD65
:10B93000841C0020A8E30208981C0020AC1C0020F6
:10B94000C01C002010B504465C3000F043F804F140
:10B95000500000F03FF804F1440000F03BF804F11F
:10B96000380000F037F804F12C0000F033F804F14F
:10B97000200000F02FF804F1140000F02BF804F17F
:10B98000080000F027F8204610BD10B504461BF053
:10B9900033F904F170001BF0CAF804F195001BF0B4
:10B9A000C5F804F1AC001BF0C3F8204610BD000040
:10B9B00010B5054C2046FFF7E8FF2046034A04492E
:10B9C000BDE8104021F0BCBBD41C002000000020CA
:10B9D00045B9000810B50446006808B1FDF772FECD
:10B9E000204610BD10B50446006808B1FDF76AFE98
:10B9F0000023C4E90133236010BD38B504460D4669
:10BA00000068013121F03CFC10B1C4E900050120BF
:10BA100038BD036810B5044623B143688B4201D397
:10BA2000012010BD2046FFF7E8FF0028F9D0A368E9
:10BA3000002BF5D122681370F2E770B50E4611465F
:10BA400004461546FFF7E5FF20B92046FFF7CAFF79
:10BA5000204670BD2068A560314621F055FCF7E70F
:10BA600038B50023C0E90033044683600D4639B180
:10BA70000846FAF785FB294602462046FFF7DDFF18
:10BA8000204638BD38B505460C4649B10846FAF798
:10BA900077FB214602462846FFF7CFFF284638BDF0
:10BAA000FFF7A0FFFAE7002202707047037810B595
:10BAB00004461BB906F046F901232370012010BD8E
:10BAC00070B50C4615461E46FFF7F0FF30B1324602
:10BAD00029462046BDE8704006F068B94FF0FF30B7
:10BAE00070BD70B50C4615461E46FFF7DFFF30B13E
:10BAF000324629462046BDE8704006F06DB94FF049
:10BB0000FF3070BD10B50C46FFF7D0FF20B12046C6
:10BB1000BDE8104006F024B94FF0FF3010BDF0B57D
:10BB200085B00C461746FFF7C1FF30B32FB3684608
:10BB300006F016F968B9019D002D08BF4FF4805535
:10BB40004CB9009BBB4206D82BB106F06DF905B08D
:10BB5000F0BD4FF48055B4FBF5F6013C3C442C4459
:10BB60006E43B4FBF5F46C43A64209D2304606F0AE
:10BB700049F90028EBD12E44F6E74FF0FF30E6E715
:10BB80000020E4E703688A685B68096818471FB506
:10BB9000044601A8FFF764FF01A92046FFF7F2FF62
:10BBA000044601A8FFF716FF204604B010BD0000B0
:10BBB0000149FFF7ECBF00BFAAED020838B5054602
:10BBC000FFF7E5FF04462846FFF7F2FF204438BDA3
:10BBD0000EB430B5C2B045AB054653F8042B019303
:10BBE0004FF4807102A821F009FD2B68044602463B
:10BBF0005B6802A928469847204642B0BDE830401D
:10BC000003B070472DE9F0478AB098469DF8486028
:10BC1000012E4FF0000398BF0A26814615468DF885
:10BC200024300DF1240AF6B2002728464146324658
:10BC30003B46FBF7DFFAD4B2092C43462A4694BFB1
:10BC400030343734BB42E4B208BFB2420AF8014D87
:10BC500005468846E9D25046FAF792FAD9F80030FC
:10BC600002465B685146484698470AB0BDE8F087EF
:10BC70000A2AF7B507460D4616460FD100290EDAF7
:10BC80000A49FFF784FF6D42044600962A46EB17E7
:10BC90003846FFF7B7FF204403B0F0BDD6B2009698
:10BCA0002A46EB17FFF7AEFFF6E700BFC4E3020832
:10BCB00038B50546FFF7DCFF04462846FFF778FF56
:10BCC000204438BD07B5D2B2009200230A46FFF7E0
:10BCD00099FF03B05DF804FB2DE9F84F19460446BF
:10BCE00010460A9E90461F46FAF702FF28B13F49C8
:10BCF0002046BDE8F84FFFF74ABF27F000453C4B10
:10BD00004FF0FF3240462946FAF7F2FE48B9384B69
:10BD10004FF0FF3240462946FAF7CCFE08B93549C4
:10BD2000E6E7354B4FF0604240463946FAF7D6FE1B
:10BD300008B13249DCE7324B4FF0604240463946A9
:10BD4000FAF7AEFE0028F4D100220023404639461F
:10BD5000FAF7A6FE054630B12A492046FFF717FF3D
:10BD600007F10047054640463946FAF7FFFE82468E
:10BD7000FAF7AAFB02460B4640463946FAF766FA3E
:10BD80000A228046894620465146FFF79BFF002E37
:10BD9000054404DD1C492046FFF7F9FE0544DFF8A1
:10BDA0006CB04FF0000A002E1DDD5B465246404647
:10BDB0004946FAF703FC89468046FAF7D7FE0A227D
:10BDC000014607462046FFF77DFF05443846FAF74F
:10BDD0007BFB02460B4640464946FAF737FA013EDE
:10BDE00080468946DFE72846BDE8F88F75E00208FF
:10BDF000FFFFEF7F6DE00208FFFFEF41C6E302089F
:10BE0000FFFFEFC1C4E30208CDDB020800002440BD
:10BE100037B5069900910546FFF75EFF04462846B0
:10BE2000FFF7C6FE204403B030BD10B5044639B953
:10BE300006F06EF902212046BDE8104006F06AB90E
:10BE4000022904D1002106F063F90121F3E7BDE8DE
:10BE50001040012106F05CB909B906F05DB9012175
:10BE6000FBE70FB400B5ADF5037D04F089FEC0B269
:10BE7000012808D185AA8499019202A821F0E2FB49
:10BE800002A806F08FFA0DF5037D5DF804EB04B00F
:10BE9000704704F069BE08B504F072FEC0B208BD78
:10BEA0007FB5092301A88DF8043010F05BF8003845
:10BEB00018BF0120404207B05DF804FB034B53F864
:10BEC0002030986800B10047704700BF046F002021
:10BED00038B50C4D002455F8043BE4B25BB11B6946
:10BEE0004BB12046FFF7EAFF28B100F00DF855F8F6
:10BEF000043C1B6998470134E3B2042B64B2EAD1D5
:10BF000038BD00BF046F002070B5324D8AB03423B5
:10BF100068468DF800300FF02DFA2B881BB90024ED
:10BF200020460AB070BD019E0FF0A6F90246002817
:10BF3000F5D12C8814F0010404D03821304600F0EB
:10BF40004BF804462B889A0706D538222021B018D2
:10BF500000F042F8204484B22B885B0707D55822B2
:10BF60004FF4C271B01800F037F8204484B22B8827
:10BF7000180708D54FF4EE724FF4D071B01800F0E6
:10BF80002BF8204484B22B88D90607D54FF45F7272
:10BF90001421B01800F020F8204484B22B889A06AF
:10BFA00008D54FF464724FF46171B01800F014F8C2
:10BFB000204484B22B885B0607D540F21472182106
:10BFC000B01800F009F8204484B200232B800FF051
:10BFD00049F9A5E7841D00201346024603F10060DD
:10BFE00010B500F578300C4605F0F8FF00280CBFBE
:10BFF0002046002010BD000008B5034806F0C0FB35
:10C00000024B00221A7008BD040300209C7D002012
:10C0100030B58BB00446342368468DF800300FF0FD
:10C02000A9F92CB3019D04F011FF08BB0FF024F90E
:10C03000F0B9E30702D5284605F0A6F8A00703D516
:10C0400005F1380005F0BCF8610703D505F158008B
:10C0500005F0D4F8220703D505F5EE7005F0E8F8F1
:10C06000A30603D505F5647005F0FCF80FF0FAF8A7
:10C070000BB030BD10B50FF0FFF80128044604D016
:10C0800030B906F09BFB204610BD6FF00500FBE7C2
:10C090006FF00600F8E770B50C4606460DF03CFB65
:10C0A0000025043CA9B2A14205F1010503D3BDE876
:10C0B00070400DF04FBB012231440DF031FBF1E730
:10C0C00038B50B78013B044615461848082B28D88C
:10C0D000DFE803F0052727271B2327271F0006F08B
:10C0E00061F9134806F05EF9124806F05BF9124B4D
:10C0F000124853F8241006F055F90B2C15D1294697
:10C100000F48BDE8384006F04DB906F04BF90D4830
:10C11000E8E706F047F90C48E4E706F043F90B4876
:10C12000E0E706F03FF90A48DCE738BDCAE3020859
:10C1300000E4020835E40208B0EB02083EE502081C
:10C1400050E502086AE402089FE40208D4E4020809
:10C1500009E5020838B50B78012B0446154607D0CF
:10C16000032B1CD003BB134806F01CF9124803E054
:10C17000104806F017F9114806F014F9104806F0B7
:10C1800011F9104B104853F8241006F00BF90B2C42
:10C190000FD129460D48BDE8384006F003B90548DF
:10C1A00006F000F90A48E7E7024806F0FBF80948FC
:10C1B000E2E738BD68E50208D3E502089EE502081B
:10C1C00035E40208B0EB02083EE5020850E502083B
:10C1D00008E602083DE6020870B5474E8AB00446FC
:10C1E000042556F8043B1BB11B6A0BB12046984747
:10C1F000013D15F0FF05F4D123780A2B0FD00E2B4B
:10C200000BD13E4806F0CEF83D4B8DF80050684605
:10C210001D708DF804500FF0F9F90AB070BD637805
:10C220000D2B63D1374806F0BDF8354B1A78042A38
:10C230001BD0022628461E7006F0C0FA32492A4654
:10C24000284606F0B7FAB8B920F0E6FF434203F0FB
:10C250001F0300F01F004FF47A7158BF584200FBD3
:10C2600001113246284606F0A7FAA37D032B1FD8FA
:10C27000DFE803F00B24272A40F20931234806F0B7
:10C2800091F8284606F09AFAEFE7214A0023138036
:10C29000237E617E1B0243EA0143E17D0B43536031
:10C2A000E37E217F1B0243EA0143A17E0B4393609F
:10C2B000D4E90101174B83E80300AEE7144A0123D8
:10C2C000E5E7134A0223E2E7237E617E104A1B0260
:10C2D00043EA0143E17D0B43D360E37E217F1B02F0
:10C2E00043EA0143A17E0B431361E1E70E2BDFD14B
:10C2F000094806F057F8DBE7046F002072E60208F1
:10C30000E41E00207DE602087DCB00088AE60208D4
:10C31000C81E0020DC1E00209AE6020804F066BC5D
:10C3200004F088BC04F0FEBC704704F059BD072837
:10C3300001D804F05BBD6FF00200704704F062BDED
:10C3400004F066BD014B1878704700BFEB1F00205A
:10C3500004F01CBC7FB5054604F018FC431EDBB29C
:10C36000012B044603D900F0FD03082B1DD101A8C1
:10C3700004F01EFC002201A91346012011F8016BF4
:10C380001EB100FA02F633439BB201320C2AF5D1FA
:10C3900004F0FD02082A01D0012C02D123F480739D
:10C3A0009BB22B80002004B070BD6FF00200FAE752
:10C3B0002DE9F0418EB080460F4604F0E7FB4B4B71
:10C3C0000093431EDBB2002401AE012BC6E90144F9
:10C3D0000546019404D900F0FD03082B40F083804A
:10C3E000FFF748FE0446002872D1B8F800302BB998
:10C3F000012D51D140F2FF13A8F800300023019322
:10C40000C6E90133B8F8000040FA03F1C907DAB20F
:10C4100010D50DF1380C02F0FE0102F0010261446A
:10C420000CEB420231F834CC32F8382C42EA0C02E0
:10C4300021F8342C01330C2BE6D105F0FD03082B39
:10C4400001D0012D0FD1BDF80C30002203F47F4341
:10C45000ADF80C3011464FF0010CD5B2072D27D99D
:10C4600009B1ADF80C30232304A88DF810300596DF
:10C470000FF0CCF8054660B9242304A88DF81030DD
:10C4800005960FF0C3F804F01FFFE0B90EF0EAFEC6
:10C4900010B36FF006041BE005F0FD03082B04BF8A
:10C4A000FF23A8F80030022DA8D140F6FF73A3E7C0
:10C4B00040FA02F5ED0741BF0CFA02F10B439BB2C3
:10C4C00001210132C9E7284604F004FF0028DDD02D
:10C4D00020460EB0BDE8F081002FF9D0304604F0C0
:10C4E00073FB0446F4E76FF00204F1E7FF0000FF7E
:10C4F00008B504F099FCC0B208BD022808B503D8FD
:10C5000004F098FC002008BD6FF00600FBE704F083
:10C510009DBC00B58BB0012368468DF800300EF04D
:10C5200029FF38B99DF80400003818BF01200BB06E
:10C530005DF804FB0020FAE730B58BB005460C46E9
:10C5400004F084FC28B92146284604F09FFB0BB078
:10C5500030BD0F2C02D86FF00600F8E7FFF7D9FFC7
:10C5600030B9014610222846FBF7DCFD0020EEE73B
:10C570000F2368468DF800300EF0FCFE0028EAD14B
:10C58000019B03F1100253F8041B45F8041B93426E
:10C59000F9D1EBE730B58BB004460D4604F056FCFC
:10C5A00028B92946204604F09DFB0BB030BD032D71
:10C5B00002D86FF00600F8E7FFF7ABFF08B920607C
:10C5C000F3E7072368468DF800300EF0D3FE00280D
:10C5D000EFD1019B1BBA2360E7E730B58BB004466F
:10C5E0000D4604F033FC28B92946204604F0BEFB72
:10C5F0000BB030BD032D02D86FF00600F8E7FFF74F
:10C6000088FF08B92060F3E7062368468DF80030FC
:10C610000EF0B0FE0028EFD1019B2360E8E730B5B3
:10C620008BB005460C4604F011FC28B9214628467B
:10C6300004F0AAFB0BB030BD0F2C02D86FF006003F
:10C64000F8E7FFF766FF30B9014610222846FBF7EE
:10C6500069FD0020EEE70E2368468DF800300EF0ED
:10C6600089FE0028EAD1019B03F1100253F8041B54
:10C6700045F8041B9342F9D1EBE704F0F9BB00B590
:10C680008BB0002368468DF800300EF073FE38B989
:10C690009DF80400032828BFF9200BB05DF804FBC7
:10C6A000F920FAE710B5FFF7EAFF0FF0FDFA0128CD
:10C6B000044606D040B9064B1870FFF7E0FF20464D
:10C6C00010BD6FF00500FBE76FF00600F8E700BF54
:10C6D000E41E002004F0DEBB08B504F017FF0038AC
:10C6E00018BF012008BD38B50C46054610F0D2FB36
:10C6F00024B12846BDE8384004F0FCBE204638BDD1
:10C7000000B58BB02D2368468DF800300EF032FE58
:10C710009DF804000BB05DF804FB04F0F1BB04F0DD
:10C7200001BC04F023BC00B58BB004F08FFB0128E2
:10C730000DD1FFF7EEFE50B1272368468DF800308B
:10C740000EF018FE00B901980BB05DF804FB04F080
:10C750001FFCF9E704F02EBC04F03EBC04F060BC02
:10C7600004F064BC1FB52E238DF8083004F00EFAD7
:10C7700002A912F07EFE05B05DF804FB1FB5302360
:10C780008DF8083004F002FA02A912F072FE05B02A
:10C790005DF804FB014B1868704700BFDC1E0020E9
:10C7A000014BB3F9000070470C210020014B93F9B5
:10C7B000000070472021002010B590B0044605A865
:10C7C0000CF0E0FC059807A912380CF061FD0C9BF9
:10C7D000094903F26C7303930A9B02930B9B013389
:10C7E0000193079B00932046DDE9083220F050FDBD
:10C7F000002010B010BD00BFA7E6020800B58BB046
:10C800001F2368468DF800300EF0B4FD18B901986A
:10C810000BB05DF804FB6FF00600F9E700B58BB0D4
:10C820001F2368468DF800300EF0A4FD20B99DF856
:10C8300008000BB05DF804FBF920FAE704F0DEBB5A
:10C84000022801D804F0E0BB6FF00200704700003E
:10C850002DE9F04F9FB00C4606A981E80C009DF829
:10C86000193003939DF81B3005939DF81C300493F9
:10C870009DF818B09DF81AA0064604F01DFB8046EE
:10C88000FFF747FE0746002800F044810DF010FF37
:10C89000054610B16FF00500DCE0A34B1A7899460D
:10C8A000002A40F0B38004F0F5FA022840F0B98085
:10C8B00000238DF8540014A88DF850300EF0A6FE19
:10C8C0008DF8368004F09AFB60B104F097FB0128E4
:10C8D00002D10020FFF7B4FF052314A88DF85030D3
:10C8E0000FF040FB914B1B78012B05D1092314A8B5
:10C8F0008DF850300FF036FB09A9E0B20EF0DAFCEB
:10C900008046FFF7C8FA60B19DF824309DF82520D5
:10C910008749884851F82810D21A0092224605F01B
:10C9200041FDB8F1000F00F0A58000238DF82830FC
:10C930000C93ADF8343099F8003073B97E4B059AFA
:10C940001E607E4B1C607E4BDA70039A5A70049A0C
:10C9500083F800B01A7183F802A00AA810F0C4F995
:10C96000784B0E9A1A600446FFF795FA002842D0D9
:10C97000342314A88DF850300EF0FCFC14A80EF0EF
:10C98000F9FC002837D1704F159B3A7893F858601E
:10C990006E484FF00C0808FB0232D2F8901305F0F5
:10C9A00001FD012E159B3A4602D0082E40F08280F0
:10C9B0001278D3F8C430664902F0070201FB023155
:10C9C000644805F0EFFC159B6348D3F8C41005F0EC
:10C9D000E9FC159B614893F9491005F0E3FC159BB0
:10C9E0005F4893F9481005F0DDFC159B5D48D96858
:10C9F000013905F0D7FC002C7FD1002D00F08D808F
:10CA0000594B1B78002B6CD1002023E004F0FAF97D
:10CA100001283FF43FAF4A4BDB78002B3FF443AF94
:10CA200038E704F037FA01287FF44AAF4F4B1B7800
:10CA3000012B0BD0022B10D0002B7FF441AF092328
:10CA40008DF83C300FA80FF08DFA39E7FFF72AFE7A
:10CA50000028F4D01FB0BDE8F08F002005F0AEFE36
:10CA60000C238DF83C3004F0DBFA00F007008DF861
:10CA70004000E7E7039B3C4D8DF82CB0ADF8344007
:10CA80000C966BB185F800A0059B6BB1049B7BB93C
:10CA900000238DF82830364B00221A703D464AE7B5
:10CAA00004F09EF92870EFE704F0ACF90028EFD00D
:10CAB0000123EEE7022E397809D13020B1FBF0F2E4
:10CAC00000FB1211CAB2D3F8C4302A4976E708FB3A
:10CAD0000133D3F8941300297FF472AFD3F8901385
:10CAE0006EE704F08FF9012803D0154BDB78002B9B
:10CAF0008AD0012389F8003086E7A4F10E03DBB267
:10CB0000012B7FF6C7AE0B2C0AD10E991A4805F0FF
:10CB100049FCBFE66FF00B009CE76FF0020099E75D
:10CB20006FF0060096E700BF871D0020212100203E
:10CB3000B0EB0208C9E60208881D0020941D002001
:10CB40008C1D00208C1E0020146F00201EE70208A0
:10CB5000C02709001BE702082DE702083FE702088B
:10CB600055E702086AE70208861D0020E41E00203F
:10CB7000EB1F0020400D030076E702081FB50021DF
:10CB8000054B0293009104AB13E90C000348FFF737
:10CB90005FFE05B05DF804FB01010300ACED020887
:10CBA0002DE9F04F43788DB00446002B40F0AF8064
:10CBB000B0F90E007B4F7C4E237C388040B233703E
:10CBC00001F050FC237B002B3BD0607C7749B7F908
:10CBD000002051F8201096F900307548DFF838929F
:10CBE000DFF838A205F0DEFBA378012B0CBF7148FB
:10CBF000714805F0D7FBE178704805F0D3FB4FF0A2
:10CC000000085FFA88FB584603F040FE054640B92D
:10CC1000227BEBB29A4200F2AB805146584605F0B7
:10CC20008BFB08F10108B8F1030FEAD1227BA16860
:10CC30006348FCF74FFD634B227B1A70624BE2782E
:10CC40001A706379012B00F09B802378012B02D1AD
:10CC50000120FFF793FF5D4B1A782AB3DFF8C091EC
:10CC600000221A7099F80030F3B996F90030584D47
:10CC7000DFF8B08100932A78B7F9003098F80010F7
:10CC8000544805F08FFB544B1B686BB1534899F81F
:10CC90000020027098F8002042702A7882703A884A
:10CCA0008280327882719847E278E02A11D04C4B2A
:10CCB0001B6873B14B48027022794270A2684260CF
:10CCC000227B0272E2894281227C027362690261E4
:10CCD0009847454E042556F8043B1BB19B690BB1A0
:10CCE00020469847013D15F0FF05F4D13F4890F8E4
:10CCF000023163B180F802518DF80B508DF8095064
:10CD00000095DDE90223B0F80011FFF7A1FDFFF760
:10CD1000C2F850B3342302A88DF808300EF02AFB75
:10CD200002A80EF027FB002838D1637C73BB304883
:10CD300005F038FBA1692F4805F034FBE1782E4857
:10CD400005F030FBB4F90E102C4805F02BFB94F9DC
:10CD500010102B4805F026FB21792A4805F022FB0C
:10CD6000039B2948996905F01DFB0DB0BDE8F08FC4
:10CD7000A2684946D25C584605F0DEFA013547E71D
:10CD800004F088F800287FF460AF61E7012B01D13F
:10CD90001E48CDE7022BCDD11D48C9E71D4805F03F
:10CDA00001FBE2E70C2100202021002030EC0208EA
:10CDB0008EE702089FE70208AAE7020811ED0208C1
:10CDC000EC1F0020EC200020ED200020F6200020A9
:10CDD000C01E0020B8E7020810210020EE2000202D
:10CDE00014210020F8200020046F0020E61E0020FF
:10CDF000D7E7020834E8020846E8020850E80208CB
:10CE00005AE8020863E8020873E80208F4E7020837
:10CE100011E8020881E80208B3E70208AAED020857
:10CE2000F72000208A1E0020F7B54178044621BB78
:10CE30000379294A294D13702378012B41D1277991
:10CE4000EFB1274805F0AEFA264B1B680BB16078AE
:10CE5000984700232B70002001F098FC224E0425F7
:10CE600056F8043B1BB15B690BB120469847013D66
:10CE700015F0FF05F4D103B0F0BD0023D9E71B483E
:10CE800005F090FA1A4B1B7893B12E78B3420FD36A
:10CE9000184B194919482F7000971A6809681B79AF
:10CEA0000068FFF7D5FC0028D3D101362E70D2E7F9
:10CEB00000232B700B4B1B68002BCCD0607898475D
:10CEC000C9E700232B70074B1B680BB10846984736
:10CED0000B4805F067FABEE7EB1F0020871D002016
:10CEE000A5E8020818210020046F0020BEE802080F
:10CEF000861D00208C1D0020941D0020881D002010
:10CF0000DFE80208014B1878704700BF212100209C
:10CF100010B50446FFF7FDFA28B1012C06D8054BE1
:10CF200000201C7010BD6FF00B00FBE76FF00200DB
:10CF3000F8E700BF2121002004F084B804F094B881
:10CF400004F0A4B804F0B4B870B5094E3478944233
:10CF500028BF14460546224608460649FCF7BAFB98
:10CF6000054B1A782A7000221A703270204670BD64
:10CF7000EC200020EC1F0020ED20002070B5044DB7
:10CF8000064604460FCD0FC42B682360304670BDA3
:10CF9000C81E0020F0B591B0002603ACC4E90166BC
:10CFA0000546039603F0F2FD431EDBB2012B0AD9BE
:10CFB000082808D005286BD00A2804D06FF0060492
:10CFC000204611B0F0BD15BB2046ADF8185003F057
:10CFD000EFFD0028F2D1BDF818302A46012114F8DF
:10CFE000010B20B101FA05F213439BB20122013576
:10CFF0000C2DF4D10AB1ADF81830002106A8FFF7C6
:10D00000D7F904460028D9D104F064F9D8E71A23E7
:10D0100001A98DF8043012F02CFA1E230090C6B23C
:10D0200006A88DF818300EF0A5F9079B0022A3F191
:10D030000C010C20D3B29E4204D8B3425AD16FF0F7
:10D040000204BDE7013200FB02F7CF59AF42F1D134
:10D050001A0910A901EB420203F00F03012101FAA2
:10D0600003F322F8343C06A823238DF818300794E4
:10D070000EF0CCFA0028A1D1242306A807948DF83D
:10D0800018300EF0C3FA0446002897D12846BBE7B3
:10D09000D5B90723ADF80C3006A823238DF8183036
:10D0A00007940EF0B3FA002888D1242306A88DF83F
:10D0B000183007940EF0AAFA00287FF47FAF2846B4
:10D0C00004F008F904467BE71E2306A88DF8183003
:10D0D0000EF050F9079933460C2000FB03F28A58F2
:10D0E000AA4203D1012202FA03F3D3E70133042B4E
:10D0F000F3D1A4E7002463E708B503F047FD431E1E
:10D10000DBB2012B03D900F0FD00082803D1BDE8F4
:10D11000084004F0D9B86FF0060008BD08B5FFF765
:10D12000EBFF024658B1064B064900209A4208BF61
:10D13000042003F5C31303F520638B42F6D108BD29
:10D14000C0AFD235C0FF953608B5FFF7D5FF024610
:10D1500058B1064B064900209A4208BF062003F545
:10D16000C31303F520638B42F6D108BD6086973662
:10D1700060D65A37FFF7C0BFFFF7BEBF014B187824
:10D18000704700BFE41E002038B50D46044610B1BC
:10D190004FF0FF3038BD1AF0DFF80028F8D0084B08
:10D1A00008491860084B4362084B8362084BC3620E
:10D1B000084B0363F2224368284698472046E9E774
:10D1C000046F0020981D002055C10008C1C0000850
:10D1D000C7D80008A1BE000800B58BB030238DF879
:10D1E00000306846192301930EF010FA0BB05DF879
:10D1F00004FB03F06FBF03F073BF03F07DBF03F0C8
:10D2000081BF03F08BBF03F08FBF03F09FBF10B54A
:10D21000044620B10120BDE8104003F0A3BF04F094
:10D22000DBF92046F7E710B5044612F018F940B9CB
:10D2300014B1143C022C04D8BDE81040002012F0B8
:10D240000EB910BD30B58BB00D46044603F09EFC00
:10D25000FFF7E9FFA0B1032368468DF80030019481
:10D260000EF0D4F938B101280CBF6FF005006FF053
:10D2700006000BB030BD2946204603F0C5FCF8E798
:10D280006FF01000F5E730B58BB00D46044603F0A3
:10D290007DFCFFF7C8FFE8B1082368468DF8003031
:10D2A00001940EF0B3F938B101280CBF6FF00500FE
:10D2B0006FF006000BB030BD092368468DF80030D2
:10D2C00001940EF0A3F90028EED12946204603F080
:10D2D000C3FCEFE76FF01000ECE730B58BB00D4604
:10D2E000044603F053FCFFF79EFFA0B10F236846EE
:10D2F0008DF8003001940EF089F938B101280CBF87
:10D300006FF005006FF006000BB030BD29462046D7
:10D3100003F0CEFCF8E76FF01000F5E730B58BB006
:10D320000D46044603F032FCFFF77DFFB0B1072342
:10D330008DF80030236868461BBA01930EF066F939
:10D3400038B101280CBF6FF005006FF006000BB07C
:10D3500030BD2946204603F0D3FCF8E76FF01000FB
:10D36000F5E730B58BB00D46044603F00FFCFFF730
:10D370005AFFC8B103F058FDC0B201280FD10223F3
:10D3800068468DF8003001940EF040F938B101285C
:10D390000CBF6FF005006FF006000BB030BD2946E2
:10D3A000204603F0CDFCF8E76FF01000F5E730B54C
:10D3B0008BB00D46044603F0E9FBFFF734FF30B3B2
:10D3C0000C2368468DF8003001940EF01FF938B137
:10D3D00001280CBF6FF005006FF006000BB030BDE8
:10D3E0000D2368468DF8003001940EF00FF90028E7
:10D3F000EED10E2368468DF8003001940EF006F948
:10D400000028E5D12946204603F0D0FCE6E76FF07E
:10D410001000E3E72DE9F04395B004460D46904631
:10D420001F4603F013FD611C064629D16A1C0AD071
:10D43000003D18BF012503F017FE854203D02846A2
:10D4400003F018FE50BBB8F1FF3F07D003F01EFEFB
:10D45000804503D0404603F01FFEF8B97B1C07D07F
:10D4600003F026FE874203D0384603F027FEA8B912
:10D47000BCB9204605F0A2F9734B1C6000200DE0FA
:10D48000B4F1000918BF4FF0010903F0DBFD81453D
:10D49000CCD0484603F0DCFD0028C7D015B0BDE86D
:10D4A000F08303F073FBFFF7BEFE002800F0C88096
:10D4B000012E40F092808DF8006003F0FDFC022305
:10D4C0008DF8050068468DF804300EF04BFD5F4B7B
:10D4D000049A1A600446002850D103F0DBFC0128AE
:10D4E00008BF5B4B0AA808BF1C7034238DF8283096
:10D4F0000DF040FF0B9B9888FFF787FEFEF7CBFCF3
:10D500000028CBD034230AA88DF828300DF032FF44
:10D510000AA80DF02FFF0028B0D14E4D0B9B2A78A2
:10D5200093F858404C480C2606FB0232D2F8901370
:10D5300004F038FF012C0B9B2A4601D0082C69D13E
:10D540001278D3F8C430454902F0070201FB0231DA
:10D55000434804F027FF0B9B4248D3F8C41004F063
:10D5600021FF0B9B404893F9491004F01BFF0B9BD4
:10D570003E4893F9481004F015FF7FE7012812D0C8
:10D580000B282BD1304D002005F018F92C68013400
:10D590002C6003F08DFD844208D900232B60049990
:10D5A000334804F0FFFE6FF0050077E700223149B1
:10D5B000104605F0FFF8044648B903F067FD4FF444
:10D5C0007A7141432246204605F0F6F8E7E740F637
:10D5D0000401294804F0E6FEE1E716B16FF0060009
:10D5E0005CE7012368468DF800308DF804300EF0BA
:10D5F0000DF80028F2D103F04DFC022807D18DF878
:10D60000040068468DF800600EF000F876E703F03D
:10D6100041FC73E7022C297809D13020B1FBF0F2EC
:10D6200000FB1211CAB2D3F8C43014498EE706FBCE
:10D630000133D3F8941300298AD1D3F8901387E7E4
:10D640006FF010002AE700BFC41E00208C1E0020CF
:10D65000E41E0020146F00201EE70208C027090006
:10D660001BE702082DE702083FE7020855E702081A
:10D6700076E7020881D60008EEE80208400D0300B4
:10D680004FF0FF331A4619460120FFF7C3BE30B5ED
:10D690008BB00C46054603F079FAFFF7C4FD88B15C
:10D6A000052368468DF800308DF804500DF0AEFF6C
:10D6B00003280AD001280BD06CB1284603F0DEFB0A
:10D6C0000BB030BD6FF01000FAE76FF00200F7E723
:10D6D0006FF00500F4E72046F2E7000030B58BB0AC
:10D6E0000C46054603F052FAFFF79DFD00283AD09C
:10D6F000FEF70FFFB8B1002368468DF800300DF03B
:10D7000039FE10B16FF0060011E09DF80430012BD6
:10D710001CD0022B22D0002BF4D1012D09D0022DD8
:10D720000BD0002DEED10CB3284603F0B9FB0BB0A3
:10D7300030BD0F4B00221A70F5E702238DF804303C
:10D7400068460DF063FF0028EDD0DBE7012DF7D030
:10D75000022DF2D0002DD5D10023EFE7012DE8D026
:10D76000022DF7D1DFE76FF01000E0E72046DEE79B
:10D77000E41E002030B58FB00D46044603F006FAD3
:10D78000FFF751FD002800F09B8001238DF8103039
:10D79000002C4DD18DF8143004A80DF037FF00286F
:10D7A0004AD1002C53D11021684603F06FFA0F23A1
:10D7B00004A88DF81030CDF814D00DF027FF002804
:10D7C0003AD10421684603F08DFA07238DF8103012
:10D7D000009B04A81BBA05930DF018FF60BB102135
:10D7E000684603F0D1FA0C2304A88DF81030CDF868
:10D7F00014D00DF00BFFF8B90D2304A88DF81030EC
:10D80000CDF814D00DF002FFB0B90E2304A88DF8A6
:10D810001030CDF814D00DF0F9FE68B903F03AFBE2
:10D820002146FFF75BFF48B9002D45D1284605E0AA
:10D8300004A80DF09FFD18B16FF006000FB030BDC9
:10D840009DF81430012B08BF8DF81400A4E70821BF
:10D85000684603F067FA022304A88DF81030CDF86B
:10D8600014D00DF0D3FE0028E6D10821684603F05D
:10D87000BDF9032304A88DF81030CDF814D00DF0B5
:10D88000C5FE0028D8D11021684603F0D3F908233B
:10D8900004A88DF81030CDF814D00DF0B7FE002894
:10D8A000CAD1092304A88DF81030CDF814D00DF09A
:10D8B000ADFE0028B8D0BFE7204603F0CDFABDE7A3
:10D8C0006FF01000BAE710B5012100B10846FFF76C
:10D8D00051FF4FF0FF33BDE810401A4619460120B2
:10D8E000FFF798BD30B58BB00C46054603F04EF9F6
:10D8F000FFF799FCC0B12D2368468DF800308DF8F4
:10D9000004500DF083FE40B9284602F0C5FC74B106
:10D91000284603F0D7FA0BB030BD03280CBF6FF0D8
:10D9200002006FF00600F6E76FF01000F3E7204604
:10D93000F1E70000F0B58D4E8BB00446042556F893
:10D94000043B1BB1DB690BB120469847013D15F044
:10D95000FF05F4D12378013B0B2B4AD8DFE813F005
:10D960000C00490049004900D20049004900490023
:10D970008C004900F300BA0065787D4E7D4F002D84
:10D9800039D17D4804F00EFD284604F017FF3560BC
:10D9900003F080FA02280AD18DF8040068468DF859
:10D9A00000500DF033FE10B1744804F0FBFC3B68EE
:10D9B0000BB10020984703F07FFA0021FFF792FF98
:10D9C00003F068FAFEF767FA98B1342368468DF8D9
:10D9D00000300DF0CFFC68460DF0CCFC002847D19C
:10D9E000674804F0DFFC019B6648D3F8E41004F0BC
:10D9F000D9FC0BB0F0BD022D1CD0EB1E012B1BD8A7
:10DA0000614804F0CFFC002004F0D8FE35680135F1
:10DA1000356003F04DFB854213D9002333603B682A
:10DA200023B15A486378436004F0AAFE584BDB6A7E
:10DA30009847C5E75748E4E72946574804F0B2FC41
:10DA4000E1E700225549104604F0B4FE054648B906
:10DA500003F01CFB4FF47A7141432A46284604F038
:10DA6000ABFEDCE740F249214B4804F09BFCD6E7D3
:10DA70004B4804F097FCBCE74A4B66781D781C467F
:10DA8000DEB9012D09D1484804F08CFC474B1B68D6
:10DA90000BB1304698470023237003F0FBF90128AF
:10DAA000A7D1434B1A78042AA3D018700B236846D9
:10DAB0008DF800300EF056FA9BE7012D99D13D48C4
:10DAC00004F070FC394B1B680BB1284698470023C3
:10DAD00023708EE76378002B8BD1354A8DF80030A8
:10DAE00004210123684611708DF804300DF08EFD7D
:10DAF00000287FF47EAF304804F054FC0220FFF78A
:10DB00003DF876E72D4B01221A702D4B227A1A70C0
:10DB10002C4B627A1A7063782B4C2370002B3FF4E5
:10DB200068AF2A4804F03EFC294B1A68002A3FF4EB
:10DB300060AF28482378037000234370837083808C
:10DB40008371904755E76378002B3FF452AF22482A
:10DB500004F028FC214804F025FC154B1A78042A0F
:10DB60001CBF03221A700923A1E700BF046F002025
:10DB7000C41E0020006F002004E9020812E9020818
:10DB800063E9020879E9020827E902080C0300208A
:10DB900014F2020845E90208EEE8020881D60008FE
:10DBA00081E802082121002088E902081C210020C8
:10DBB000E41E00209AE90208B0E90208F6200020DD
:10DBC0008A1E0020C01E0020F7200020BBE90208AA
:10DBD00010210020EE2000209AE60208D6E9020873
:10DBE00030B58BB00C46054602F0D0FFFFF71BFBAB
:10DBF00068B1292368468DF8003001950DF006FDC7
:10DC000040B954B1284603F081F90BB030BD6FF034
:10DC10001000FAE76FF00600F7E72046F5E730B5A9
:10DC20008BB00C46054602F0B1FFFFF7FCFA68B175
:10DC30002A2368468DF8003001950DF0E7FC40B9C5
:10DC400054B1284603F074F90BB030BD6FF01000EA
:10DC5000FAE76FF00600F7E72046F5E730B58BB03E
:10DC60000C46054602F092FFFFF7DDFA70B11D2366
:10DC700068468DF800308DF804500DF0C7FC40B9AF
:10DC800054B1284603F078F90BB030BD6FF01000A6
:10DC9000FAE76FF00600F7E72046F5E770B58AB0BF
:10DCA0000C46054602F072FFFFF7BDFA00B32723CA
:10DCB00068468DF8003001950DF0A8FC18B16FF0A2
:10DCC00006000AB070BD282305F57A7668468DF8FF
:10DCD000003001960DF09AFC0028F0D15CB130467E
:10DCE00003F06EF90028ECD1284603F057F9E8E775
:10DCF0006FF01000E5E72046E3E770B58AB00C4608
:10DD0000054602F043FFFFF78EFA00B3282368466A
:10DD10008DF8003001950DF079FC18B16FF0060018
:10DD20000AB070BD2723A5F57A7668468DF80030D5
:10DD300001960DF06BFC0028F0D15CB1304603F089
:10DD40002DF90028ECD1284603F03AF9E8E76FF006
:10DD50001000E5E72046E3E770B58AB00C460546BB
:10DD600002F014FFFFF75FFAC8B12E236EB26846C7
:10DD70008DF800308DF804600DF048FC40B9304655
:10DD800002F0FEFA74B1284603F02CF90AB070BD17
:10DD900003280CBF6FF002006FF00600F6E76FF08B
:10DDA0001000F3E72046F1E730B58BB00C4605468E
:10DDB00002F0ECFEFFF737FA88B11F2368468DF8B2
:10DDC00000300DF0D7FA68B9684601950DF01EFCD9
:10DDD00058B96CB1284603F0B7F80BB030BD6FF0FE
:10DDE0001000FAE76FF00600F7E76FF00200F4E7C3
:10DDF0002046F2E770B58AB00C46054602F0C6FE32
:10DE0000FFF711FA08B31F2668468DF800600DF081
:10DE1000B1FAB8B9212368468DF800308DF8085062
:10DE20000DF0F4FB68468DF800608DF808500DF099
:10DE3000EDFB28B964B1284603F056F80AB070BD6E
:10DE4000032807D06FF00600F8E76FF01000F5E741
:10DE50002046F3E76FF00200F0E700002DE9F047FD
:10DE600096B00546F9F7CCFD02F0DEFFC0B20128FE
:10DE70002AD001F093FC002403F00CF8022805D00E
:10DE800002F0E4FF10B1934BDB6A984702F0CCFF3D
:10DE9000C0B2012814D19CB903F0E6F880B103F0B8
:10DEA000D1F8054603F0E0F8064603F0EFF8074620
:10DEB00003F0FEF83A46034631462846FFF7AAFA31
:10DEC000204616B0BDE8F087CDB911F0A3FD824819
:10DED000824B0360824B4360824B83498360834B58
:10DEE000C3600023C1E90033814B8B602A46814B1C
:10DEF000CB600CF0DBFF88B16FF00604BCE7142D9B
:10DF000004D1022011F086FD0025E0E7152D01D196
:10DF10000320F7E7162DDAD10420F3E7764B012230
:10DF20001A7035238DF8083002A8744B03930DF056
:10DF30006DFB0028E0D16B1E012B03D905F0FD031A
:10DF4000082B29D100230CA8ADF8063002F030FED2
:10DF50000446002890D1BDF806300CAA01460124E1
:10DF600012F8016B26B104FA00F10B439BB20121B8
:10DF700001300C28F4D109B1ADF80630FFF7BCF838
:10DF80000146002800F09480FFF7B6F8FFF702F88A
:10DF9000044600287FF470AF052D00F08E8002F05B
:10DFA00055FF0021FFF7E6FB044600287FF464AF2D
:10DFB00000F0DCFD044600287FF45EAF02F06AFF4B
:10DFC0002146FFF78BFB044600287FF455AF02F093
:10DFD0004FFF2146FFF75BFB044600287FF44CAF60
:10DFE00002F06AFF2146FFF77DFC044600287FF41B
:10DFF00043AF02F073FF2146FFF7FCFE0446002802
:10E000007FF43AAF02F0ACFF2146FFF7CDFE02F0FD
:10E0100077FF2146FFF7E4FD044600287FF42CAF8C
:10E0200002F0A4FF2146FFF719FE044600287FF402
:10E0300023AF02F0ADFF2146FFF730FE0446002873
:10E040007FF41AAF02F0C8FF2146FFF785FE0446B1
:10E0500000287FF411AF03F059FA0EF01BFF3425AE
:10E0600002A88DF808500DF085F9039E03F068F8BA
:10E07000B08003F083F8003818BF012086F8AF01A4
:10E0800002F0E4FE002841D01D4812F04BFF1D486D
:10E0900017F0F4F8FFF7A0F80DF0E4F800287FF48B
:10E0A0002BAF1949FFF770F800283FF4E5AE23E7DE
:10E0B0000DF10600FEF77CF96AE7FFF71DF800286E
:10E0C0003FF46DAF0020FEF765FF044600283FF4E3
:10E0D00066AFD1E614F20208B01E002029CE000877
:10E0E000A1CB000835D90008A01E0020D9C1000826
:10E0F00011C00008F9BF0008EA1F0020000300015A
:10E10000F4020020FC020020901E00200CA88DF8D4
:10E1100030500DF02FF90D9F03F04EF8064603F036
:10E1200069F8054603F080F8824603F097F88146C7
:10E1300003F0AEF8382180463046FDF7ACFF736B34
:10E14000984209D133463A4606F1380153F8040B98
:10E1500042F8040B8B42F9D120212846FDF79BFFA2
:10E16000EB6998420AD12B4607F1380205F12001EC
:10E1700053F8040B42F8040B8B42F9D14FF4C271EF
:10E180005046FDF788FFDAF88031984206D14FF407
:10E19000C272514607F15800FBF79CFA4FF4D07158
:10E1A0004846FDF778FFD9F89C31984206D14FF4E4
:10E1B000D072494607F5EE70FBF78CFA002308F1A0
:10E1C000040207F5657758F8031009B1D158F950E2
:10E1D0000C33B3F5587FF6D102F04AFE00283FF425
:10E1E00053AF02F069FE0021FFF77CFB00283FF4EB
:10E1F0004BAF41E638B502F017FEC0B201280DD092
:10E2000002F028FB02F038FB03F0E8FBD8B11E490E
:10E210001E4804F0C7F86FF0060412E002F0B6FCE6
:10E22000A0F11403DBB2022B054698BF0025FDF7D1
:10E2300021FF04460028E3D0284611F010F90028F9
:10E24000DED0204638BD00F0C3FC0028E3D102F048
:10E25000EBFDC0B2012801D00024F2E702F096FCE9
:10E26000A0F11403DBB2022B054698BF002502F093
:10E270008DFCFFF7F3FD04460028EDD0284611F091
:10E28000EEF80028E8D0DCE710EC0208EDE902081F
:10E29000F0B58BB00646F9F7C7FB10F0FF0F00F0A2
:10E2A0008580022E04D16FF0100420460BB0F0BD23
:10E2B000042EF8D002F06AFC864200F0A4803046BA
:10E2C000FEF7B1FF0028EED0FDF7D4FE044618B1EA
:10E2D0004E4B1B78002BE8D100F07AFC0028E4D1EB
:10E2E00002F0F8FF07460028DFD102F0B3FA02F08F
:10E2F000C3FA002E60D1012011F08CFB3546444951
:10E3000044482A460CF0D2FD002879D12C236846D7
:10E310008DF800300DF02EF8002871D19DF8040022
:10E3200002F0D0FD04460028BFD1202768468DF8B2
:10E3300000700DF01FF8002862D19DF8080002F06F
:10E34000D3FD04460028B0D168468DF800700DF06A
:10E3500011F8002854D1019802F0F6FD0446002877
:10E36000A3D12F2368468DF800300DF003F8002864
:10E3700046D19DF8040002F035FE0446002894D1F1
:10E380006B1EDBB2012B29D905F0FD03082B25D02C
:10E39000002E18BF3546284602F0FEFB0446002832
:10E3A00083D12846FFF75AFD04467EE7022E81D02E
:10E3B000042E3FF47FAF76E7142E04D1022011F033
:10E3C00029FB3D469BE7152E01D10320F7E7162ECA
:10E3D00001D10420F3E735463E4690E72423684602
:10E3E0008DF800300CF0C6FF50B9019802F0ECFB3C
:10E3F000044600287FF459AF02F06CFF0028C7D014
:10E400006FF0060451E700244FE700BFEA1F002029
:10E41000A01E0020B01E002013B5064C636898476C
:10E4200028B9E36A019302B0BDE81040184702B072
:10E4300010BD00BF14F20208014B5B68184700BF13
:10E4400014F2020808B5034B5B689847003818BF00
:10E45000012008BD14F20208014B1870704700BF7C
:10E46000146F0020024B034A1B78D054704700BF42
:10E47000146F0020222100202DE9F0438BB02323CC
:10E48000054668468DF800300CF074FF02460028FF
:10E4900051D12A4B2A4CD3F800C093F906E0064626
:10E4A0002046B7B2002101EB0209CC451FFA81F8E2
:10E4B0002ED114F90190F1452AD1B8F10F0F1AD1DC
:10E4C000052F06D14FF0FF321A6000200BB0BDE8D7
:10E4D000F0830136019A32F81620310102F0010270
:10E4E0009A80425C19609A71144B03CB2860696072
:10E4F0006FF00D00EAE7013101240A4404FA01F14A
:10E50000019C1A6034F81640825C21409980EAE749
:10E5100001311029C7D10136062E02F1100204F193
:10E520001004BED100221A60019A128802F0010282
:10E530009A800278D7E76FF00600C7E7140300203F
:10E540002221002010B58AB088B3FDF7E0FF012832
:10E55000044609D1FDF7DDFF30B94FF0FF331A460D
:10E5600019462046FEF756FF00200EF093FC0122CC
:10E570001149042004F01EF9024698B941F288318D
:10E58000042004F019F94623012468468DF8003070
:10E590008DF804400DF03AF82046FEF738FE0020D2
:10E5A0000AB010BD4721054803F0FCFEEBE704204C
:10E5B00004F004F9F3E700BF5DE60008D2E80208C2
:10E5C0002DE9FF47214D224E224FDFF88C808DF838
:10E5D000080001232B704323337000238DF809308A
:10E5E0008DF80B304FF0E00957F8042BDCB2B2B1D4
:10E5F0001369A3B12046FDF761FC80B157F8043CD4
:10E60000DB68984758B198F80AA0D8F80C10524621
:10E610003046FBF75FF885F800A08DF80890631C82
:10E62000DAB2042A5BB2DFD10023009304AB13E912
:10E630000C0029780648FEF70BF920B9064B5870F4
:10E6400004B0BDE8F0874FF0FF30F9E7186F002005
:10E6500082210020046F0020985F002010B5FDF794
:10E6600056FF0128044609D1FDF753FF30B94FF09A
:10E67000FF331A4619462046FEF7CCFEBDE810408F
:10E680000220FFF79DBF00002DE9FF414FF480728B
:10E6900000213A483A4E3B4CF9F744FD00233370D1
:10E6A0000CF01EF880B2C82884BF143880B2E3682A
:10E6B00006389842606146D30021A17023713378F7
:10E6C0002E4F2278FA545A1CD2B26078B8549A1C51
:10E6D000D2B2A078B854DA1CD2B2E078B854581D3F
:10E6E0000433DBB294F8048007F80380A368C5B252
:10E6F0004246194457FA80F0FAF7ECFF05EB08029E
:10E70000D2B200233846D9B28A4230D81E4B1B48B9
:10E710001B788DF8083001238DF80B30A369003B7E
:10E7200018BF01238DF80C3000238DF809300093B9
:10E73000013204ABD1B213E90C003170FEF788F856
:10E7400004B0BDE8F08121695B1AB3FBF0F5EAB2D1
:10E7500000FB15354DB9A270A278984202F1FF3244
:10E7600028BF1846A2702071A9E70132F3E717F815
:10E77000011B855C294481540133C4E774220020C5
:10E7800074230020346F0020752300200D4A137875
:10E79000BBB10D4B80B9997809B9117070471A78DF
:10E7A000197960F341021A70DA780132DA701A6965
:10E7B0000A441A61FFF768BF1A7842F002021A7021
:10E7C000F8E770477C230020346F00202DE9F843E0
:10E7D0001C46431EDBB2DE2B0E46054611462AD8E8
:10E7E000B4F5806F27D8164F164BDFF864904FF0C2
:10E7F00001082246384683F80080FAF76BFFC9F813
:10E800000040114C237823F0030343EA08032370EC
:10E81000FF2003F0C3FF00232361D9F80030E36039
:10E820000A4B607084F803801D70A760A661BDE884
:10E83000F843FFF729BF6FF00200BDE8F88300BF7F
:10E84000506F00207C230020346F002075230020AF
:10E850007823002084B0F0B58BB010AC84E80F00B2
:10E860006C4A119800238DF80330114616464C6807
:10E87000A04200F0CC800133042B01F13401F6D129
:10E8800000255168ECB2002940F0B68010AB4FF47F
:10E89000807713F8082B8DF87050CDE9020316AB82
:10E8A000CDE90431022A4FF6FF7306938DF81C2040
:10E8B0001A9BADF804708DF8064060D1002B32D061
:10E8C00008939DF86C308DF8243001A80DF000FA03
:10E8D000002840F09C809DF806000DF1030207A976
:10E8E0000DF088FA9DF8033023F00303184310F06D
:10E8F000FF0F40F08C80342404FB056410AD0FCD75
:10E900000FC40FCD0FC40FCD0FC42B684148236037
:10E9100002F0C6FC002818BF6FF006000BB0BDE87F
:10E92000F04004B07047FDF713FD0A286FD8DFE808
:10E9300000F0060A161A1C1E20220A240A00364B72
:10E940000893022302E0354B089308238DF8243006
:10E95000089B1A939DF824308DF86C30B5E7304B46
:10E9600008930023F2E72F4BFAE72F4BF8E72F4BE2
:10E97000F6E72F4BF4E72F4BE2E72F4BF0E74BB1D5
:10E9800008939DF86C308DF82430BDF86E30ADF8EA
:10E9900026309AE7FDF7DCFC0A2838D8DFE800F0DB
:10E9A000060A161A1C1E20220A262800234B08934A
:10E9B000032302E0194B089308238DF82430089BA9
:10E9C0001A939DF824308DF86C30DEE71C4B0893C9
:10E9D0000223F2E71B4BEAE7134BE8E7134BE6E7AA
:10E9E000194BE4E7134B08930423E6E7174BDEE7E4
:10E9F0000A4B08930A23E0E70135042D02F13402A3
:10EA00007FF43FAF124834220021F9F78BFB6FF0FF
:10EA10000F0083E75073002000EA0637A070083724
:10EA200020441E1E8068D92E2876E81908E6D333C4
:10EA3000E013F336F080A633E069CD3340F70937B1
:10EA400020937F1D4026CA2E6063053710D62D0502
:10EA500020740020F8B51B4E00233246354651681D
:10EA6000814229D1342707FB035595F830000DF07A
:10EA700091F9044618B16FF006052846F8BD014625
:10EA80003A462846F9F74EFB0E4802F009FC0546C7
:10EA90000028F0D1034672680AB10134E4B20133B0
:10EAA000042B06F13406F6D1002CE6D1FDF712FE58
:10EAB0002146FEF713FEE0E70133042B02F1340296
:10EAC000CDD1D8E750730020F0B58FB0264C064664
:10EAD0003422002101A8F9F725FB012384F8313005
:10EAE000022384F86530032384F89930042384F8E2
:10EAF000CD3034220DEB030130461EF041FB90B9BE
:10EB0000194B324603F130051C4603CCAC42106071
:10EB10005160234602F10802F6D1186810606FF0C8
:10EB20000D000FB0F0BD274600253422394630468F
:10EB30001EF026FB90B9032DF3D0342305FB0333DD
:10EB40002344324603F130051C4603CCAC4210602E
:10EB50005160234602F10802F6D1DEE70135042DAB
:10EB600007F13407E1D1CBE7507300202DE9F043E2
:10EB7000BFB002F091FBD02201460AA8FAF7AAFD25
:10EB80000AAE4FF000084FF03409736853B908F12A
:10EB90000108B8F1040F06F13406F6D100203FB0A9
:10EBA000BDE8F0833EAB09FB0834A4F1D007C03CBC
:10EBB0000FCC6D460FC50FCC0FC523682B6097E8AF
:10EBC0000F00FFF747FE0028E1D06FF00600E6E7F0
:10EBD00038B5094C0025606830B90135042D04F1C1
:10EBE0003404F8D1002038BDFFF734FF0028F4D0FA
:10EBF0006FF00600F7E700BF50730020064B1B685C
:10EC000010B5044603B19847044B0CB100225A706A
:10EC100000225A7110BD00BF20740020A3240020E0
:10EC200070B5064E04464518AC4200D170BD14F8CC
:10EC3000011B304603F0B6FBF6E700BF48EC0208C4
:10EC400008B5074B00225A70FDF725F918B10549A0
:10EC5000054803F0A7FBBDE8084003F0E3BA00BF96
:10EC6000A324002055ED0208D6F7020838B5114C50
:10EC700000236370A37002F0D7F810F0FF0F0CBFF1
:10EC80000D480E4803F08EFB0D4B02225A720D4ABE
:10EC9000156815B193E80700A847E37843B92379CD
:10ECA00033B9094B1B6B9847BDE8384003F0BABA3B
:10ECB00038BD00BFA32400204DEC020868EC020818
:10ECC000AC2400202474002014F20208134B99781D
:10ECD000002210B55A701A4619B9D97809B91B79AA
:10ECE00013B10123537010BD02F09EF810F0FF0F16
:10ECF0000CBF0B480B4803F055FB0B4B01225A721B
:10ED00000A4A146814B193E80700A047084B1B6B2C
:10ED10009847BDE8104003F085BA00BFA324002047
:10ED200083EC0208A0EC0208AC240020247400202C
:10ED300014F2020813B5114C00236370104B1B68CA
:10ED400003B1984702F070F810F0FF0F0CBF0D48A8
:10ED50000D4803F027FB03F065FA23795BB101232B
:10ED600063700A4C236B9847636B0193002002B0D9
:10ED7000BDE81040184702B010BD00BFA32400201A
:10ED800028740020BDEC0208CFEC020814F202083F
:10ED900008B502F049F8C0B208BD0000044B58782D
:10EDA00020B9987810B9D87800B91879704700BFA1
:10EDB000A324002002F09ABA044B054A034493426C
:10EDC0008CBF6FF002000020704700BF802E0FF74D
:10EDD000809E473002F09CBA053807288CBF6FF040
:10EDE00002000020704708B502F0A4FA7D2806D082
:10EDF000FA2806D0B0F5FA7F08BF022008BD00202F
:10EE0000FCE70120FAE7000010B5044602F00CF818
:10EE100010F0FF0F0DD17D2C01D1002010BDFA2C78
:10EE2000FBD0B4F5FA7FF8D0092CF6D96FF00200C8
:10EE3000F4E701F0F9FFC0B20228EED1024BA4F5CD
:10EE400096549C42F1E700BF780D070002F08EBA9D
:10EE500003288CBF6FF002000020704702F098BAC0
:10EE6000042894BF6FF002000020704702F0A2BA9D
:10EE7000053811288CBF6FF002000020704702F0A7
:10EE8000ABBA02F0AFBA02F0B9BA02F0C9BA02F0F6
:10EE9000E1BA02F0F1BA08B502F086FB003818BFFB
:10EEA000012008BD02F086BB2DE9F04FFF29ADF52A
:10EEB0000D7D0C46164675D80DF598780A46014624
:10EEC0004046FAF707FC14F00F010ABF1022C1F107
:10EED00010011146234618BFCAB20C449C425DDCA7
:10EEE0000FAD10212846FFF7D2FF5FFA84F9AA463A
:10EEF000C4F303142A46002312F8011BC9B90133D5
:10EF0000102BF9D1294B5F694FF0040BB847030A66
:10EF10008AF80C008AF80D30BBF1010B4FEA104360
:10EF20004FEA10608AF80E308AF80F00AAF1040A3E
:10EF3000ECD195E80F000DF11C0A8AE80F001022B1
:10EF400000212846F9F7EEF810212846FFF7A1FF27
:10EF50009AE80F000BAF87E80F00102103A8FFF716
:10EF600092FF2A46102103A8FBF740FC314600958A
:10EF7000534622464046FBF746FC4E443B4603CBF5
:10EF8000AB42306071601F4606F10806F6D109F108
:10EF90001000C0B20DF50D7DBDE8F08F08F803201C
:10EFA00001339BE76FF00200F4E700BF14F20208A0
:10EFB0002DE9F0411446C8B0A1F111020646024401
:10EFC00007A810230746013B12F8015F00F8015B18
:10EFD0009BB2002BF7D110398DB2FCF75CFF48B122
:10EFE000C54803F0DFF938461021FFF719FEC34882
:10EFF00003F0D8F910210DF12C0803A8FFF743FF07
:10F000004246102103A8FBF7F1FB3B462A09CDF845
:10F01000008021463046FBF706FC6219284612F8AC
:10F02000013C012B04D1681EC0B248B0BDE8F0819C
:10F03000022B05D112F8023C022BF5D1A81EF3E7F2
:10F04000032B09D112F8023C032BEDD112F8033C3B
:10F05000032BE9D1E81EE7E7042B0DD112F8023C9F
:10F06000042BE1D112F8033C042BDDD112F8043C4F
:10F07000042BD9D1281FD7E7052B11D112F8023C58
:10F08000052BD1D112F8033C052BCDD112F8043C4D
:10F09000052BC9D112F8053C052BC5D1681FC3E764
:10F0A000062B15D112F8023C062BBDD112F8033CF9
:10F0B000062BB9D112F8043C062BB5D112F8053C49
:10F0C000062BB1D112F8063C062BADD1A81FABE739
:10F0D000072B19D112F8023C072BA5D112F8033CDB
:10F0E000072BA1D112F8043C072B9DD112F8053C47
:10F0F000072B99D112F8063C072B95D112F8073C43
:10F10000072B91D1E81F8FE7082B22D112F8023C80
:10F11000082B89D112F8033C082B85D112F8043C46
:10F12000082B81D112F8053C082B7FF47DAF12F833
:10F13000063C082B7FF478AF12F8073C082B7FF4CD
:10F1400073AF12F8083C082B7FF46EAFA5F10800EE
:10F150006AE7092B2AD112F8023C092B7FF464AF2D
:10F1600012F8033C092B7FF45FAF12F8043C092B23
:10F170007FF45AAF12F8053C092B7FF455AF12F813
:10F18000063C092B7FF450AF12F8073C092B7FF4A3
:10F190004BAF12F8083C092B7FF446AF12F8093C3C
:10F1A000092B7FF441AFA5F109003DE70A2B2FD1D0
:10F1B00012F8023C0A2B7FF437AF12F8033C0A2BFB
:10F1C0007FF432AF12F8043C0A2B7FF42DAF12F813
:10F1D000053C0A2B7FF428AF12F8063C0A2B7FF47B
:10F1E00023AF12F8073C0A2B7FF41EAF12F8083C3D
:10F1F0000A2B7FF419AF12F8093C0A2B7FF414AFE5
:10F2000012F80A3C0A2B7FF40FAFA5F10A000BE7B6
:10F210000B2B34D112F8023C0B2B7FF405AF12F804
:10F22000033C0B2B7FF400AF12F8043C0B2B7FF454
:10F23000FBAE12F8053C0B2B7FF4F6AE12F8063C41
:10F240000B2B7FF4F1AE12F8073C0B2B7FF4ECAEE6
:10F2500012F8083C0B2B7FF4E7AE12F8093C0B2B9D
:10F260007FF4E2AE12F80A3C0B2B7FF4DDAE12F80D
:10F270000B3C0B2B7FF4D8AEA5F10B00D4E60C2B86
:10F280003ED112F8023C0C2B7FF4CEAE12F8033CB8
:10F290000C2B7FF4C9AE12F8043C0C2B7FF4C4AEE7
:10F2A00012F8053C0C2B7FF4BFAE12F8063C0C2B79
:10F2B0007FF4BAAE12F8073C0C2B7FF4B5AE12F80F
:10F2C000083C0C2B7FF4B0AE12F8093C0C2B7FF4F9
:10F2D000ABAE12F80A3C0C2B7FF4A6AE12F80B3C36
:10F2E0000C2B7FF4A1AE12F80C3C0C2B7FF49CAEDF
:10F2F000A5F10C0098E600BFE1EC0208AAED0208B7
:10F300000D2B3ED112F8023C0D2B7FF48DAE12F87E
:10F31000033C0D2B7FF488AE12F8043C0D2B7FF4D8
:10F3200083AE12F8053C0D2B7FF47EAE12F8063C3E
:10F330000D2B7FF479AE12F8073C0D2B7FF474AEE1
:10F3400012F8083C0D2B7FF46FAE12F8093C0D2B20
:10F350007FF46AAE12F80A3C0D2B7FF465AE12F80A
:10F360000B3C0D2B7FF460AE12F80C3C0D2B7FF4A0
:10F370005BAE12F80D3C0D2B7FF456AEA5F10D00DF
:10F3800052E60E2B43D112F8023C0E2B7FF44CAE0A
:10F3900012F8033C0E2B7FF447AE12F8043C0E2B00
:10F3A0007FF442AE12F8053C0E2B7FF43DAE12F80E
:10F3B000063C0E2B7FF438AE12F8073C0E2B7FF480
:10F3C00033AE12F8083C0E2B7FF42EAE12F8093C37
:10F3D0000E2B7FF429AE12F80A3C0E2B7FF424AEDC
:10F3E00012F80B3C0E2B7FF41FAE12F80C3C0E2BC8
:10F3F0007FF41AAE12F80D3C0E2B7FF415AE12F806
:10F400000E3C0E2B7FF410AEA5F10E000CE60F2B78
:10F4100048D112F8023C0F2B7FF406AE12F8033CE1
:10F420000F2B7FF401AE12F8043C0F2B7FF4FCADE0
:10F4300012F8053C0F2B7FF4F7AD12F8063C0F2BAA
:10F440007FF4F2AD12F8073C0F2B7FF4EDAD12F80C
:10F45000083C0F2B7FF4E8AD12F8093C0F2B7FF42A
:10F46000E3AD12F80A3C0F2B7FF4DEAD12F80B3C33
:10F470000F2B7FF4D9AD12F80C3C0F2B7FF4D4ADD9
:10F4800012F80D3C0F2B7FF4CFAD12F80E3C0F2B72
:10F490007FF4CAAD12F80F3C0F2B7FF4C5ADA5F178
:10F4A0000F00C1E5102B08BFA5F11000BCE500BF9F
:10F4B0002DE9F0432C4D4FF00009C1B080460C46B9
:10F4C00017461E4685F8019085F8029001F084FFEA
:10F4D000002840D04FF4807249466846F8F722FE73
:10F4E00023071EBF24F00F041034A4B221466A463D
:10F4F0004046FFF75DFDC4B2224669461B48DFF86F
:10F500006C80FAF7E7F801F08FFC10F0FF0F0CBFEA
:10F51000174818483246394602F044FF2146404613
:10F52000FFF77EFB144802F03DFF144900234B72A5
:10F53000134BCF801B680E720C71C1F800800BB1A9
:10F5400007C99847EB780BB92B793BB101236B7056
:10F5500041B0BDE8F08322464146CFE7094B1B6B23
:10F56000984702F05FFEF3E7A3240020A4230020C5
:10F57000F2EC020804ED0208AAED0208AC24002017
:10F580002474002014F2020801F0A8BF01F0ACBFFF
:10F5900001F0D4BFF82801D801F0D6BF6FF0020007
:10F5A000704701F0B9BF01F0BDBF01F0D9BF01F054
:10F5B000DDBF01F0E7BF000070B5074B5D6C04468E
:10F5C000010A4FF4E860A847E1B22B4640F24170CF
:10F5D000BDE87040184700BF14F202082DE9F04F53
:10F5E0009BB001F0BDFF0C9001F096FF0D9001F073
:10F5F000A5FF109001F078FF119001F06FFF0E90C1
:10F6000001F0C0FF129002F055FB002800F0A2802C
:10F6100014A802F05BFBBDF86230DDF850B09DF835
:10F6200064809DF854700B9301F0FEFB10F0FF0F07
:10F6300040F08880169C9DF86060013601F0F4FB74
:10F6400010F0FF0242D1139201F078FF6FF07F4378
:10F6500008930D9B07930C9BDFF83CA103930B9B36
:10F66000139A0F905FFA86F9CDE90193DAF81C300E
:10F67000009701201D46CDE90522049023464FFA4C
:10F6800088F1A8470F9B139AB3FA83F35B09099398
:10F690000D9B08930C9B0393BDF8403002930B9B8A
:10F6A000CDE90023DAF818300120CDE90420CDE9B6
:10F6B00006221D463A464B462146A8470120DAF865
:10F6C0005430FF2198471298FFF776FF01F0ACFB0A
:10F6D000C0B20228304F2ED100206FF07F43CDE919
:10F6E00007030B9B119AF6B2CDE901630E9B0093C1
:10F6F000FB694FF0010A1D46CDE90500CDE9030A7B
:10F7000023464FFA88F1A847052302930B9BBD6956
:10F710000E9ACDF824A00020CDE90003CDE9070022
:10F72000CDE905A0CDE9030033462146A8477B6D0E
:10F73000FF21504698475846FB68984700201BB069
:10F74000BDE8F08F01F070FBC0B2022804BF179C27
:10F75000640870E701F0CAFD834601F02BFE804685
:10F7600001F0D6FD074601F013FE0B9001F05CFBA3
:10F7700010F0FF0F06D1FFF736FB044601F0F6FD4F
:10F78000461C5BE701F050FBC0B20228F6D1FFF740
:10F790002AFB4408F2E700BF14F202080A4808B541
:10F7A0000A4B03600A4B83600A4B43600A4BC360F9
:10F7B0000A4B03610A4B83610A4B1B689847FFF7AA
:10F7C0000DFF002008BD00BF8023002035ED00089C
:10F7D000B1F4000841EC0008CDEC00086DEC000825
:10F7E000FDEB000814F20208F8B5294B17465A78C9
:10F7F00005460C461E460AB11B79E3B101F0ECFD4B
:10F80000E0B12146234A2846FFF74EFBC4B2224D01
:10F81000FFF7E4FE02F0FEFC2B6B984701237370A8
:10F8200097B17371AB6B98477379002BFCD17378E8
:10F8300053B902F0F7FC6FF0050028E02246294694
:10F840001448F9F747FFE2E7124EAB6A214630460B
:10F850009847FCF720FBD0B101F0BEFD58B10F482E
:10F8600002F0A0FDA4F1100030441021FFF7D8F9F8
:10F870000B4802F097FD21460A4802F093FD054827
:10F880002146FFF7CDF9064802F08CFD0020F8BDB7
:10F89000A3240020A423002014F2020816ED02087D
:10F8A000AAED020827ED0208B0F5803F70B50446C6
:10F8B00042D2431E0D2B224B4FF0000298BF0F2463
:10F8C000C3E900229A601F4B5CB19A781AB9DA78C2
:10F8D0000AB91A792AB11C4802F064FD6FF00500DC
:10F8E00070BD0122194D5A704CB99C705C70DC706F
:10F8F0001C7102F097FC2B6B98470020F0E74FF645
:10F90000FF718C426E6B09D19A70FFF767FE2B6B0B
:10F9100098470020B04702F07DFCEEE74FF6FE71FD
:10F920008C4201D1DA70F0E74FF6FD718C4201D1C3
:10F930001A71EAE72046EDE76FF00200D0E700BF5A
:10F94000AC240020A324002041ED020814F2020898
:10F9500008B5074B074A0344934205D801F0CCFC95
:10F96000FFF73CFE002008BD6FF00200FBE700BF80
:10F97000802E0FF7809E473008B5431F072B05D810
:10F9800001F0CCFCFFF72AFE002008BD6FF002005A
:10F99000FBE7000010B5044601F046FA10F0FF0046
:10F9A0000CD17D2C14D0FA2C1CD0B4F5FA7F1BD0CE
:10F9B000092C0ED96FF00204204610BD01F034FA74
:10F9C000C0B2022805D1094BA4F596529A42F0E73D
:10F9D0000446204601F0B8FC04460028ECD1FFF7AD
:10F9E000FDFDE9E70124F4E70224F2E7780D0700C2
:10F9F000032808B505D801F0BFFCFFF7EFFD002094
:10FA000008BD6FF00200FBE7042808B505D901F036
:10FA1000C5FCFFF7E3FD002008BD6FF00200FBE727
:10FA200008B5431F112B05D801F0CAFCFFF7D6FD1E
:10FA3000002008BD6FF00200FBE70000084BA0F5B6
:10FA400016729A4210B5044606D8FFF7C7FD204645
:10FA5000BDE8104001F02ABD6FF0020010BD00BFEC
:10FA6000E80A0300084BA0F516729A4210B5044646
:10FA700006D8FFF7B3FD2046BDE8104001F022BDD7
:10FA80006FF0020010BD00BF8891040010B501F0B6
:10FA90007FFD0446F7F7B4FFFFF7A0FD204610BD39
:10FAA00008B502F0B7FB024A13680133136008BDC2
:10FAB00014280020094B1B6810B513B1084B1B6DAF
:10FAC0003BB9084C236823B102F0ACFB2368013B2F
:10FAD0002360BDE81040044802F064BC0C270020FD
:10FAE000280300201428002061ED0208F7B5164C09
:10FAF000164E2368164D30682F68013B2360154B66
:10FB000021681A6864234343511A3844B3FBF0F365
:10FB1000114802F047FC236810493BB14B6B01933D
:10FB200041F2883003B0BDE8F04018470C4833601C
:10FB300002782B600B6B019322F00802027003B075
:10FB4000BDE8F040184700BF0C270020DC2400204F
:10FB5000E0240020102700206CED020814F20208B7
:10FB6000E4240020024A136801331360FFF7BEBF8C
:10FB7000DC240020FFF7F6BF10B5064C20680130EA
:10FB80002060114604481A4602F00CFCBDE8104003
:10FB9000FFF7ACBFE02400208AED0208F8B52D4D38
:10FBA0002D4A2B78976A2D4C2D4E002B33D0236D88
:10FBB000013B2365606CD3689847E17D2948B847CD
:10FBC000616C294802F0EEFB3268216D2748511A1A
:10FBD00002F0E8FBE36C626C13446364626CA36C38
:10FBE0009A4282BF224B1B686364236D23B1BDE838
:10FBF000F840204809F09EBC1F4A1E48137823F0A5
:10FC00000403137009F0FEFB10B11A4809F042FC1E
:10FC100000232B70F8BD194D12482B68013B2B6057
:10FC2000E17DB847326829681048511A02F0BAFBE2
:10FC30002B68002BDBD1104A0E48137823F0040305
:10FC4000137009F0DFFB0028E4D0BDE8F840094854
:10FC500009F020BC0827002014F202082803002025
:10FC60001027002014270020ADED0208BFED020888
:10FC700004270020E8240020E42400200C27002092
:10FC8000F8B52E4D2E4A2B78976A2E4C2E4E002B0F
:10FC900035D0236D013B2365606CD3689847E17DC7
:10FCA0002A48B847616C2A4802F07CFB3268216D13
:10FCB0002848511A02F076FB226D33689B1A264AB7
:10FCC0001178B3FBF1F201FB1233244A52F82330CE
:10FCD0006364236D23B1BDE8F840214809F02ABCD4
:10FCE000204A1F48137823F00403137009F08AFB9D
:10FCF00010B11B4809F0CEFB00232B70F8BD1A4D44
:10FD000012482B68013B2B60E17DB84732682968B7
:10FD10001048511A02F046FB2B68002BDBD1114A28
:10FD20000F48137823F00403137009F06BFB0028CD
:10FD3000E4D0BDE8F8400A4809F0ACBB0827002031
:10FD400014F20208280300201027002014270020A6
:10FD5000ADED0208BFED02080025002004250020BB
:10FD6000E8240020E42400200C27002070B50D4C6E
:10FD7000C00000220221824201D1002070BDC1F3E7
:10FD8000001383EA1123D51043EA410302F007066A
:10FD9000C3F3080103F00103B340665D33436355C9
:10FDA0000132E8E714270020064B10B5064C1B6B08
:10FDB0009847236823B102F035FA2368013B23609A
:10FDC00010BD00BF14F202081428002038B50D4DF4
:10FDD000287810F0010411D1FFF762FE2B7843F070
:10FDE00001032B70084B186B93F82410074B4FF648
:10FDF000FF72DB6B49B29847204638BD6FF00500B3
:10FE0000FBE700BFE42400202803002014F20208CE
:10FE10000F4B104810B500221A7009F0F3FA10B118
:10FE20000C4809F037FB0C4809F0ECFA10B10A480D
:10FE300009F030FB094B0A4CDB6A9847236803B989
:10FE400010BD02F0EFF92368013B2360F6E700BF25
:10FE5000E4240020E82400201C6F002014F2020893
:10FE6000142800202DE9F04F284A137899078DB007
:10FE7000834647D4264C274D206B43F00203137072
:10FE8000EB689847206894F82410A26A6368A66813
:10FE90000A93277B0B96A68A94F816C094F818E06C
:10FEA00094F8198094F81A9094F81BA0E36AB6B2FB
:10FEB000CDE907A30B9B0093CDE901760A9BEE6980
:10FEC000CDE90589CDE903CE49B2C0B2B047636B35
:10FED000B3B96B6B6FF07F409847322001F02FFF72
:10FEE0002B6C00209847EB6AABF800009847074A54
:10FEF000137823F00203137000200DB0BDE8F08FDB
:10FF00006B6EE7E76FF00500F7E700BFE424002021
:10FF10002803002014F2020810B50446FFF7C0FDC4
:10FF2000226B144B1344144A934220D894F8243083
:10FF30000933DBB21F2B1AD86368062B17D8A368C6
:10FF4000053B072B13D8237B013B032B0FD82368DA
:10FF5000022B0CD8A36A094AA3F59653934206D8FC
:10FF600007485422214609F0A2FB002010BD6FF083
:10FF70000200FBE7802E0FF7809E4730780D0700C8
:10FF80002803002008B50349542209F090FB002003
:10FF900008BD00BF280300202DE9F04F324C257822
:10FFA0008DB015F004050B905BD1FFF779FD237838
:10FFB0002E482F4E43F00403237002F0F3F92D482E
:10FFC0002D4B03602D4B83602D4B43602D4B2E4CEE
:10FFD000C3602E4B036133689847E07DFFF7C6FE90
:10FFE000206BF3689847206894F82410A26A63682D
:10FFF000A7680A9794F80CC0A78A94F816E094F8BA
:020000040801F1
:10000000188094F8199094F81AA094F81BB0E46A38
:10001000BFB2CDE907B40A9C0094CDE903E8CDE96D
:1000200001C749B2C0B2CDE9059AF469A047184B9F
:100030000B9A1A601A68174B17481A604FF0FF3175
:10004000164B00952A4609F0C3F94FF4FA7112488D
:1000500009F0AAFA104809F06DFA28460DB0BDE87B
:10006000F08F6FF00500F9E7E4240020DBED0208D3
:1000700014F20208B8240020B5FA000879FB000841
:10008000A9FD000865FB00082803002075FB000897
:100090000C27002010270020E82400209DFB0008EA
:1000A0002DE9F04F2B4D0446287810F008088DB04C
:1000B0004DD1002C4BDDFFF7F3FC2B78264843F0A5
:1000C00008032B70254B0360254B8360254B264D81
:1000D0004360264BC360264B03612B689847254B32
:1000E0001C601A68244C254B206B1A60EB689847FB
:1000F00020686168A268237B26690B930A96A68A0A
:10010000276A94F816C094F817E0237E94F81990A3
:1001100094F81AA094F81BB0247FCDF80CC0CDE958
:1001200004E3B6B20A9B0093BFB2CDE908B40B9BBF
:10013000AC69C0B2CDE9069ACDE90167A04741F2AA
:1001400088306B6B984740460DB0BDE8F08F6FF07C
:100150000500F9E7E4240020B8240020B5FA0008DF
:1001600079FB0008A9FD000814F2020865FB0008ED
:1001700075FB00080C270020280300201027002012
:100180002DE9F04F364C257815F004058DB0074663
:1001900063D1FFF785FC23783248334E43F00403E4
:1001A0002370324B324C01221A70324B0360324BB7
:1001B0008360324B4360324BC360324B0361336820
:1001C00098477B6C6364BB6CA364FB6CE3643B6D1E
:1001D0002365E07DFFF7CAFD2B4B626C1A602B4B49
:1001E000226D1A60606CF3689847206894F82410B8
:1001F000A26A6368A7680B9794F80CC0A78A94F862
:1002000016E094F8188094F8199094F81AA094F8CD
:100210001BB0E46ABFB2CDE907B40B9C0094CDE9F2
:1002200003E8CDE901C749B2C0B2CDE9059AF46946
:10023000A047174B174800952A464FF0FF3109F0A9
:10024000C7F84FF4FA71134809F0AEF9114809F0F4
:1002500071F928460DB0BDE8F08F6FF00500F9E7A1
:10026000E4240020B824002014F20208082700200B
:1002700028030020B5FA000879FB0008A9FD000852
:1002800065FB000875FB00080427002010270020EC
:100290009DFB0008E824002038B50546FCF758F817
:1002A000224C0A283DD8DFE800F0060F14191E235F
:1002B000282D323C37001E4B1E495B5DA36028464B
:1002C00011F02AF9606038BD1B4B1C495B5DA360CF
:1002D000F5E71B4B1B495B5DA360F0E71A4B1B491D
:1002E0005B5DA360EBE71A4B1A495B5DA360E6E731
:1002F000194B1A495B5DA360E1E7194B19495B5D36
:10030000A360DCE7184B19495B5DA360D7E7184B86
:1003100018495B5DA360D2E7174B18495B5DA3608A
:10032000CDE70723A36000236360CCE72803002008
:10033000D0F0020838EF0208D8F0020858EF02089F
:10034000D0F0020898EF0208D0F00208B8EF0208D7
:10035000D0F00208D8EF0208D0F00208F8EF020847
:10036000E8F0020838F00208D0F0020818F002089D
:10037000EEF0020890F00208D8F0020850F00208EF
:10038000014B83F824007047280300202DE9F04F2B
:10039000914B197811F004048BB00646984640F052
:1003A00017818E4FFFF77CFB21464FF400728C487B
:1003B000F7F7B8FE3C7021462246894C8029CBB223
:1003C00040F0BE80002A40F0C380022001F062FFAE
:1003D0001CF0FEFE00256FF000493B78AB4200F3B5
:1003E000BE8098F800307F487F4F804C43F0040374
:1003F00088F800307E4B01221A707E4B03607E4BE2
:1004000083607E4B43607E4BC3607E4B03613B68E1
:100410009847734B7C481B686364B36CA364F36CAC
:10042000E364336D2365616C01F0BCFFA16C774818
:1004300001F0B8FFE16C764801F0B4FF216D75481A
:1004400001F0B0FFE07DFFF791FC734B626C1A6026
:10045000724B226D1A604FF47A73E3622168704820
:1004600001F0A0FF94F824106E4849B201F09AFF01
:10047000A16A6D4801F096FF61686C4801F092FF37
:10048000A1686B4801F08EFF217B6A4801F08AFF6A
:10049000A18A694889B201F085FFA17D674801F012
:1004A00081FF217E664801F07DFF617E654801F095
:1004B00079FFA17E644801F075FFE17E634801F099
:1004C00071FFE16A624801F06DFFE17D614801F072
:1004D00069FF206894F82410A26A6368A66894F8FB
:1004E0000CC0A58A94F816E094F8188094F8199036
:1004F00094F81AA094F81BB0E46A0096ADB2CDE966
:1005000003E8CDE901C5CDE907B449B2FC69C0B241
:10051000CDE9059AA04700244F4B5048009422464D
:100520004FF0FF3108F054FF4FF4FA614B4809F0E7
:100530003BF84A4808F0FEFF20460BB0BDE8F08FBC
:10054000706CF26C02FB0102B06C824202D9013B7A
:100550003B703AE744F82120013101222EE71CF0DC
:100560005BFE3A7854F82510531B99FBF3F30133E3
:1005700090FBF3F32B449D4208BF002354F8230063
:10058000414044F8251054F8251054F82300414008
:1005900044F8231054F8251054F82300414044F83F
:1005A000251054F8231054F82200414044F8231039
:1005B00054F8231054F82200414044F8221054F813
:1005C000231054F822204A4044F82320013504E740
:1005D0006FF00500B1E700BFE424002000250020F3
:1005E00004250020B824002014F20208280300206B
:1005F00008270020B5FA000879FB0008A9FD0008CB
:1006000065FB000875FB0008E5ED0208FAED02083D
:100610000EEE020824EE0208042700201027002016
:1006200031EE020841EE020851EE020860EE0208C7
:1006300074EE020887EE02089AEE0208B0EE020895
:10064000C1EE0208D1EE0208E5EE0208F9EE02085A
:100650000EEF020822EF020881FC0008E8240020C7
:1006600008B503490C2209F022F8002008BD00BF9C
:100670001C03002038B505460B4CFFF711FAAB6898
:10068000A3602B68094823606B68094D6360094BC0
:1006900043602B6898472068EB6B228994F904101B
:1006A0009847002038BD00BF1C030020B82400205C
:1006B00014F20208A9FD00081B2937B5434B054673
:1006C0000C460FD00CD80A2934D00D2932D0082975
:1006D0000BD01A78012A5ED15B2C64D1022202E091
:1006E0007F29F5E701221A7053E0394900221A7078
:1006F0000B68002B4DD0013B0B6036490824CA54CF
:10070000284601220DF107018DF8074001F0EEFDAA
:10071000202301220DF1070128468DF8073001F052
:10072000E5FD01220DF1070128468DF8074001F093
:10073000DDFD2EE000221A70264B1B7803B300F07B
:1007400001FA88B10A2301220DF1070128468DF82C
:10075000073001F0CBFD0D2301220DF107012846E2
:100760008DF8073001F0C2FD1A48F5F709FD194967
:100770000246284616F026FE1749184801F012FED8
:1007800040F6010213480021F7F7CCFC104B002281
:100790001A6003B030BD022A05D1A4F14102012A3A
:1007A00001D800229FE70A49002018700B6840F228
:1007B000FE729342EDD85A1C0A600649CC54885404
:1007C00000F0C0F90028E4D0ABE700BF18280020F3
:1007D000703000206C280020ACED0208FEF002080A
:1007E00008B50B490B4801F0DDFD142200210A4831
:1007F000F7F798FC40F6010208480021F7F792FC51
:10080000074B00221A60BDE8084017F0A9B800BFE6
:10081000ACED0208FEF002081C2800206C28002025
:100820007030002010B5094C0948224640F2DC61C6
:1008300001F02CFBE368013307D1204640F2DC6273
:10084000BDE810400021F7F76DBC10BDC076002058
:1008500000E00308024840F2DC620021F7F762BCC6
:10086000C0760020024A03484FF4257101F0B6BB60
:100870002C74002000F00308024A034840F2DC61B7
:1008800001F0ACBBC076002000E00308024B03443B
:1008900093F8BC01704700BF2C740020044A104438
:1008A00080F8BC1103484FF4257101F097BB00BFDD
:1008B0002C74002000F003080829034608D90648D4
:1008C00002681A6042685A60027A1A72F5F758BCD8
:1008D0006FF00800704700BFF5750020082908B5C3
:1008E0000A4612D80A4B0021196059601972014654
:1008F0001846F8F7EFFE6FF4E4728218BDE808407E
:1009000004484FF4257101F069BB6FF0020008BD87
:10091000F575002000F00308014BD3F8D4017047AF
:100920002C740020034A4FF42571C2F8D401024808
:1009300001F054BB2C74002000F00308014B93F825
:10094000700270472C740020054A08B54FF42571D9
:1009500082F87002034801F041FBC0B208BD00BF3D
:100960002C74002000F003081F290AD9064B03F15C
:10097000200253F8041B40F8041B9342F9D10020D5
:100980007047F720704700BF277600201F290AD93B
:10099000064B03F1200253F8041B40F8041B93425A
:1009A000F9D100207047F720704700BF477600203C
:1009B0001F290AD9064B03F1200253F8041B40F803
:1009C000041B9342F9D100207047F720704700BF05
:1009D00067760020034A4FF42571C2F8B40102483B
:1009E00001F0FCBA2C74002000F00308034A4FF415
:1009F0002571C2F8B801024801F0F0BA2C74002049
:100A000000F00308024B034493F8BF01704700BF96
:100A10002C740020044A104480F8BF1103484FF49E
:100A2000257101F0DBBA00BF2C74002000F0030830
:100A3000014BD3F8C40170472C740020034A4FF4D3
:100A40002571C2F8C401024801F0C8BA2C74002014
:100A500000F003080F290AD9064B03F1100253F8DE
:100A6000041B40F8041B9342F9D1002070476FF03B
:100A70000800704716760020102938B504460D4648
:100A80001BD804D00E4810220021F7F74BFB234659
:100A900029198B420CD12A4621460948F8F71AFE3B
:100AA000BDE83840074A08484FF4257101F096BA6E
:100AB00013F8012B203A5E2AEBD96FF0020038BD03
:100AC000167600202C74002000F00308112930B5A0
:100AD00003460FD9094A02F11005144603CCAC4273
:100AE00018605960224603F10803F6D122881A8063
:100AF000002030BD6FF00800FBE700BF0476002047
:100B0000122938B505460C4612D804D00A481222DC
:100B10000021F7F707FB224629460748F8F7DAFDD8
:100B2000BDE83840054A06484FF4257101F056BA31
:100B30006FF0020038BD00BF047600202C74002046
:100B400000F00308014B93F8C80170472C74002093
:100B5000034A4FF4257182F8C801024801F03EBAF9
:100B60002C74002000F00308034A4FF4257182F82A
:100B7000FA01024801F032BA2C74002000F0030898
:100B8000014B93F8FA0170472C740020014B93F845
:100B9000300070472C740020034A4FF4257182F80E
:100BA0003000024801F01ABA2C74002000F003084B
:100BB000044A1368036053684360936883600020AD
:100BC000704700BFCE740020064A03681360436874
:100BD0005360836893600448A23A4FF4257101F092
:100BE000FDB900BFCE74002000F00308072981BFC3
:100BF000044A13680360536886BF436000206FF0A7
:100C0000080070476574002008290BD1074A036863
:100C1000C2F839304368C2F83D3005484FF42571B9
:100C200001F0DCB96FF00200704700BF2C740020A7
:100C300000F003080F290AD9064B03F1100253F8FC
:100C4000041B40F8041B9342F9D1002070476FF059
:100C5000080070476D74002010290ED1084B00F178
:100C6000100250F8041B43F8041B9042F9D1054AC6
:100C700005484FF4257101F0B1B96FF002007047DB
:100C80006D7400202C74002000F003080F290AD98D
:100C9000064B03F1100253F8041B40F8041B934267
:100CA000F9D1002070476FF0080070477D74002074
:100CB00010290ED1084B00F1100250F8041B43F824
:100CC000041B9042F9D1054A05484FF4257101F003
:100CD00085B96FF0020070477D7400202C740020ED
:100CE00000F00308032981BF044BD3F8613003608F
:100CF000002098BF6FF00800704700BF2C740020E0
:100D0000042908D1054A0368C2F8613004484FF449
:100D1000257101F063B96FF0020070472C74002058
:100D200000F00308072981BF044A13680360536871
:100D300086BF436000206FF0080070475D7400209C
:100D400008290BD1074A0368C2F831304368C2F85A
:100D5000353005484FF4257101F040B96FF00200BD
:100D6000704700BF2C74002000F00308032981BFE6
:100D7000044BD3F865300360002098BF6FF0080083
:100D8000704700BF2C7400200F290AD9064B03F1CD
:100D9000100253F8041B40F8041B9342F9D10020C1
:100DA00070476FF0080070479574002010290ED12D
:100DB000084B00F1100250F8041B43F8041B90424A
:100DC000F9D1054A05484FF4257101F007B96FF0D4
:100DD00002007047957400202C74002000F0030876
:100DE000014B93F8B10070472C740020034A4FF474
:100DF000257182F8B100024801F0F0B82C7400208F
:100E000000F00308014B93F8B00070472C740020E9
:100E1000034A4FF4257182F8B000024801F0DEB8B1
:100E20002C74002000F00308014B187A704700BFB3
:100E30002C740020034A4FF425711072024801F00F
:100E4000CDB800BF2C74002000F00308014B93F8CC
:100E5000AE0070472C740020034A4FF4257182F8CD
:100E6000AE00024801F0BAB82C74002000F003086C
:100E7000014B93F8B40070472C740020034A4FF4E0
:100E8000257182F8B400024801F0A8B82C74002043
:100E900000F00308014B93F8AF0070472C7400205A
:100EA000034A4FF4257182F8AF00024801F096B86A
:100EB0002C74002000F00308014B93F8B200704737
:100EC0002C740020034A4FF4257182F8B2000248C6
:100ED00001F084B82C74002000F00308014B93F853
:100EE000B30070472C740020034A4FF4257182F838
:100EF000B300024801F072B82C74002000F003081F
:100F0000014BD3F8B80070472C740020034A4FF40B
:100F10002571C2F8B800024801F060B82C740020B6
:100F200000F00308014BD3F8BC0070472C7400207C
:100F3000034A4FF42571C2F8BC00024801F04EB8D4
:100F40002C74002000F00308034A4FF42571C2F806
:100F5000C800024801F042B82C74002000F00308D9
:100F6000014BD3F8C80070472C740020014B93F854
:100F7000CC0070472C740020034A4FF4257182F88E
:100F8000CC00024801F02AB82C74002000F00308BD
:100F9000014BD3F8C00070472C740020034A4FF473
:100FA0002571C2F8C000024801F018B82C74002066
:100FB00000F00308014BD3F8C40070472C740020E4
:100FC000034A4FF42571C2F8C400024801F006B884
:100FD0002C74002000F00308014B93F8B500704713
:100FE0002C740020034A4FF4257182F8B5000248A2
:100FF00000F0F4BF2C74002000F00308014B93F8BC
:10100000CD0070472C740020034A4FF4257182F8FC
:10101000CD00024800F0E2BF2C74002000F003086D
:10102000014B93F8CE0070472C740020034A4FF414
:10103000257182F8CE00024800F0D0BF2C74002049
:1010400000F00308014B93F8CF0070472C74002088
:10105000034A4FF4257182F8CF00024800F0BEBF6A
:101060002C74002000F00308014B93F8D000704767
:101070002C740020034A4FF4257182F8D0000248F6
:1010800000F0ACBF2C74002000F00308014BD3F833
:10109000D40070472C740020034A4FF42571C2F825
:1010A000D400024800F09ABF2C74002000F003081E
:1010B000014BD3F8D80070472C740020034A4FF43A
:1010C0002571C2F8D800024800F088BF2C740020B7
:1010D00000F00308014B93F8680270472C7400205D
:1010E000034A4FF4257182F86802024800F076BF87
:1010F0002C74002000F00308014BB3F96A0270471A
:101100002C740020034A4FF42571A2F86A020248A9
:1011100000F064BF2C74002000F00308014BD3F8EA
:101120006C0270472C740020034A4FF42571C2F8FA
:101130006C02024800F052BF2C74002000F003083B
:10114000014B9888704700BFC0760020034A40F2E8
:10115000DC619080024800F041BF00BFC0760020F3
:1011600000E00308034A4FF4257182F89302024815
:1011700000F034BF2C74002000F00308014B93F8FA
:10118000930270472C74002030B4094C034600F1E0
:10119000380518685968224603C20833AB42144622
:1011A000F7D130BC024A034840F2DC6100F016BFC0
:1011B000C076002000E0030800487047C076002099
:1011C00030B4094C034600F12005186859682246DE
:1011D00003C20833AB421446F7D130BC034A04487B
:1011E00040F2DC6100F0FABEF8760020C076002004
:1011F00000E0030800487047F876002008B5084B67
:1012000001464FF4C2721846F8F764FABDE8084088
:10121000A0F1580240F2DC61024800F0DFBE00BFDE
:101220001877002000E00308004870471877002076
:1012300008B5084B01464FF4D0721846F8F74AFA41
:10124000BDE80840A0F5EE7240F2DC61024800F013
:10125000C5BE00BF9C78002000E00308004870472E
:101260009C78002008B5084B01464FF45872184688
:10127000F8F730FABDE80840A0F55F7240F2DC6193
:10128000024800F0ABBE00BF3C7A002000E003083B
:10129000004870473C7A00200048704708750020DD
:1012A00008B5074B0146D0221846F8F713FABDE8F7
:1012B0000840A0F1DC024FF42571024800F08EBE18
:1012C0000875002000F00308014BD3F8AC0170470B
:1012D0002C740020034A4FF42571C2F8AC01024877
:1012E00000F07CBE2C74002000F00308014BD8688D
:1012F000704700BF2C740020034A4FF42571D06062
:10130000024800F06BBE00BF2C74002000F0030800
:10131000014B187C704700BF2C740020034A4FF427
:1013200025711074024800F059BE00BF2C740020D3
:1013300000F00308034B1A7A0AB9588A7047D86A32
:10134000704700BF2C740020064B1A7A32B95882BD
:10135000044A05484FF4257100F040BE022A08BF38
:10136000D862F5E72C74002000F00308014B187DCB
:10137000704700BF2C740020034A4FF4257110758C
:10138000024800F02BBE00BF2C74002000F00308C0
:10139000014BD88A704700BF2C740020034A4FF4D9
:1013A0002571D082024800F019BE00BF2C740020C5
:1013B00000F00308014B187E704700BF2C7400201A
:1013C000034A4FF425711076024800F007BE00BFB3
:1013D0002C74002000F00308014B987E704700BF7A
:1013E0002C740020034A4FF425719076024800F0D7
:1013F000F5BD00BF2C74002000F003080F290AD9A6
:10140000064B03F1100253F8041B40F8041B9342EF
:10141000F9D1002070476FF0080070479D760020DA
:1014200010290ED1084B00F1100250F8041B43F8AC
:10143000041B9042F9D1054A05484FF4257100F08C
:10144000CDBD6FF0020070479D7600202C74002007
:1014500000F003080F290AD9064B03F1100253F8D4
:10146000041B40F8041B9342F9D1002070476FF031
:1014700008007047AD76002010290ED1084B00F10E
:10148000100250F8041B43F8041B9042F9D1054A9E
:1014900005484FF4257100F0A1BD6FF002007047C0
:1014A000AD7600202C74002000F00308034A4FF4AE
:1014B00025719062024800F091BD00BF2C7400209D
:1014C00000F00308034A4FF425715062024800F00F
:1014D00085BD00BF2C74002000F00308014B586A42
:1014E000704700BF2C740020014B986A704700BF02
:1014F0002C740020034A4FF4257182F8B60002488C
:1015000000F06CBD2C74002000F00308014B93F830
:10151000B60070472C740020014B93F85C027047B2
:101520002C740020034A4FF4257182F85C020248B3
:1015300000F054BD2C74002000F00308014BD3F8D8
:10154000600270472C740020034A4FF42571C2F8E2
:101550006002024800F042BD2C74002000F0030835
:10156000014B93F8670270472C740020034A4FF434
:10157000257182F86702024800F030BD2C7400200B
:1015800000F00308014BB3F8640270472C7400208C
:10159000034A4FF42571A2F86402024800F01EBD10
:1015A0002C74002000F00308014B93F8910270475F
:1015B0002C740020034A4FF4257182F891020248EE
:1015C00000F00CBD2C74002000F00308014B93F8D0
:1015D000920270472C740020034A4FF4257182F860
:1015E0009202024800F0FABC2C74002000F00308BC
:1015F0002DE9F0410025202600F2FB170446324673
:10160000294680F8FA513846F6F78CFD294BD3F875
:1016100000804046F4F7B4FD41460246384604F2E5
:101620001B27F8F757F8324629463846F6F77AFD71
:10163000214BD3F800804046F4F7A2FD4146024614
:10164000384604F23B27F8F745F832462946384633
:10165000F6F768FD194B1E683046F4F791FD3146E8
:1016600002463846F8F736F841F22443C4F86432AB
:101670004FF6B073A4F86A320523C4F86C32102612
:10168000012384F870323246294684F85C52C4F84B
:10169000605284F8685204F27120F6F743FD324636
:1016A000294604F28120F6F73DFD84F89152BDE809
:1016B000F08100BF88000020800000207C00002016
:1016C000F0B50C46ADF5497D6A464FF4487100F01F
:1016D000DDFBBC4F23687E9ABB48009EBB4208BF1F
:1016E0006568BA4B18BF00254FF4FA719A4208BFDB
:1016F000032507F0F7FF4FF4F871864208BF022573
:10170000B148009E07F0EEFF4FF42572864208BFF5
:10171000012500212046F6F705FD002D55D0012DAD
:1017200056D19DF80430237202AE0FCE04F10C05A1
:101730000FC50FCE0FC533682B604FF4C2720BA9D3
:1017400004F13000F7F7C6FF6CAA92E8030004F535
:10175000DA7383E803006E9BA4F8BC311B0C84F899
:10176000BE316F9BC4F8C4319DF8C03184F8C831D4
:10177000DDF8C131C4F8C931DDF8C531C4F8CD3167
:101780009DF8C93184F8D13174AE739BC4F8D4315B
:101790000FCE04F5EC750FC533682B8004F5F57298
:1017A0000DF5F1730DF5F97153F8040B42F8040BC4
:1017B0008B42F9D10022A4F8BF2184F8C121204630
:1017C000FFF716FF0423276063600DF5497DF0BD28
:1017D000AB1E012B51D89DF80430237202AE0FCE00
:1017E00004F10C050FC50FCE0FC533682B604FF405
:1017F000C2720BA904F13000F7F76CFF6CAA92E8F3
:10180000030004F5DA7383E803006E9BA4F8BC318F
:101810001B0C84F8BE31BDF8BB31A4F8BF319DF874
:10182000BD3184F8C131709BC4F8C4319DF8C43116
:1018300084F8C831DDF8C531C4F8C931DDF8C931E3
:10184000C4F8CD319DF8CD3184F8D13175AE749B9B
:10185000C4F8D4310FCE04F5EC750FC533682B8076
:1018600004F5F5720DF5F3730DF5FB7153F8040BE8
:1018700042F8040B8B42F9D1A1E7042DA5D14FF416
:10188000257269462046F7F725FF94F8FA31FF2BB9
:1018900004BF002384F8FA3194F8FB31FF2B10D1F8
:1018A00004F2FB15202200212846F6F73BFC484BAA
:1018B0001E683046F4F764FC314602462846F7F7C6
:1018C00009FF94F81B32FF2B10D104F21B252022B4
:1018D00000212846F6F726FC3E4B1E683046F4F7FA
:1018E0004FFC314602462846F7F7F4FE94F83B32A7
:1018F000FF2B10D104F23B25202200212846F6F7C9
:1019000011FC354B1E683046F4F73AFC314602466E
:101910002846F7F7DFFE94F87032FF2B04BF01234F
:1019200084F8703294F85C32FF2B04BF002384F8F3
:101930005C32D4F86032F82B84BF0023C4F86032E4
:1019400094F86632FF2B01BF41F22443A4F86432BD
:10195000002384F8663294F86732FF2B04BF00231B
:1019600084F8673294F86832FF2B04BF002384F8B0
:10197000683294F86A32FF2B04BF4FF6B073A4F8B4
:101980006A3294F86C32FF2B04BF0523C4F86C3222
:1019900094F89332FF2B04BF012384F8933294F818
:1019A0008132FF2B05D11022002104F28120F6F7AD
:1019B000B9FB94F89132FF2B04BF002384F89132D5
:1019C00000E700BFDDCCBBAA307400201EDD0E0096
:1019D00088000020800000207C000020F0B5984A9C
:1019E000984E10685168ADF5297D01AB03C303AA79
:1019F00095484FF4257100F049FA039BB34202D198
:101A0000049B042B1CD0904803A9FFF759FE039BAD
:101A1000B34217D1049D281F454245418B4B4FF4DB
:101A2000257200211846F6F77DFB044665B14FF498
:101A3000257203A9F7F74EFE00200DF5297DF0BDB4
:101A40000125EBE70025E9E70423436040F2011399
:101A5000A0F8BC314FF4E133C0F8C43101AB0660EB
:101A600080F8BE5103CB0123C4F8C901C4F8CD11DD
:101A7000C4F8D45184F8C85184F8FA512372F5F7A8
:101A8000D3FF10F0FF0F00F0AD80052384F8303055
:101A900041F2883641F27072C4E92E624FF47A71D5
:101AA0004FF4FA62C4E930124FF6B07200250123F8
:101AB000A4F86A220522A4F8AE30A4F8B430C4F821
:101AC0006C22A4F8B050082740F2DC622946604836
:101AD00084F8B63084F8CC3084F8703284F89332CD
:101AE000C4E9357584F8B25084F8CF5084F8D050EA
:101AF00084F86852F6F716FBD02229465548F6F7C7
:101B000011FBF5F791FF544AC4F81B50C3B2534878
:101B10006582AB4208BF1046072323740E23237649
:101B200041F23333C4E909364D4EE06044F6206398
:101B3000E362102241F224432946756006F25620E2
:101B4000A4F864322575E782A57684F85C52C4F85F
:101B5000605284F86752F6F7E5FA1022294606F239
:101B60006620F6F7DFFA3F4B84F891521C68204656
:101B7000F4F706FB1F2843D82022294606F5F0700B
:101B8000F6F7D0FA2046F4F7FBFA2146024606F5AE
:101B9000F070F7F79FFD344B1C682046F4F7F0FA1D
:101BA0001F2838D8202200213048F6F7BBFA2046FB
:101BB000F4F7E6FA214602462C48F7F78BFD2C4B4A
:101BC0001C682046F4F7DCFA1F282ED820220021BA
:101BD0002848F6F7A7FA2046F4F7D2FA214602463B
:101BE000244827E7022384F830304FF6FF73A4F827
:101BF000A2304FF0FF33C4E92933A4F8AC3047E7F3
:101C000006F5F07604F1200354F8042B46F8042B73
:101C10009C42F9D1BFE7154B04F1200254F8041B94
:101C200043F8041B9442F9D1C9E7124B04F1200296
:101C300054F8041B43F8041B9442F9D1FCE600BF9E
:101C400003F10208DDCCBBAA007003082C7400204D
:101C5000C07600200875002080A1031C00A1BC33C1
:101C60004774002088000020800000204776002074
:101C70007C0000206776002010B50B4C0B482246F4
:101C80004FF4257100F002F908482146FFF718FDCE
:101C90002268074B9A4202D16368042B03D0BDE847
:101CA0001040FFF79BBE10BD2C74002000F003080D
:101CB000DDCCBBAA014B1878704700BF8C300020E8
:101CC000014B1870704700BF8C30002030B5074CB6
:101CD000034604F11805224603CAAA421860596057
:101CE000144603F10803F6D1012030BD7430002002
:101CF00030B5074C034600F11805186859682246AC
:101D000003C20833AB421446F7D1012030BD00BFF7
:101D10007430002070B50646022000F0BBFA84192A
:101D200041F1000500F03CFD022000F0B3FAA942A9
:101D300008BFA04200D370BDF6F762F8F4E714F0D4
:101D40000AB800001FB5054C23782BB9684614F07B
:101D5000D7F808B90123237004B010BD8D300020DE
:101D60001FB5104B1B780446C3B1C8B1684614F0C8
:101D700061F930B104289ABF0B4B185C072004B0FE
:101D800010BD009A2260019A6260029A9DF80E309E
:101D9000A260BDF80C20A281A373F0E70120EEE75A
:101DA0000320ECE78D3000200CF1020838B5084D17
:101DB0002D784DB151B14AB114F04EF904289ABFB3
:101DC000044B185C072038BD0120FCE70320FAE72C
:101DD0008D3000200CF1020838B5084D2D784DB13A
:101DE00051B14AB114F084F904289ABF044B185C2D
:101DF000072038BD0120FCE70320FAE78D300020E2
:101E00000CF1020808B5064B1B783BB114F0DEF963
:101E100004289ABF034B185C072008BD0120FCE78B
:101E20008D3000200CF1020808B5064B1B783BB141
:101E300014F016FA04289ABF034B185C072008BD5B
:101E40000120FCE78D3000200CF1020808B5054B9D
:101E5000187830B114F040FA04289ABF024B185C8D
:101E6000072008BD8D3000200CF1020808B5054B95
:101E7000187830B114F08AFA04289ABF024B185C23
:101E8000072008BD8D3000200CF102082DE9F04F2D
:101E900087B083460D46914614F0DEFAB0F5805FB8
:101EA000044657D8BBFBF0F800FB08F8ABEB08037F
:101EB0005A19B2FBF0F100FB1120019308B101FBAC
:101EC0000442B2FBF4F3CDE90283A4EB0B03DFF889
:101ED0008CA00493019B2E46002703EB0A0B039B67
:101EE000BB4203D1002007B0BDE8F08F1B49029828
:101EF000224614F081FADFB9049B03EB0802AA42E0
:101F00000ED2484659460592F7F7E4FB059A019B25
:101F100091441A1B1644029B234401370293DEE7C7
:101F200048462A465946F7F7D5FBA944761BF2E7FF
:101F3000039B7A1C934205D8324651464846F7F730
:101F4000C9FBE8E7484622465146F7F7C3FBA144E0
:101F5000361BE0E76FF00800C5E700BF90300020B7
:101F60002DE9F84F00AF81460C46924614F074FA02
:101F7000ADF5806D6E464FEA90284FF0000B5FFA8A
:101F80008BF1414501D3012021E0B4F5806F09EBCD
:101F900081200AEB812532460ED34FF48061FFF792
:101FA00075FF4FF48062294630461BF0E9F80BF1CB
:101FB000010B78B100200AE02146FFF767FF2246B7
:101FC000294630461BF0DCF8B0FA80F04009BD46E7
:101FD000BDE8F88FA4F58064D1E700002DE9F04F4B
:101FE00087B083460D46144614F036FAB0F5805F8C
:101FF000074670D8224629465846FFF7B1FF18B168
:10200000002007B0BDE8F08FBBFBF7F807FB08F82E
:10201000ABEB08035A19B2FBF7F107FB112002934F
:1020200008B101FB0772B2FBF7F30393002301939E
:10203000A7EB0B03DFF8A4A00493029BC1462E4636
:1020400003EB0A0B039B019A9342D9D023493A46EA
:10205000484614F0D1F9019BF3B9049B03EB080245
:10206000AA4211D2214658460592F7F733FB059A4A
:10207000029B1444DA1B16443946484614F0C4F94E
:10208000E8B16FF00600BCE721462A465846F7F74C
:1020900021FB2C44761BEFE7019B5A1C039B9A42C1
:1020A00005D3324621465046F7F714FBE4E72146B4
:1020B0003A465046F7F70EFB3C44F61BDCE7484631
:1020C0003A46514614F076F9B9440028D9D1019B1B
:1020D00001330193B6E76FF0080092E790300020DB
:1020E00038B505460C4614F0B7F9AB070AD1B4FB76
:1020F000F0F300FB134040B921462846BDE83840C4
:1021000014F082B96FF0090038BD6FF00A00FBE7E8
:10211000F8F7D8BBF8F7FABBF8F726BCF8F7D6BC47
:10212000F8F714BDF8F79CBB2DE9F041304F0220C1
:1021300000F0B0F8D7E90026841A2E4A61EB0605B4
:10214000106800218D4208BF844203D26FF0050061
:10215000BDE8F08114F0D4FC8028F7D1FEF7EEFB47
:10216000254D0646002455F8043B03B19847013439
:10217000102CF8D1214DDFF88C80FFF767FE00F0BE
:10218000F3FA19F061FA00F081F800F08DFA00F02E
:1021900019FBFFF7C3FF00F07FF8EB68984798F84A
:1021A000004004BBAB68164D984700F077F8FFF786
:1021B000B7FF00F0DBFAFFF759FE00F009FB00F073
:1021C00075FA00F065F819F041FA55F8043B03B1CF
:1021D00098470134102CF8D1022000F05BF8C7E9D1
:1021E00000010020B4E72B6830469847D7E700BFCE
:1021F000904000208C030020E07D00207C03002024
:10220000A07D00209C7D0020014B00221A707047A9
:102210009C7D0020024A136801331360704700BFA1
:10222000247E0020024A13680BB1013B1360704703
:10223000247E002038B5114B1D680446D5B9FCF743
:1022400001F90F4B18700F4B01221A704CB129463F
:102250000D4814F005F914F027F92946204614F02A
:1022600013F9FCF7D9F8FFF75FFF0446FCF7E4F831
:10227000204638BD6FF00704FAE700BF247E002037
:10228000287E00209C7D00200922010814F026BA37
:1022900014F080BAF8F7C8BCF8F7D8BCF8F7D7BC88
:1022A0002DE9F04702289DF820909DF824A00446CF
:1022B0000E461746984613D80A4D55F820300BB1F4
:1022C0005B689847084B45F82430CDE9089A1D68AB
:1022D0003A46434631462046AC46BDE8F0476047A3
:1022E000BDE8F087984000209803002002282DE9DF
:1022F000F04104460D46164610D8FEF783FB88B918
:102300000B4B53F8243083B19F680A4B3246294661
:102310002046BC461B68BDE8F04160476FF00200F4
:10232000BDE8F0816FF00700FAE74FF0FF30F7E704
:1023300098400020B80300200EB430B50446ADF537
:10234000027DFEF7A3FA022C1FD82046FEF75AFBA7
:10235000F0B9124D55F82430EBB186AA8599019257
:1023600002A81BF06FF902A8F3F70AFF55F8243012
:102370009D680B4B02461B6802A92046A8470DF535
:10238000027DBDE8304003B070476FF00200F6E711
:102390006FF00700F3E74FF0FF30F0E798400020C0
:1023A000B80300200FB42DE9F047ADF5027D8AAFE8
:1023B000002457F8049B174EDFF85CA025465FFA0F
:1023C00084F84046FEF762FAB8B94046FEF71AFBB9
:1023D00098B933688BB13A46494602A801971BF079
:1023E00031F902A8F3F7CCFE336802469D68DAF8AB
:1023F000003002A94046A84705460134032C06F1E7
:102400000406DCD128460DF5027DBDE8F04704B096
:10241000704700BF98400020B8030020022810B485
:1024200009D8084C54F820304BB1DC68064BA44660
:102430001B6810BC60476FF0020010BC70474FF083
:10244000FF30FAE798400020B8030020022805D8A2
:10245000054A52F8203023B11B6918476FF002007B
:1024600070474FF0FF30704798400020022807D88F
:10247000044A52F820301BB1034A5B6911681847BF
:10248000704700BF98400020B80300202DE9F843B2
:10249000DFF83880DFF838900B4E0025EFB2384671
:1024A000FEF7B0FA044650B901213846FEF7B2FAF9
:1024B000C8F80040C9F800403460746034720135D7
:1024C000032DEBD1BDE8F883B0400020AC400020E4
:1024D000A840002038B50024E5B22846FEF792FA5D
:1024E000012803D100212846FEF794FA0134032C79
:1024F000F2D138BD2DE9F04F87B004468DF80710B2
:1025000003A80921FEF7D8F99DF80730374D0D2BA8
:10251000074629D019D8082B19D00A2B24D02A68AD
:10252000082A0ED8511C296031498B54314B53F87D
:1025300024309D68304B01221B680DF107012046B5
:10254000A8472E4A136801330CE07F2BE7D12B6894
:10255000002B40D0013B264A2B600021D154274A52
:102560001368013B136036E0244E336863B3DFF831
:102570008490DFF8848059F824302149D3F808A0EA
:10258000D8F8003002222046D0473268092AC246D5
:10259000CB4610D11B49164800921AF0BDFE009A96
:1025A00048B959F8243018499F68D8F800301522E6
:1025B0002046B84708E0BA4210D10D4803A91AF0E6
:1025C000DFFD58B9FFF786FF094A00232B6033600F
:1025D00013605360137207B0BDE8F08F5BF82430CE
:1025E0000A499F68DAF800301122E1E7AC40002088
:1025F000B040002098400020B8030020A8400020F0
:10260000AAED020811F102081BF1020830F10208DC
:10261000082901D9FEF750B96FF002007047082968
:1026200010B40BD803460C18A34202D110BCFEF71D
:1026300055B913F8012B203A5E2AF5D96FF0020044
:1026400010BC7047022801D8FEF7DCB900207047A3
:10265000022810B5044610D8FEF7D4F9012803D09B
:1026600000212046FEF7D6F9044A00231360044AED
:102670001360044A13605360137210BDAC40002015
:10268000A8400020B0400020022805D8054A52F892
:10269000203023B19B6918476FF0020070474FF05C
:1026A000FF30704798400020F8F72EBEF8F77CBE48
:1026B000F8B52A4E0546375C0C46FEF7E7F8324679
:1026C00000284AD04F2C705D3BD020D82B2C2ED028
:1026D00014D80A2C2DD00D2C14BF07230623204913
:1026E00001EBC001CB5C53550B2B36D1072F2AD100
:1026F00000235355BDE8F84018F0AABF422C1ED065
:102700004D2C18D0412C14BF07230023E7E76D2C74
:1027100011D008D8612C10D0622C10D0542C14BFCA
:1027200007230123DBE76F2C0BD0742CF7E7022380
:10273000D5E70623D3E70523D1E70023CFE703231B
:10274000CDE70423CBE70A2F07D1002353550548D3
:102750004560BDE8F84000F013B8F8BDA440002083
:1027600041F1020890030020F8F78ABAF8F78ABA14
:10277000024A8021082014F00BB900BFBC400020A1
:10278000014A082114F060B9ED7B000814F026B965
:10279000F8F794BAF8F7A4BAF8F7A7BAF8F7AABA0C
:1027A000F8F7AABA70477047014B1B68184700BF7B
:1027B000BC030020F8F750BBF8F776BBF8F796BBE0
:1027C000F8F7D6BA014B5B69184700BFCC0300206D
:1027D000014B9B69184700BFCC03002038B5104C53
:1027E000237805460BB9012038BD02F011F9227893
:1027F0004FF47A73B3FBF2F3B0FBF3F000F0D0FCCC
:1028000004460028EFD10F2DEDD8024629464FF09F
:10281000FF3000F071FC034B20461D60E4E700BF71
:10282000E8030020EC03002010B5032000F052FC68
:1028300002F0EEF8064B18600F20FFF7CFFF0446BA
:1028400018B912F0A3FF204610BD0124FBE700BF1A
:10285000C8040020034A044B11681B780B44136022
:10286000704700BF2C7E0020E8030020014B186851
:10287000704700BF2C7E002038B50446FFF7F6FFF6
:10288000631C1CBF054B1B78054618BFE418FFF7F7
:10289000EDFF431BA342FAD338BD00BFE80300207D
:1028A000024A136823F002031360704710E000E04F
:1028B000024A136843F002031360704710E000E01F
:1028C000014B1868704700BF9075FF1F014B1868D7
:1028D000704700BF9475FF1F014B1868704700BF19
:1028E0009875FF1F8068C0F3800070472DE9F341A1
:1028F000002301930446002800F00A81856D25B964
:10290000F7F73CFDE56584F8545020688368D900EA
:1029100040F1B3808368DA0000F1C680A36D43F014
:102920001003A365E36D43F00103E3650121FFF7A5
:10293000D9FFA36D03F010031843A36D40F0EA80A4
:1029400023F4817343F002032268A3659368DB07D5
:1029500000F1AC80D368A568666823F018032B43A8
:10296000D360E36C06F0404C4CEA030594F83C302D
:10297000012B09D1D4E910373B432B43A56C2B43E2
:1029800043EA0C0343F001051769644B3B402B43BA
:10299000136126F00043B3F1804F0AD0B6F1004F27
:1029A00007D05F4F3B6806F4701623F470131E4384
:1029B0003E60637E267EE768D4F830C094F82C80B1
:1029C000DB0343EA8633A67E3B43BCF1000F43EAB8
:1029D000463318BF4FF4805C276943EA480343EA53
:1029E0000C0394F820C0002FB4BF27F0004E4FF422
:1029F000001EBCF1010F43EA0E0E03D1002E57D189
:102A00004EF4803E666A2EB1A36A06F4E0761E4359
:102A10004EEA060ED66826F4FE3626F4F37646EA2B
:102A20000E06D660D2F810C03E4E0CEA06063543BC
:102A300015615569666B25F0070535435561556984
:102A4000A66B25F0700545EA06155561002F38D1B3
:102A5000906A60F00F009062D068334A024072457D
:102A60004CD10023E365A36D23F0030343F001037E
:102A7000A365084602B0BDE8F08183682B4A23F0C5
:102A8000104323F0170343F080538360284B1B68E7
:102A9000B3FBF2F301335B000193019B002B3FF486
:102AA00039AF019B013BF7E7002140E7054680E78E
:102AB000A66D46F02006A665E66D46F00106E665C1
:102AC000A0E7B7F5001FC7D1266E850026FA05F5E9
:102AD00005F00F050F2D0ED001300828F5D1906AB2
:102AE000E0690138800000F01C006FF00F0505FA66
:102AF00000F03043AFE70128AAD0F0E7A36D23F040
:102B0000120343F01003A365E36D43F00103E36593
:102B10000121AEE743F01003A365F9E702FCFF1FB4
:102B20000827014002FCFFDFE7FF3F83400D030061
:102B3000C8040020F8B54569082D04460E460AD0A1
:102B40000368DB68D90705D5836D43F020038365EF
:102B50000120F8BD0425FFF789FE074620680368B9
:102B60002B4222D0A36D43F40073A365C36813F412
:102B7000406F14D1A37E93B903681B070FD5FFF7ED
:102B8000B1FE38BB2268536823F00C035360A36D79
:102B900023F4807323F0010343F00103A365207E37
:102BA00008BB23680C221A60D3E7721CD7D0FFF74A
:102BB0005DFEC01BB04201D8002ECFD123681B6838
:102BC0002B40CBD1A26D84F8543042F00402A265B0
:102BD0000320BEE7A36D43F02003A365E36D43F03C
:102BE0000103E365DBE70020B3E70368186C704777
:102BF000F7B50023019390F85430012B044600F000
:102C0000BB80012380F854300068FFF76BFE00287A
:102C100040F0AC80486823690A68022823F0040366
:102C20007CD0B3F1004F2568C2F3110E13D1AB6A0B
:102C300043EA0E03AB628B68686903EA022323F060
:102C40007C4323F0FF0320EA02210B43002A6B613F
:102C500026DB002050E0236E00F01F074FF00F0C22
:102C60000CFA07FC6FEA0C0623EA0C0CBEF1000F0D
:102C700011D1C2F38463BB4043EA0C03236680088E
:102C8000E36901309842D6D8A86AC2F38363BB4097
:102C900006403343CEE792FAA2F3B3FA83F3EAE7AE
:102CA000364937480B68824203F0E07517D11B02A2
:102CB000CFD40B68334A23F0E0732B4343F4000373
:102CC0000B60314B1B68B3FBF2F20C2302FB0333A6
:102CD0000193019B002BBCD0019B013BF8E72B48E3
:102CE00082420ED113F08070B3D10B6823F0E073F1
:102CF0002B4343F080730B60002384F8543003B0FF
:102D0000F0BD23488242A4D113F48000A1D10B6806
:102D100023F0E0732B4343F48003ECE7B3F1004F5F
:102D200006D121688B6AC2F3110023EA00038B628B
:102D3000002A8EDA1248114982420B6807D10A68CC
:102D400003F0A07322F0E07213430B6081E70F4899
:102D5000824203D10A6803F44003F3E70C4882423D
:102D60007FF477AF0A6803F0C073EBE7A26D42F01F
:102D70002002A2651846BFE70220C0E708270140ED
:102D8000001000B0400D0300C8040020004000B84F
:102D9000002000B438B504460068FFF7A3FD08B969
:102DA000002038BD22689368990707D4936823F000
:102DB000004323F0170343F010039360FFF756FD21
:102DC000054623689B685B07EAD5FFF74FFD401B6C
:102DD0000228F6D923689B685A07F2D5A36D43F001
:102DE0001003A365E36D43F00103E3650120D8E719
:102DF00073B50023026801939368DD07044602D58A
:102E0000002002B070BD9168214B194209D0A36D1A
:102E100043F01003A365E36D43F00103E365012074
:102E2000EFE7936823F0004323F0170343F0010317
:102E30009360184B1B6818021CD4637E012BDFD0F3
:102E4000FFF714FD144E054622681368DB07D7D43C
:102E50009368D9075FBF9368334043F001039360E1
:102E6000FFF704FD401B0228EED923681B68DA0730
:102E7000EAD4CCE7094B0A4A1B68B3FBF2F30133EF
:102E80000193019B002BD8D0019B013BF8E700BFC9
:102E90001700008008270140E8FFFF7FC8040020DA
:102EA000400D030038B504460068FFF71BFD0546DA
:102EB00020BB94F85430012B20D0012384F85430E7
:102EC0002046FFF795FFB0B9A36D226823F4706325
:102ED00023F0010343F48073A3651C23E0651360B2
:102EE00084F85400936823F0004323F0170343F061
:102EF0000403936038BD84F85450FBE70220F9E7DF
:102F0000026838B5936891680446C80701D4002068
:102F100038BD9907FBD4936803F00503012B19D141
:102F2000936823F0004323F0170343F002039360F8
:102F300003231360FFF79AFC054623689B68DB07B1
:102F4000E5D5FFF793FC401B0228F6D923689B6860
:102F5000DA07F2D5A36D43F01003A365E36D43F0E8
:102F60000103E3650120D3E770B50446002841D092
:102F7000836D43F002038365FFF70CFF054668B9D4
:102F80002046FFF7BDFF054608B90123A365226867
:102F9000936823F0104323F01703936023685A6863
:102FA00022F4677222F003025A6040F29F321A60E4
:102FB000D968114A0A40DA601A6922F040421A615F
:102FC0005A6922F007025A611A6A02F0F0221A6264
:102FD0009A6A0A4A00269E62136823F0FE73136001
:102FE0002046F7F797FAE6652666A66584F85460EA
:102FF000284670BD0125FBE700023E8308270140FB
:1030000010B590F85430012B044615D0012380F8F8
:103010005430FFF7BFFE58B92046FFF771FF38B9AB
:10302000A36D23F4807323F0010343F00103A36530
:10303000002384F8543010BD0220FCE713B50023B0
:10304000019390F85430012B044640D0012380F8BE
:103050005430FFF755FF23689A68D20733D4A26D26
:1030600022F4817242F00202A265D968DA6822F085
:103070000302DA609A6842F0004201F003019A60AC
:103080009A68002A12DA019A01320192019AB2F585
:103090002E3FF5D3A36D23F0120343F01003A36575
:1030A000002384F85430012002B010BDDA680A43CE
:1030B000DA60A36D23F0030343F00103A36500234B
:1030C00084F85430F0E7A36D43F01003F6E70220D4
:1030D000EAE700000749CA6822F4E062030212042A
:1030E00003F4E063120C134343F0BF6343F4003373
:1030F000CB60704700ED00E0164B30B5DC68C4F3E0
:103100000224C4F10703251D042B28BF0423062D28
:103110004FF0FF3505FA03F38CBF033C002421EA8E
:103120000303A34005FA04F422EA0402002843EA58
:103130000203ACBF00F16040074A4FEA0313B8BF77
:1031400000F00F00DBB2AABF00F56140135480F815
:10315000003330BD00ED00E014ED00E0002808DB96
:103160000123420900F01F0003FA00F0014B43F86D
:103170002200704700E100E000280DDB4309012236
:1031800000F01F0002FA00F02033044A42F8230046
:10319000BFF34F8FBFF36F8F704700BF00E100E0B8
:1031A0000138B0F1807F0AD2064B074A5860F021FF
:1031B00082F823100020072298601A6070470120CF
:1031C000704700BF10E000E000ED00E0002809DBE0
:1031D0004309012200F01F0002FA00F06033024AA6
:1031E00042F82300704700BF00E100E0C368A3B1CC
:1031F000A1B1B1F5802F10D102681968D163596867
:10320000916399685163D96811631969D1615969EA
:10321000916199695161DB691361704702681968AE
:10322000D1615968916199685161DB68F4E770B5C3
:1032300006460C46FFF71AFB054632685368DB0763
:1032400001D5002070BD611CF8D0FFF70FFB401BBB
:10325000A04201D8002CF0D10120F3E72DE9F04184
:10326000794E04460F460FCE8CB06D460FC50FCE7B
:103270000FC596E80F0085E80F00A36AE56903B95A
:10328000AD0023681A68002D00F0CD8022F4C04202
:1032900042F400521A601A6815F00F0642F001025B
:1032A0001A601FD04FEA15184FEA88080026B0456B
:1032B00023685ED8C5F3810200218A4240F08B80EA
:1032C00015F0030540F09380013104299D60FBD186
:1032D00039462046FFF7ABFF2368002800F09E80A8
:1032E0001A6833E0AD08B54203D800200CB0BDE841
:1032F000F081A38FA16922689BB2204651F8233048
:103300009360A38F01339BB2A387A38F9BB251F825
:1033100023309360A38F01339BB2A387A38F9BB20B
:1033200051F823309360A38F01339BB2A387A38FFF
:103330009BB251F823309360A38F01339BB2A387D4
:103340003946FFF774FF23681A6868B122F001025A
:103350001A60636D43F0100363650120002384F855
:10336000510084F85030C1E742F080021A60043600
:10337000B9E7A28FA16992B2204651F822209A6043
:10338000A28F013292B2A287A28F92B251F822206C
:103390009A60A28F013292B2A287A28F92B251F8A4
:1033A00022209A60A28F013292B2A287A28F92B29B
:1033B00051F822209A60A38F01339BB2A38739462C
:1033C000FFF735FF23681A680028BFD142F080025A
:1033D0001A6004366BE7A08FA66980B2013156F8F7
:1033E00020009860A08F013080B2A08765E7A18F90
:1033F000A06989B2013250F82110606805EB4005E0
:103400000CA800EB850555F8300C014099600021AF
:10341000042A3FF45DAF99600132F9E71A6842F07F
:1034200080021A6062E7616822F006020A431A60AD
:103430001A6822F4C04242F400521A601A6842F03C
:1034400001021A60284651E780DA020810B50446E6
:10345000E8B190F8513003F0FF021BB980F850201A
:1034600012F048FCD4E9013021680A68034360691E
:1034700022F4A022034322F0660213430B600020D3
:1034800001236065A06584F85130636410BD01209C
:10349000FCE738B50546012480B102684464002485
:1034A000C487A0F840408487136823F001031360A9
:1034B00012F040FC85F8514085F85040204638BD58
:1034C000704770477047C38F026830B59BB2456B39
:1034D00055F823309360C38F01339BB2C387C38FEA
:1034E0009BB285B055F823309360C38F01339BB2F4
:1034F000C387C38F9BB2044655F823309360C38FB4
:1035000001339BB2C387C38F9BB255F823309360BE
:10351000C38F01339BB2C387FFF789FE88B122684E
:10352000136823F001031360636D43F010036365B8
:10353000012384F85130002384F850302046FFF7EF
:10354000C1FF23681A6842F080021A60DA680092AC
:10355000DA680192DA68DB680393B4F842300292C9
:1035600003339B080021B4F8402092B29A4201D262
:10357000042901D105B030BDB4F84020A06B5DF83E
:10358000215092B2013140F82250B4F8402001326B
:1035900092B2A4F84020E6E7F0B5C36AB0F8425012
:1035A000012B85B004460E461FD1826D012A1BD126
:1035B000C36D2B44C365B4F84230AD08180718BF7B
:1035C00025F00305FFF752F90746E28FB4F84030C3
:1035D00092B295429BB201D99D4249D8B4F842308B
:1035E0001A0762D1002027E083652268A168E5659B
:1035F0000027A787136823F4C04313602046FFF712
:10360000F5FD226A23681168D96251689962916850
:103610005962D2681A621A6842F001021A60314691
:10362000FFF705FE50B1636D84F8507043F010034E
:103630000120636584F8510005B0F0BD226813686D
:1036400043F08003136031462046FFF707FE002851
:1036500040F08680226802236364136823F4C04329
:1036600043F480431360136823F470031360A2E7EC
:1036700031462046FFF727FF711CA6D0FFF7F6F86A
:10368000C01BB04201D8002E9FD12268136823F0DE
:1036900001031360636D43F0100363650120002391
:1036A00084F8510084F85030C6E72168086800F0BB
:1036B0001800102808BF08684FEA131202F101022F
:1036C00008BF20F470004FEA021703F11005C3EBA6
:1036D000021208BF40EA0250A5EB070508BF0860C8
:1036E000AD08930718BF01350022AA4229D12B4605
:1036F0000022032B31D931462046FFF798FD0028E0
:10370000C8D123681A6842F080021A60DA68009211
:10371000DA680192DA68DB6802920393A8423FF408
:1037200061AFB4F84030A26B5DF820109BB201305D
:1037300042F82310B4F8403001339BB2A4F8403073
:10374000ECE7E38F606B9BB2013250F823308B6063
:10375000E38F01339BB2E387C7E78A600133C8E791
:10376000012069E7F0B5C36AB0F84250012B85B07B
:1037700004460E461FD1826D012A1BD1C36D2B4416
:10378000C365B4F84230AD08180718BF25F003052B
:10379000FFF76CF80746E28FB4F8403092B29542DA
:1037A0009BB201D99D4249D8B4F842301A0762D180
:1037B000002027E083652268A168E5650027A787C8
:1037C000136823F4C04313602046FFF70FFD2269FE
:1037D00023681168D9625168996291685962D26808
:1037E0001A621A6842F001021A603146FFF71FFDA3
:1037F00050B1636D84F8507043F01003012063658D
:1038000084F8510005B0F0BD2268136843F08003CE
:10381000136031462046FFF721FD002840F08E80DE
:10382000226802236364136823F4C04343F4804393
:103830001360136823F470031360A2E73146204637
:10384000FFF741FE711CA6D0FFF710F8C01BB04275
:1038500001D8002E9FD12268136823F00103136062
:10386000636D43F0100363650120002384F8510069
:1038700084F85030C6E72168086810F0180F08BFB8
:1038800008684FEA131202F1010208BF20F4700029
:103890004FEA021703F11005C3EB021208BF40EA1A
:1038A0000250A5EB070508BF0860AD08930718BFD5
:1038B00001350022AA4232D12B460022032B3AD9ED
:1038C00031462046FFF7B3FC40B1012384F8513064
:1038D000002384F850302046FFF7F4FD23681A686F
:1038E00042F080021A60DA680092DA680192DA68BF
:1038F000DB68029203930022AA423FF459AFB4F866
:103900004030A16B5DF822009BB2013241F82300E8
:10391000B4F8403001339BB2A4F84030ECE7E38FB9
:10392000606B9BB2013250F823308B60E38F013320
:103930009BB2E387BEE78A600133BFE7012061E7FE
:10394000F8B590F85160069D012E0446F0B278D18A
:1039500094F850700226012F84F8516077D0C4E9A2
:103960000D13636A84F850000026E687A4F84060CF
:103970000BB9920092B22368A4F842201A6822F090
:1039800018021A601A68334B1340602B52D009D8C2
:10399000402B0FD0304B134063B1636D43F02003D5
:1039A0006365F8BDB3F5803FF7D129462046FFF7A0
:1039B000F3FD43E0E36A012B03D1A26D012A10D08D
:1039C000A365A1682046FFF711FC63694BB122692A
:1039D00023681168D9625168996291685962D26806
:1039E0001A62226802236364136843F001031360C0
:1039F000E28FB4F84210B4F8403092B2B2EB910FBB
:103A00009BB24FEA910001D298420ED82268136807
:103A100023F001031360012384F8513001230020B7
:103A200084F8513084F85000BBE729462046FFF760
:103A30004AFDDDE729462046FFF794FE0028B0D175
:103A4000ECE7636D43F0080363650120A9E73046A6
:103A5000A7E700BF6000010040000100F8B5044680
:103A600090F85100069E0128C5B240F0BA8094F843
:103A700050700220012F84F8510000F0B880C4E992
:103A80000D13636A84F850500020E087A4F84000CA
:103A90000BB9920092B22368A4F842201A6822F06F
:103AA000180242F010021A601968524A0A40602A4D
:103AB00000F08F8009D8402A0FD04F4A0A4062B1E7
:103AC000636D43F02003636536E0B2F5803FF7D1C4
:103AD00031462046FFF760FD7FE0E26A012A03D10C
:103AE000A16D01293FD0A2656269A168402A67D013
:103AF00094F83070002F5AD11A6822F0180242F060
:103B000008021A602046FFF771FB2268136843F031
:103B1000010313603146FFF78AFB23681A6868B116
:103B200022F001021A60636D84F8507043F01003B4
:103B30006365012384F851302846F8BD42F08002C5
:103B40001A601A6822F0180242F010021A606369C3
:103B50004BB1226923681168D962516899629168F2
:103B60005962D2681A62226802236364136843F0C0
:103B700001031360E28FB4F84210B4F8403092B2FF
:103B8000B2EB910F9BB24FEA910001D298421BD841
:103B90002268136823F001031360012384F8513075
:103BA0000123002584F8513084F85050C4E72046A2
:103BB000FFF71CFB2268136843F018031360C6E785
:103BC0002046FFF713FBC2E731462046FFF77BFC98
:103BD000D0E731462046FFF7C5FD05460028ABD1AA
:103BE000DEE7636D43F0080363650125A4E705463E
:103BF000A2E700BF6000010040000100F0B50568C9
:103C00002B6859058DB004460DD56B685A0742BF25
:103C1000436D43F0010343656B689B0742BF436DEF
:103C200043F0020343656B68DF0740F1ED802B68CA
:103C30009E0540F1E9802B68D4F814C043F080035E
:103C4000BCF1600F2B6003D0BCF5803F40F0DC81FD
:103C50002A6812F4005200F01381A44F0FCF6E4671
:103C60000FC60FCF0FC697E80F0086E80F00A26AB5
:103C7000E36902B99B00A28F92B2B3EB820F00F20C
:103C80008180022363642B68B4F8422023F4C0438C
:103C900043F480432B602B6823F470032B60BCF546
:103CA000803F01BFA38F01339BB2A3874AB92B6822
:103CB00023F4C0632B60012384F8513084F8502032
:103CC000A2E00F2A4FEA92032CD9E18F606B89B2F0
:103CD00050F82110A960E18F013189B2E187E18FAD
:103CE00089B250F82110A960E18F013189B2E187D2
:103CF000E18F89B250F82110A960E18F013189B2BA
:103D0000E187E18F89B250F82110A960E18F01317C
:103D100089B2E187E18F89B2994275D112F00F0F14
:103D200072D117E0296811F01801C2F1100215D103
:103D3000BCF1600F01BF296821F4700141EA025112
:103D40002960900718BF0133002199420BD100224E
:103D5000042B14D12046FFF7B3FB55E01029F0D116
:103D6000BCF5803FE6E7E28F606B92B2013150F81C
:103D70002220AA60E28F013292B2E287E5E7AA60D0
:103D80000133E5E7A18F89B2C1EB930103294FEA23
:103D9000930254D994F86030012B10D12B68002283
:103DA00043F080032B6084F860202B6823F4C06309
:103DB0002B60032384F85130042363647EE7A38FD0
:103DC000A2699BB252F82330AB60A38F01339BB240
:103DD000A387A38F9BB252F82330AB60A38F01332C
:103DE0009BB2A387A38F9BB252F82330AB60A38F03
:103DF00001339BB2A387A38F9BB252F82330AB60F1
:103E0000A38F01339BB2A3870DB0F0BDA18FA6692C
:103E100089B2013056F82110A960A18F013189B211
:103E2000A1879042F2D313F003030CD1AB60A18FB2
:103E30000132013189B2042AA187F7D1E4E70020D9
:103E400002F00302EDE7A18FA06989B250F82110BA
:103E5000606803EB40030CA800EB830353F8303C8D
:103E60000B40AB60A38F01339BB2A38700210132CB
:103E7000042AC9D0A960A38F01339BB2A387F6E7B8
:103E8000EB680093EB680193EB680293EB68039394
:103E9000B4F84230DE1CB6081046B4F8401089B2BF
:103EA000B14201D2042823D1E08FB4F84060B6B209
:103EB000B6EB930F80B24FEA93012AD3B3EB800F96
:103EC00027D86369B3F5803F02D1A36D012B03D0DE
:103ED0002B6823F4C0632B60012384F85130002346
:103EE00084F850302046FFF7ECFA8DE780DA0208BC
:103EF000B4F840C0A16B5DF820701FFA8CFC013053
:103F000041F82C70B4F84010013189B2A4F8401087
:103F1000C3E7E08F80B2081A032840D994F86020E4
:103F2000012A0FD12B68002243F080032B6084F814
:103F300060202B6823F4C0632B60032384F8513086
:103F400005233AE7E28F606B92B250F82220AA6014
:103F5000E28F013292B2E287E28F92B250F82220D1
:103F6000AA60E28F013292B2E287E28F92B250F8F9
:103F70002220AA60E28F013292B2E287E28F92B2EF
:103F800050F82220AA60E28F013292B2E287E28FDB
:103F900092B291427FF438AF13F00F0FC0E6286859
:103FA0001909013110F018004FEA0116C3EB011195
:103FB00018D16069602801BF286820F4700040EAC9
:103FC0000150286010339B1B89074FEA930300D0F0
:103FD00001339A420CD10022032B3FF6BBAEAA60FC
:103FE0000133F9E71028EDD16069B0F5803FE2E7D1
:103FF000E18F606B89B2013250F82110A960E18F26
:10400000013189B2E187E4E794F85130022B64D1A1
:10401000EB68B4F842100093EB680193EB680293ED
:10402000C81CEB68039380080022B4F840309BB2B0
:104030008342B4F840309BB201D2042A10D1B3EBD2
:10404000910F4FEA910218D12B6823F4C0632B60C3
:10405000012384F851302B6823F001032B603EE7E5
:10406000A66B5DF8227046F82370B4F84030013337
:104070009BB2A4F840300132D7E794F86030012BAE
:104080003FF450AFE38F616B9BB251F82330AB60CC
:10409000E38F01339BB2E387E38F9BB251F8233068
:1040A000AB60E38F01339BB2E387E38F9BB251F8A0
:1040B0002330AB60E38F01339BB2E387E38F9BB286
:1040C00051F82330AB60E38F01339BB2E387E38F7A
:1040D0009BB29A427FF498AE3CE6636D43F00803CE
:1040E00063652046FFF7EEF98EE600BF70B5D0E9B4
:1040F00013456560446D14B1D0E916456560D0E99B
:10410000105404F01C060124B4406C600468636021
:104110008368102B0BBFA260A160E160E26070BDFC
:104120000268416CD3B210B5083B1424B3FBF4F31E
:104130000B4CA24288BF0B4A21F0030199BF01F149
:10414000804202F50232521807338264064AC26482
:1041500003F01F03012202FA03F3036510BD00BF41
:10416000070402401C0802408008024010B50028E5
:1041700060D00268304B9A424FF014044DD82F495A
:104180001144B1FBF4F189004164A3F207430364D5
:10419000022380F82530136823F4FF4323F07003D3
:1041A0001360D0E90234234304691168234344694E
:1041B000234384692343C4692343046A23430B4391
:1041C0001360FFF7ADFF8368816CB3F5804F04BFC8
:1041D00000234360426802F07F030B60D0E91314B0
:1041E000013A032A4C6020D8154A164C84651A44BB
:1041F000013B9200012103F0030301FA03F30021C4
:104200004265C3651160636000230122C36380F8C7
:10421000243080F82520184610BD0B4B1344B3FB07
:10422000F4F39B004364094BB1E70023C0E9153365
:10423000C365E9E70120EFE707040240F8FFFDBF8F
:104240003F82001040090240F8FBFDBF000402401D
:1042500038B5002845D001680B6823F001030B60D6
:10426000214B99424FF0140433D8204A0A44B2FB40
:10427000F4F292004264A3F207430364D0E91023EE
:10428000012403F01C0304FA03F300250D605360BE
:10429000FFF746FF836C41681D60D0E913325A6016
:1042A0004A1E032A06D8124B0B449B0094401D6003
:1042B000104B5C600023C363C0E91533C0E90B33C6
:1042C000C0E90D33C36580F8253080F824301846E6
:1042D00038BD094B0B44B3FBF4F39B004364074B1D
:1042E000CBE70120F4E700BF07040240F8FFFDBF61
:1042F0003F82001040090240F8FBFDBF000402406D
:1043000070B590F82450012D04463CD090F82560FB
:104310000125AE4280F824504FF000062DD1022531
:1043200080F82550C6630668356825F001053560BC
:10433000FFF7DCFE026B0368BAB11A6842F00E02A6
:104340001A60A26C1168C90342BF116841F4807100
:104350001160626D1AB1116841F4807111601A68C0
:1043600042F001021A60002070BD1A6822F00402B7
:104370001A601A6842F00A02E2E78023C36380F8F9
:1043800024602846F0E70220EEE740B190F825309F
:10439000022B06D00423C363002380F824300120BD
:1043A00070470368816C1A6822F00E021A600A686E
:1043B00022F480720A601A6822F001021A60D0E9C1
:1043C000101303F01C02012393404B60D0E9133219
:1043D0005A60436D33B11A6822F480721A60D0E9D2
:1043E00016325A60012380F82530002380F82430EB
:1043F0001846704710B590F82530022B03D00423DF
:10440000C363012010BD03681A6822F00E021A600F
:104410001A6822F001021A60826C136823F4807318
:104420001360D0E9101303F01C02012393404B608A
:10443000D0E913325A60436D33B11A6822F48072A6
:104440001A60D0E916325A60012380F82530836B58
:10445000002480F8244013B198472046D2E718463C
:10446000D0E7000070B4426C046C036826681D68D5
:1044700002F01C020421914031420FD015F0040FCC
:104480000CD01A6892065EBF1A6822F004021A6005
:10449000036B6160002B33D070BC18470221914040
:1044A000314217D015F0020F14D01A68940606D4C2
:1044B0001A6822F00A021A60012280F82520114AA7
:1044C00093428CBF104B114B5960002380F824306D
:1044D000C36ADFE708219140314211D029070FD587
:1044E000196821F00E011960012303FA02F26260DB
:1044F000C36380F82530002380F82430436BC9E77C
:1045000070BC70478000024000040240000002407E
:1045100090F825007047C06B704700002DE9F04F00
:10452000524C00234FF00F090A6832FA03F501D10B
:10453000BDE8F08F012505FA03F818EA020200F041
:104540008F804E68032706F003054FEA430E07FAF3
:104550000EFC6F1E012F6FEA0C0C32D8876807EA39
:104560000C0ACF6807FA0EF747EA0A078760476820
:1045700027EA0808C6F300179F4047EA0807476084
:10458000C76807EA0C088F6807FA0EF747EA0807BA
:10459000022DC76017D14FEAD30800EB880803F05B
:1045A000070AD8F820704FEA8A0A09FA0AFB27EAB4
:1045B0000B0B0F6907FA0AF747EA0B07C8F82070D8
:1045C00001E0032DDCD1076807EA0C0C05FA0EF7B1
:1045D00047EA0C0716F4403F076041D023F0030779
:1045E00007F1804707F5803703F0030CBD684FEAF9
:1045F0008C0C4FF0070E0EFA0CFEB0F1904F25EA2E
:104600000E0E2FD01A4DA8422ED005F58065A84277
:104610000CBF0225072505FA0CF545EA0E05BD601D
:10462000D4F88050D74316F4803F0CBF3D4015436B
:10463000C4F88050D4F8845016F4003F0CBF3D40BD
:104640001543C4F88450256816F4801F0CBF3D4004
:10465000154325606568B60254BF3D40154365604B
:10466000013361E70025D6E70125D4E700080058AB
:1046700000040048374A2DE9F04F00234FF0010AAB
:104680004FF0070B4FF00F0931FA03F401D1BDE8E9
:10469000F08F0AFA03FC1CEA010654D023F003044D
:1046A00004F1804404F5803403F00307A568BF00DB
:1046B0000BFA07F8B0F1904F08EA050E45D0264DE9
:1046C000A84244D005F58065A8420CBF0225072505
:1046D000BD40754517D1D2F8805025EA0605C2F8CD
:1046E0008050D2F8845025EA0605C2F88450156837
:1046F00025EA06051560556825EA06065660A56890
:1047000025EA0805A560056803265C0006FA04F49E
:1047100023FA06F6254300EB8606056003F007053D
:10472000376AAD0009FA05F527EA0505356285689F
:1047300025EA04058560456825EA0C054560C568DD
:1047400025EA0404C46001339EE70025C0E7012583
:10475000BEE700BF00080058000400480369194282
:1047600014BF0120002070470AB181617047816247
:1047700070470000044AD168014208B502D0D060F9
:10478000F6F776F808BD00BF00080058024A136823
:1047900043F480731360704700040058024B18689C
:1047A00000F4C060704700BF000400580B4A136853
:1047B00023F0070343F001031360094B1A69012832
:1047C00042F004021A6105D130BF1A6922F00402D6
:1047D0001A61704740BF20BF20BFF6E700040058B1
:1047E00000ED00E00B4A136823F0070343F00203D7
:1047F0001360094B1A69012842F004021A6105D1BD
:1048000030BF1A6922F004021A61704740BF20BF0E
:1048100020BFF6E70004005800ED00E04FF0B04381
:104820001868C0F3404070474FF0B0431868C0F3B9
:10483000802070474FF0B0431868C0F340007047C5
:104840004FF0B042536823F47F4343EA00235360A0
:1048500070474FF0B0431868C0F3406070470000E5
:104860007FB54FF0B0432C4AD3F80831C0F30310A2
:1048700003F00F0352F82040284A52F82330B4FBCB
:10488000F3F4FFF78BFF264B054693E80700B5F5D9
:10489000007F04AB03E9070010D0224B9C4218D3E1
:1048A00003F5B70303F67F539C4229D903F574132C
:1048B00003F510639C4225D802230BE01A4B9C425F
:1048C00007D91A4B9C421BD903F5370303F5D8537C
:1048D000F0E7002304AA02EB830353F80C4C144DB9
:1048E0002B6823F0070323432B60FDF7BFFF064629
:1048F0002B6803F007039C4206D1002004B070BD72
:104900000123E7E70024EAE7FDF7B0FF801B022858
:10491000EED90320F2E700BF6CF702080CF702089B
:10492000B0DA0208C0CF6A00BFEA21013F93340227
:10493000004000584FF0B04310B59A68D96812F0A3
:104940000C0205D00C2A4AD101F00303012B50D1EF
:104950004FF0B0412B480B6813F0080306D00B68EA
:1049600013F0080337D1D1F8941007E00C6824073E
:1049700056BFD1F894300968C3F3032350F82330AD
:10498000002A0CBF184600204FF0B0418A6802F0A0
:104990000C020C2A1ED1CA6802F00302022A2ED091
:1049A000032A06D10B68184813F4801F174B18BF51
:1049B00003464FF0B040C168C268C068C1F3062129
:1049C000C2F30212400F4B4301320130B3FBF2F34A
:1049D000B3FBF0F010BD0B68C3F30313CEE7042A5A
:1049E0000AD0082A05D11B6813F4801304D10748A4
:1049F000CAE700231846C7E703480023C4E7024B71
:104A0000D7E700BF6CF702080024F4000048E80173
:104A100008B5FFF78FFF4FF0B043044A9B68C3F31C
:104A2000031352F82330B0FBF3F008BD0CF7020873
:104A30002DE9F0410446002855D04FF0B0439E6860
:104A4000DD680368990606F00C0605F003056BD5D2
:104A50001EB10C2E49D1012D47D1FFF7EBFE10B14D
:104A6000236A002B3FD04FF0B043A06A1A681207A8
:104A700056BFD3F894301B681B0903F0F00398422B
:104A80001ED9FFF7EDFE00282DD14FF0B04213687C
:104A900043F0080313601368A16A23F0F0030B438B
:104AA0001360606AFFF7CCFEFFF7B2FFAC4B1860F3
:104AB000AC4B1868FDF792FE002835D0BDE8F081B8
:104AC0004FF0B042136843F008031360136823F0FB
:104AD000F00303431360606AFFF7B2FEA06AFFF7BA
:104AE000BFFE0028E0D00120E8E7226A4FF0B04383
:104AF000002A54D01A6842F001021A60FDF7B6FE8F
:104B00000746FFF797FE002842D04FF0B0421368E7
:104B100043F0080313601368A16A23F0F0030B430A
:104B20001360606AFFF78CFE2368DB0748D42368B4
:104B30009F0700F1908023681D0740F1FC80A36966
:104B40004FF0B045002B00F0E380D5F89430E169D8
:104B500003F01002914200F0C68003F00302022A23
:104B6000C1D0D80740F1B580D5F8943023F00103C7
:104B7000C5F89430FDF77AFE0746D5F894309907CA
:104B800040F1A780FDF772FEC31B112BF5D904E09D
:104B9000FDF76CFEC01B0228B3D903208EE71A680C
:104BA00022F001021A60FDF761FE0746FFF742FEA0
:104BB0000028B9D0FDF75AFEC01B0228F6D9ECE751
:104BC000082E03D00C2E09D1032D07D1FFF726FEA6
:104BD0000028ACD06368002BA9D184E74FF0B04324
:104BE000A1681A6822F480120A431A606268B2F55A
:104BF000803F10D11A6842F480321A60FDF736FE09
:104C00000746FFF70BFE002891D1FDF72FFEC01BD2
:104C10006428F6D9C1E7B2F5041F04D11A6842F43A
:104C200000121A60E6E7196821F4803119601968EA
:104C300021F400111960002AE0D1FDF717FE0746A4
:104C4000FFF7ECFD00283FF472AFFDF70FFEC01B2D
:104C50006428F5D9A1E7042E03D00C2E12D1022D21
:104C600010D1FFF7E1FD18B12369002B3FF43BAFF2
:104C70004FF0B0426169536823F0FE4343EA016399
:104C8000536058E722694FF0B04382B11A6842F48A
:104C900080721A60FDF7EAFD0546FFF7C5FD0028A2
:104CA000E6D1FDF7E3FD401B0228F6D975E71A6847
:104CB00022F480721A60FDF7D9FD0546FFF7B4FDB6
:104CC00000283FF438AFFDF7D1FD401B0228F5D98D
:104CD00063E74FF0B042E169D2F8943023F010035B
:104CE0000B43C2F894304FF0B045D5F8943043F000
:104CF0000103C5F89430FDF7B9FD0746D5F89430A7
:104D00009A0718D4FDF7B2FDC31B112BF6D944E75F
:104D1000D5F8943023F00103C5F89430FDF7A6FDD3
:104D20000746D5F894309B0705D5FDF79FFDC31BBB
:104D3000112BF6D931E72368580753D50A4D2B6854
:104D4000D90513D4FFF722FDFDF790FD07462B6828
:104D5000DA050BD4FDF78AFDC31B022BF7D91CE73C
:104D6000C8040020EC03002000040058E3684FF062
:104D7000B045002B58D023F08003052B02BFD5F897
:104D8000903043F00403C5F890304FF0B045FDF784
:104D90006DFDD5F8903043F001030746C5F890301B
:104DA00041F28838D5F890309B0705D4FDF75EFDB9
:104DB000C31B4345F6D9F0E6E36823F00403812BD7
:104DC0001BD1FDF753FDD5F8903043F08003C5F8B3
:104DD000903007464FF0B04541F28838D5F8903012
:104DE000180504D5E06A00284AD1002066E6FDF7E0
:104DF0003DFDC01B4045F1D9CFE6FDF737FDD5F8A5
:104E0000903023F08003C5F8903007464FF0B0454E
:104E100041F28838D5F890301905E3D5FDF726FD25
:104E2000C01B4045F6D9B8E6FDF720FDD5F8903017
:104E300023F080030746C5F8903041F28838D5F852
:104E400090301A0516D4FDF711FDD5F8903023F0F7
:104E50000103C5F8903007464FF0B04841F288355D
:104E6000D8F890309B07BDD5FDF700FDC31BAB42C2
:104E7000F6D992E6FDF7FAFCC01B4045DFD98CE677
:104E80000C2E53D04FF0B04302281A6822F08072E3
:104E90001A6033D1FDF7EAFC0546FFF7DAFC38BBB0
:104EA000D4E90C314FF0B0420B43D0682F49014098
:104EB0000B43E16B0B43216C0B43616C0B43A16B08
:104EC00043EA0123D360136843F080731360D3680F
:104ED00043F08053D360FDF7C9FC0446FFF7B9FCEB
:104EE000002882D1FDF7C2FC001B0A28F6D954E63F
:104EF000FDF7BCFC401B0A28CFD94EE6DA6822F049
:104F00000302DA60DA6822F0885222F48032DA6032
:104F1000FDF7ACFC0446FFF79CFC00283FF465AFAE
:104F2000FDF7A4FC001B0A28F5D936E601283FF45A
:104F3000C5AD4FF0B043226BDB6803F00301914233
:104F40007FF4D1AD616B03F070028A427FF4CBAD88
:104F5000A16B03F4FE42B2EB012F7FF4C4AD626C8F
:104F600003F0604393423FF440AFBCE58C80C11135
:104F70002DE9F0410D46044610B90120BDE8F0814D
:104F8000674E336803F007038B4216D323689807F4
:104F900027D54FF0B046A268B36823F0F00313435F
:104FA000B360FDF763FC0746B368D90319D4FDF776
:104FB0005DFCC31B022BF7D911E0336823F0070314
:104FC0000B433360FDF752FC0746336803F00703D9
:104FD000AB42DBD0FDF74AFCC01B0228F5D9032009
:104FE000CCE723685A0617D54FF0B0466269D6F869
:104FF000083123F00F0343EA1213C6F80831FDF716
:1050000035FC0746D6F80831DB0305D4FDF72EFC46
:10501000C31B022BF6D9E2E723685E0713D54FF0D6
:10502000B046E268B36823F4E0631343B360FDF76E
:105030001DFC0746B368980305D4FDF717FCC31B96
:10504000022BF7D9CBE72368190714D54FF0B046E8
:105050002269B36823F4605343EAC203B360FDF7E7
:1050600005FC0746B3685A0305D4FDF7FFFBC31BD5
:10507000022BF7D9B3E72368DB070FD4284C23684A
:1050800003F00703AB4237D8FFF7C2FC254B18608B
:10509000254BBDE8F0411868FDF7A0BB6368022B03
:1050A0001ED1FFF7BBFB00283FF467AF4FF0B046BF
:1050B0006268B36823F003031343B360FDF7D6FBC4
:1050C00041F288380746B368626803F00C03B3EB1B
:1050D000820FD3D0FDF7CAFBC01B4045F3D97EE752
:1050E000032B02D1FFF7B5FBDDE713B9FFF7A2FBF6
:1050F000D9E7FFF799FBD6E7236823F007032B4393
:105100002360FDF7B3FB0646236803F00703AB42B9
:10511000BAD0FDF7ABFB801B0228F5D95FE700BFD3
:1051200000400058C8040020EC03002008B5FFF739
:105130006FFC4FF0B043044A9B68C3F3022352F85C
:105140002330D84008BD00BF4CF7020808B5FFF770
:105150005FFC4FF0B043044A9B68C3F3C22352F88C
:105160002330D84008BD00BF4CF7020830B590F896
:105170002C30012B4FF0020222D0194B80F82D2049
:10518000CA24012580F82C505C6253245C62B1F57E
:10519000807F046B16D19A6922F488529A615A6C06
:1051A00024F0010422F000425A640463DD650C4BD4
:1051B000FF225A620123002280F82D3080F82C2033
:1051C000104630BD996921F408519961D96C24F0D9
:1051D000020421F00041D9640463DA65E7E700BF07
:1051E0000028004070B50B4D036B6E6D1E40F2073A
:1051F000044603D50123EB65F2F75EFFB30704D540
:105200000223EB65204600F0C5F9012384F82D3018
:1052100070BD00BF0028004038B50A4CE36823F099
:105220002003E360FDF722FB0546E3689B0601D5FA
:10523000002038BDFDF71AFB401BB0F57A7FF4D98A
:105240000320F6E7002800402DE9F041114DEC68FD
:1052500014F0400407461AD1EB6843F08003EB607A
:10526000FDF704FB4FF003080646EB685B0601D42C
:10527000032C02D12046BDE8F081FDF7F7FA801B30
:10528000B0F57A7F84BF87F82D800324EDE70024F2
:10529000F0E700BF00280040104BDA6822F08002DF
:1052A00010B5DA609A699206044606D4FFF7B4FF97
:1052B00010B1032084F82D0010BD9A6922F020025D
:1052C0009A61FFF7A9FF10B1032084F82D00034A6B
:1052D000936943F020039361EEE700BF002800408C
:1052E00038B50446002847D090F82D3003F0FF026F
:1052F0001BB980F82C2010F0E3FB204D022384F82A
:105300002D30CA236B6253236B622046FFF79CFF4C
:1053100070BBAB6923F08E6323F04003AB6121695E
:105320006368AA690B431343A2691343AB61D4E9D1
:10533000022343EA02432B61D4E90931EA680B43B3
:1053400022F4F8521343EB602046FFF7A5FF78B92B
:10535000D4E90713AA690B4322F060421343626940
:105360001343AB61FF236B62012384F82D3038BDFA
:10537000024BFF225A62FAE70120F8E700280040BA
:105380000023092803D840EA0310C0B270470A3846
:105390000133C0B2F5E700002DE9F04790F82C305A
:1053A000012B05464FF0020067D0012385F82C3011
:1053B0004C4B85F82D00DE6806F44076B6F5807F0C
:1053C00076D04C69087891F8018091F802A091F8A4
:1053D0002470002A53D19A6912F0400208BFCA70A3
:1053E000FFF7CEFF81464046FFF7CAFF8046504692
:1053F000FFF7C6FF82463846FFF7C2FF0A6ACB783E
:10540000144344EA835444EA0A0343EA094343EA5F
:10541000082343EA0063334ACA2050625320506293
:105420008C6A8869B4F5807F946943D124F48854E8
:1054300094610124D465B6F5807F0ABFCB691364FB
:1054400018435064274B4A681A672A6B42F00102DE
:105450002A639A6942F488529A61234AD2F88030CA
:1054600043F40033C2F880301E4BFF225A62002002
:10547000012385F82D3085F82C00BDE8F087B4F1C4
:10548000803F07D0B4F5000F04D09A6912F04002B3
:1054900008BFCA700A6A144344EA0A0444EA004393
:1054A000C87843EA082343EA805343EA0763B2E734
:1054B0000023B0E724F4085494610224D465B6F5BF
:1054C000807F0ABFCB6993641843D064054B4A6858
:1054D0005A672A6B42F002022A639A6942F4085220
:1054E000BAE700BF002800400008005890F82C20C0
:1054F000012A03464FF0020012D00A4A83F82D0019
:10550000CA21516253215162916941F02001916198
:10551000FF2151620020012283F82D2083F82C0006
:10552000704700BF0028004090F82C20012A034655
:105530004FF0020019D00D4A83F82D00CA215162A4
:105540005321516291690A4841F080019161D0F87C
:10555000801041F48021C0F88010FF2151620020AA
:10556000012283F82D2083F82C007047002800408A
:1055700000080058064B5A6D520610B5044603D574
:105580004022DA65F2F79AFD012384F82D3010BD30
:10559000002800407047890001F1804101F5314148
:1055A0000A607047890001F1804101F531410868C6
:1055B000704700002DE9F74F994600238DF803301E
:1055C000044688461746FDF751F90C9D4D442D1AA7
:1055D000FDF74CF92C4BD4F800B01B6823265E4332
:1055E000360D6E43824601962268936803EA0803EB
:1055F000BB4201D100203AE0B8F5C06F07D137B9FE
:105600009BF80C30DBB28DF803309DF80330B9F114
:10561000FF3FEAD0FDF72AF9A0EB0A00A84229D300
:1056200023685A6822F0E0025A606268B2F5827F0D
:105630000AD1A268B2F5004F02D0B2F5806F03D153
:105640001A6822F040021A60A26AB2F5005F07D120
:105650001A6822F400521A601A6842F400521A6062
:10566000012384F85D30002384F85C30032003B00C
:10567000BDE8F08F019B002B019B03F1FF3308BFB6
:1056800000250193B0E700BFC80400202DE9F347CF
:105690001F46894690460446FDF7E8F80A9D3D44BA
:1056A0002D1AFDF7E3F8264B1E68C6F3CB366E4382
:1056B000824601962268936839EA03030CBF0123EE
:1056C0000023434501D100202EE07B1CF3D0FDF7E1
:1056D000CDF8A0EB0A00A84229D323685A6822F02B
:1056E000E0025A606268B2F5827F0AD1A268B2F520
:1056F000004F02D0B2F5806F03D11A6822F0400249
:105700001A60A26AB2F5005F07D11A6822F400524B
:105710001A601A6842F400521A60012384F85D305E
:10572000002384F85C30032002B0BDE8F087019BC1
:10573000002B019B03F1FF3308BF00250193B9E75C
:10574000C80400204368B3F5827FF7B504460E46CF
:1057500017460BD18368B3F5004F02D0B3F5806FC5
:1057600004D12268136823F0400313600097334686
:10577000002280212046FFF789FF054628B1236ECD
:1057800043F020032366032514E06368B3F5827FAA
:1057900010D1A368B3F5004F02D0B3F5806F09D1E3
:1057A0000097334600224FF4C0612046FFF702FF06
:1057B0000028E4D1284603B0F0BD73B50B46009233
:1057C0000D4616464FF4C05100220446FFF7F2FE84
:1057D000024628B1236E43F020032366032011E024
:1057E00000962B4680212046FFF750FF02460028F6
:1057F000F0D100962B464FF4C0612046FFF7DAFE49
:105800000028E7D102B070BDF8B5044600287CD06E
:10581000436A002B4FD14268B2F5827F00D0C3614A
:1058200094F85D3003F0FF0223B984F85C20204631
:1058300010F07EF92268E168022384F85D30136875
:10584000B1F5E06F23F0400313604FF000035ED822
:105850004FF4805500D0A3626368A768A069A66A68
:1058600007F4044703F482733B43276907F00207F8
:105870003B43676907F001073B4300F400773B4374
:10588000E76907F038073B43276A07F080073B4387
:1058900006F400573B43B6F5005F136011D1236B4C
:1058A00083BBB1F5E06F0AD902232363136843F485
:1058B0000063136005E00023C0E90433B0E701236F
:1058C0002363636A676B03F0100307F008073B4329
:1058D00001F47061000C194300F004000143B6F5B7
:1058E000005F08BFA38D45EA0105556008BF13613D
:1058F000D36923F40063D36100200123206684F878
:105900005D30F8BD022BDCD1D0E70120F9E71D4660
:10591000B1F5706F9EE72DE9F7431F4690F85C30B4
:10592000012B04460D46904600F0C980012380F803
:105930005C30FCF79BFF94F85D30012B8146D8B2B8
:1059400040F0BB80002D79D0B8F1000F76D0032352
:1059500084F85D3000232366C4E91333A4F83E8045
:105960002364A4F84430A4F84630A3682668A563ED
:10597000B3F5004FA4F83C8007D1336823F040030F
:105980003360336843F480433360A36AB3F5005F48
:1059900007D1336823F400533360336843F4005372
:1059A00033603368E2685B065EBF336843F04003F0
:1059B0003360B2F5E06F636849D913B1B8F1010FF4
:1059C00007D135F8023BF360A563E38F013B9BB23F
:1059D000E387E38F9BB2F3B9A36AB3F5005F04D109
:1059E0002268136843F4805313604A4639462046C0
:1059F000FFF7E3FE08B120232366A36833B90193C0
:105A00002368DA6801929B680193019B206E00383D
:105A100018BF012012E0226893689D0705D5A36B8B
:105A200033F8021BD160A363CFE7FCF71FFFA0EBA5
:105A30000900B842CDD3781CCBD00320012384F8D1
:105A40005D30002384F85C3003B0BDE8F08313B10F
:105A5000B8F1010F13D1E38F9BB2012B06D935F8B2
:105A6000023BF360A563E38F023B06E02B783373C0
:105A7000A36B0133A363E38F013B9BB2E387E38F07
:105A80009BB2002BA8D02268936899070CD5E18FB0
:105A9000A36B89B2012904D933F8021BD160A36337
:105AA000E1E71B781373E3E7FCF7E0FEA0EB0900E6
:105AB000B842E4D37B1CE2D0BFE70220BEE702205D
:105AC000C2E72DE9FF479946002303938DF80B3079
:105AD00090F85C300C9F012B04460E46924600F075
:105AE000B081012380F85C30FCF7C0FE94F85D3093
:105AF000D4E90051012B2A6880465FFA83FC68686C
:105B00000BD0B1F5827F40F09A81A368002B40F062
:105B10009681BCF1040F40F09281002E00F072815A
:105B2000BAF1000F00F06E81B9F1000F00F06A8148
:105B300094F85D30C4F840A0042B1CBF052384F802
:105B40005D3000232366C4E91333A36AA4F84690AA
:105B5000B3F5005FA4F84490A663A4F83E90A4F8BF
:105B60003C9007D12B6823F400532B602B6843F43F
:105B700000532B60D4F80CC06B68BCF5E06F02D802
:105B8000B9F1010F3AD923F480536B602B685B069F
:105B90005EBF2B6843F040032B60BCF5E06F7FD9FC
:105BA00011B1B9F1010F07D136F8023BEB60E38F79
:105BB000A663013B9BB2E3874FF0010902F00406A4
:105BC00000F00805E38F9BB2DBB9B4F846309BB216
:105BD000BBB9A36AB3F5005F40F0FD800122CDF8A8
:105BE00000803B4611462046FFF750FD002800F09C
:105BF000EA80236E43F0020323662AE043F48053D5
:105C0000C3E723689A68900707D5E28F92B222B162
:105C1000B9F1000F28D14FF00009996811F0010186
:105C20000FD0B4F8462092B25AB1DA68236C23F848
:105C3000022B2364B4F84630013B9BB2A4F84630F3
:105C40008946FCF713FEA0EB0800B842BAD3791CD2
:105C5000B8D00325012384F85D30002384F85C303C
:105C6000284604B0BDE8F087A26B32F8021BD96069
:105C7000E18FA263013989B2E187E28F92B2002AF3
:105C8000C9D1A26AB2F5005FC5D126B91DB11A68A3
:105C900042F400721A601A6842F480521A60BAE73D
:105CA00011B1B9F1010F0BD1E38F9BB2012B4BD98D
:105CB00036F8023BEB60E38FA663023B9BB2E387BF
:105CC000012502F0040600F00809E38F9BB22BB90E
:105CD000B4F846309BB2002B3FF47BAF21688B6851
:105CE0009A0705D5E38F9BB213B1002D34D100255F
:105CF00021688B6813F001031DD0B4F8462092B2DE
:105D0000CAB1B4F84600226C80B201284FD9C868E5
:105D100022F8020B2264B4F84620023A92B2A4F8A8
:105D20004620B4F8462092B2012A03D84A6842F4C9
:105D300080524A601D46FCF799FDA0EB0800B8426E
:105D4000C3D37B1CC1D084E733782B73A36B01339F
:105D5000A363E38F013BB1E7E28FA36B92B2012A09
:105D60001DD933F8022BCA60A363E38F023B9BB2B9
:105D7000E387E38F9BB2002BB9D1A36AB3F5005F31
:105D8000B5D1236836B9B9F1000F03D01A6842F4CF
:105D900000721A601A6842F480521A60A7E71B78F2
:105DA0000B73A36B0133A363E38F013BDFE7097B35
:105DB0001170226C01322264B4F84620013A92B28A
:105DC000A4F84620B6E7E3682568B3F5706F1BD1E9
:105DD000EB680393039B2268956815F0100507D0C4
:105DE000236E43F0020323664FF6EF7393600125A1
:105DF000424639462046FFF7E0FC00283FF42AAF30
:105E000020232366012525E72B7BDBB28DF80B30A1
:105E10009DF80B30236B022BDDD10122CDF80080E1
:105E20003B4611462046FFF731FC00287FF4E1AEE7
:105E30002B7BDBB28DF80B309DF80B30CBE70225C6
:105E400008E702250CE72DE9FF411D4600230393D7
:105E50008DF80B304368B3F5827F044688461746B9
:105E60000CD1836853B9042380F85D301346009544
:105E70000A46FFF726FE04B0BDE8F08194F85C30D6
:105E8000012B00F0FC80012384F85C30FCF7EEFC71
:105E900094F85D30012B0646D8B240F0EE80B8F1A0
:105EA000000F00F09F80002F00F09C80042384F8F6
:105EB0005D3000232366C4E91333A4F84670A3635E
:105EC000A387E387A36A2268C4F84080B3F5005F24
:105ED000A4F844700DD1136823F4005313601368C1
:105EE00043F400531360B4F84630013B9BB2A4F86E
:105EF0004630E1685368B1F5E06F8CBF23F48053FE
:105F000043F480535360A368B3F5004F07D113687F
:105F100023F040031360136823F480431360136875
:105F20005B065EBF136843F040031360B1F5E06F9A
:105F300023D9B4F846309BB223B323689A68D107BB
:105F400057D5DA68236C23F8022B2364B4F8463063
:105F5000013B9BB2A4F84630EBE723689A68D70769
:105F600038D5226C1B7B1370236C01332364B4F887
:105F70004630013B9BB2A4F84630B4F846309BB2A1
:105F8000002BEAD1A36AB3F5005F42D122681368FF
:105F900043F480531360012200962B46114620469D
:105FA000FFF774FBE8B9E1682268236CB1F5E06F94
:105FB0008BBFD268127B1A801A70012200962B4682
:105FC00011462046FFF762FBD8B1236E43F002036F
:105FD000236606E0FCF74AFC801BA842CDD3681C70
:105FE000CBD00320012384F85D30002384F85C309B
:105FF00041E7FCF73BFC801BA8429AD36A1C98D06F
:10600000EFE7E2682768B2F5706F1AD1FB68039377
:10601000039B324629462046FFF794FB08B1202314
:10602000236622689368DB0606D5236E43F00203DD
:1060300023664FF6EF739360206E003818BF01207F
:10604000D0E73B7BDBB28DF80B30B2F5E06F9DF80B
:106050000B30DED1236B022BDBD1012200962B46C5
:1060600011462046FFF712FB0028AED13B7BDBB286
:106070008DF80B309DF80B30CBE70220B2E7022001
:10608000F9E60000034AD2F8903043F40043C2F826
:106090009030704700040058034AD2F8903023F43F
:1060A0000043C2F89030704700040058074B1A684C
:1060B00022F040021A6040F441704FF4B852186068
:1060C0005A601A6842F040021A6070470000015896
:1060D00013B50446002842D0837903F0FF0213B9B8
:1060E0004271F1F7F7FE0223A3714FF0B043D3F8EA
:1060F000942022F40042C3F894201A4A11681C220A
:106100004A43D20C64214A430192019AF2B9012117
:10611000A160FFF7B7FF144AD2F8903043F48053E0
:10612000C2F89030114B9A6842F400629A604FF4C2
:1061300000629A6129B92068FFF7B8FF0123237133
:10614000A1600123A371084602B010BD019A013A73
:106150000192D3F8941011F48041D6D1D9E70121EE
:10616000F1E700BFC80400200008005800040058F0
:1061700013B50246174804681C236343DB0C6424F0
:106180006343154C01930346019898B90120906030
:10619000124C217019681C234B43DB0C64214B43C8
:1061A0000D490193019B6BB9012090600A4BDB689C
:1061B00002B010BD019801380190A0688007E3D5B6
:1061C0000020E5E7019B013B01938B68DB07E9D5E4
:1061D000ECE700BFC8040020000001580C00015883
:1061E00037B50246184804681C236343DB0C64245B
:1061F0006343164C019303460198A8B901209060AF
:10620000134CFF2525701C681C236343DB0C64249E
:1062100063430E4C0193019B73B9012090600B4BBB
:10622000DB680B7003B030BD019801380190A068A5
:106230008007E1D50020E3E7019B013B0193A368C0
:10624000DB07E8D5EBE700BFC804002000000158D9
:106250000C0001580F4B13B51A680F4C1823534309
:106260001B0D64225343014601936269019B02F0B6
:10627000040223B902238B60012002B010BD019BF0
:10628000013B0193606910F00200F6D0002AECD1C6
:106290001046F2E7C80400200004005807B503794F
:1062A000012B0FD10A4B1A68182353431B0C01937F
:1062B000FFF7F2FE019B013B0193019B002BF9D1FB
:1062C000FFF7E0FE03B05DF804EBFFF7C3BF00BFCC
:1062D000C8040020F8B51E468379012B15460446F4
:1062E0000F46DAB22DD14379012B2AD00223427115
:1062F0008371FFF7D3FFFFF7CFFE0D212046FFF795
:1063000037FF390A2046FFF733FFF9B22046FFF77F
:106310002FFF2E44B5420ED1FFF7B4FE2046FFF703
:1063200099FFA06801230038A3714FF0000318BF44
:1063300001206371F8BD15F8011B2046FFF718FF17
:10634000E8E70220F6E7F8B51E468379012B1546EB
:1063500004460F46DAB22FD14379012B2CD042717B
:10636000FFF79CFFFFF798FE1D212046FFF700FF77
:10637000390A2046FFF7FCFEF9B22046FFF7F8FE87
:1063800000212046FFF7F4FE2E44B5420ED1FFF760
:1063900079FE2046FFF75EFFA06801230038A37155
:1063A0004FF0000318BF01206371F8BD2946204655
:1063B000FFF716FF0135E8E70220F6E7F8B51F46BC
:1063C0008379012B154604460E46DAB22CD1437967
:1063D000012B29D04271FFF761FF06F0EF03A3F113
:1063E0008402534253412371FFF756FE3146204643
:1063F000FFF7BEFE2F44AF4210D1FFF743FE842EBD
:1064000002D02046FFF726FFA06801230038A371C1
:106410004FF0000318BF01206371F8BD15F8011B90
:106420002046FFF7A5FEE6E70220F6E7F8B51E4690
:106430008379012B154604460F46DAB227D14379FA
:10644000012B24D04271FFF729FFFFF725FE0E2113
:106450002046FFF78DFE39462046FFF789FE2E4481
:10646000B5420ED1FFF70EFE2046FFF7F3FEA068FF
:1064700001230038A3714FF0000318BF012063719E
:10648000F8BD15F8011B2046FFF772FEE8E7022071
:10649000F6E7F8B51E468379012B154604460F46EC
:1064A000DAB22BD14379012B28D04271FFF7F6FEE7
:1064B000FFF7F2FD1E212046FFF75AFE394620461F
:1064C000FFF756FE00212046FFF752FE2E44B5424C
:1064D0000ED1FFF7D7FD2046FFF7BCFEA0680123D1
:1064E0000038A3714FF0000318BF01206371F8BD9D
:1064F00029462046FFF774FE0135E8E70220F6E75B
:10650000F8B51E468379012B154604460F46DAB2CC
:1065100027D14379012B24D04271FFF7BFFEFFF74B
:10652000BBFD39462046FFF723FE00212046FFF73A
:106530001FFE2E44B5420ED1FFF7A4FD2046FFF703
:1065400089FEA06801230038A3714FF0000318BF33
:1065500001206371F8BD29462046FFF741FE013551
:10656000E8E70220F6E737B50023ADF8043001AACA
:10657000022312210446FFF7C3FF9DF805309DF862
:106580000450DA0743EA052502D5204602F0B6FC9E
:10659000AB0702D5204602F0B7FC680702D52046BB
:1065A00002F0DCFC290702D5204602F0DDFCEA06F9
:1065B00002D5204602F0DEFCAB0602D5204602F0F2
:1065C000C7FC680602D5204602F0A4FC290607D5C0
:1065D000EA05C5F30021204648BF012102F0A0FCD6
:1065E000AB0502D5204602F0ABFC022301AA1946F6
:1065F0002046FFF7E3FE03B030BD026852E8003FDB
:1066000023F0C00342E8003102680029F5D102F10D
:10661000080353E8003F23F4000302F1080C4CE8A0
:1066200000310029F3D12023C0F8843070470000E6
:1066300010B5026852E8003F23F4907342E800313D
:1066400002680029F5D10F4C02F1080353E8003F1E
:10665000234002F1080C4CE800310029F4D1C36E4C
:10666000012B07D152E8003F23F0100342E800312C
:106670000029F7D12023C0F888300023C3660367C0
:1066800010BD00BFFEFFFFEF38B50546C0B12423A3
:10669000C0F8843003681A68002422F001021A60EE
:1066A0001C605C609C600FF04BF9C5F88C4085F86D
:1066B0008040C5F884402046C5F88840EC6638BD67
:1066C0000120FCE7026838B5D0F88430D0F8885053
:1066D0009168090604461FD5212B1DD102F108033C
:1066E00053E8003F23F0800302F1080040E8003146
:1066F0000029F3D1A06F60B1FDF747FE48B1A06F4C
:10670000FDF709FF202804D11023C4F88C300320A2
:1067100038BD2046FFF771FF2268906810F04000F6
:10672000F6D0222D18D102F1080353E8003F23F0E0
:10673000400302F1080040E800310029F3D1E06F86
:1067400038B1FDF722FE20B1E06FFDF7E4FE20280E
:10675000DAD02046FFF76CFF0020D9E77047806A47
:106760000268D0F8843010B5D0F8884092681206DC
:1067700006D5212B04D10023A0F85630FFF73DFFAA
:1067800003689B685B0606D5222C04D10023A0F881
:106790005E30FFF74DFFD0F88C3043F01003C0F8A7
:1067A0008C30F4F76BFF10BD08B5806A0023A0F8A9
:1067B0005E30A0F85630F4F761FF08BD0368DA696F
:1067C00019682DE9F04140F60F0632429D680446F3
:1067D00010D1960640F1968001F0200605F0805712
:1067E0003E4300F08F80036F002B00F08480BDE8F3
:1067F000F0411847A74EA8482E400840304300F00B
:106800008180D70709D5C80507D501201862D4F8BB
:106810008C0040F00100C4F88C00970709D5E80708
:1068200007D502201862D4F88C0040F00400C4F8A8
:106830008C00570709D5E80707D504201862D4F85B
:106840008C0040F00200C4F88C0017070BD501F053
:106850002000304307D008201862D4F88C0040F0A4
:106860000800C4F88C0016050AD5480108D54FF475
:1068700000601862D4F88C3043F02003C4F88C30E8
:10688000D4F88C30002B36D093060AD501F02001C5
:1068900005F0805551EA050303D0236F0BB1204664
:1068A00098472368D4F88C509B6805F0280503F0BE
:1068B00040031D43204620D0FFF7BAFE22689368AC
:1068C0005F0615D502F1080353E8003F23F04003AB
:1068D00002F1080040E800310029F3D1E06F38B13F
:1068E0006E4B8363FDF786FD28B1E06F836B7EE717
:1068F0002046F4F7C3FEBDE8F081F4F7BFFEC4F80C
:106900008C50F8E7E06E012840F08180D6067ED5F5
:10691000C8067CD510221A629A68510647D5E26FE4
:1069200011684A6892B2002AE5D0B4F85C0090423F
:10693000E1D9A4F85E200A6892062ED453E8002F0D
:1069400022F4807243E800210029F7D103F1080204
:1069500052E8002F22F0010203F1080040E8002174
:106960000029F3D103F1080252E8002F22F040027F
:1069700003F1080040E800210029F3D12022C4F8E7
:106980008820E16653E8002F22F0100243E800213E
:106990000029F7D1E06FFDF7F8FCB4F85E30B4F8E9
:1069A0005C10C91A89B22046F4F774FDA3E7B4F865
:1069B0005E108AB2B4F85E1089B200299BD0B4F898
:1069C0005C10891A89B2002995D053E8002F22F46F
:1069D000907243E800200028F7D1314D03F10802FE
:1069E00052E8002F2A4003F1080646E8002000285C
:1069F000F4D12022C4F888202067E06653E8002FF5
:106A000022F0100243E800200028F7D1CBE7D7029C
:106A100009D56E0207D54FF4801220461A62BDE8F0
:106A2000F041F4F7AFBD10060BD501F0800005F47E
:106A30000005284305D0636F002B3FF45CAF204670
:106A4000D5E6570611D54E060FD553E8002F22F094
:106A5000400243E800210029F7D12023C4F8843004
:106A600061672046FFF77AFE45E7150206D5480024
:106A700004D52046BDE8F04100F019BCD3017FF5F4
:106A80003AAF0029BFF637AF2046BDE8F04100F02D
:106A90000DBC00BF0100001020010004A96701081F
:106AA000FEFFFFEF806A08B5C36E012B05D1B0F879
:106AB0005C104908F4F7EEFC08BDF4F7DBFCFBE7DB
:106AC00008B50346806A1B681B6813F0200331D1A8
:106AD000A0F85E30026852E8003F23F4807342E879
:106AE000003103680029F5D103F1080252E8002FB4
:106AF00022F0010203F1080C4CE800210029F3D137
:106B000003F1080252E8002F22F0400203F1080CC2
:106B10004CE800210029F3D12022C0F88820C26E61
:106B2000012A07D153E8002F22F0100243E8002188
:106B30000029F7D1C36E012B04D1B0F85C10F4F733
:106B4000A9FC08BDF4F74CFCFBE710B590F88030C9
:106B5000012B1ED0012380F880302423C0F884301C
:106B6000026852E8003F23F00C0342E80034016859
:106B7000002CF5D151E8002F42F0080241E8002333
:106B8000002BF7D12022C0F8842080F880301846EE
:106B900010BD0220FCE710B590F88030012B1ED00C
:106BA000012380F880302423C0F88430026852E842
:106BB000003F23F00C0342E800340168002CF5D1BB
:106BC00051E8002F42F0040241E80023002BF7D1E6
:106BD0002022C0F8842080F88030184610BD0220A2
:106BE000FCE7D0F88C007047F8B5044603682169CB
:106BF000A2681D68C0690A4361690A437E4902436D
:106C000029400A431A605A68E16822F440520A4354
:106C10005A607A4AA16993421CBF226A11439A685A
:106C200022F06E4222F430620A439A60DA6A616AA4
:106C300022F00F020A43DA62714A93421CD14FF0EC
:106C4000B043D3F8883003F0030343F44033A3F593
:106C50004033013B022B00F2C8806A4A9B5CB0F5CE
:106C6000004F40F08A80082B24D8DFE803F061C190
:106C70008423812323236500634A934209D14FF083
:106C8000B043624AD3F8883003F00C0343F4402346
:106C9000E4E75A4A93420DD14FF0B043D3F888301D
:106CA00003F44063B3F5006F1AD005D853B1B3F5C0
:106CB000806F12D0012009E0B3F5406FFAD14FF494
:106CC00000400EE0FEF732FA58B900204FF00113F1
:106CD000A3660023C4E91C33F8BDFDF72BFEF3E7E0
:106CE0004B4865684B4B626A05EB450133F812204F
:106CF000B0FBF2F39942DDD8B3EB053FDAD80023BD
:106D00000021F0F777FA0F0247EA106706026808D9
:106D100030182A464FF0000347F10001F0F76AFAF5
:106D20003D4BA0F540729A42C4D82368D860CCE7A6
:106D3000FEF7FCF90028C8D06268616A354B33F869
:106D40001130B0FBF3F3500800EB4300B0FBF2F05E
:106D500083B2A3F110014FF6EF729142AAD820F04E
:106D60000F00226880B2C3F342031843D060ACE73F
:106D7000FDF7E0FDDEE72648DEE7082B9AD801A202
:106D800052F823F0CF6D0108DB6D0108E76D0108B3
:106D9000B56C0108E16D0108B56C0108B56C01081E
:106DA000B56C0108A96D01084FF400406368616A81
:106DB000184A32F81120B0FBF2F000EB5300B0FBA0
:106DC000F3F080B2A0F110024FF6EF73ABE7FEF7DD
:106DD000ADF900283FF479AFE8E7FEF7B7F9F8E737
:106DE000FDF7A8FDF5E70A48E0E7B0F5004FF4D15C
:106DF000FEF7ACF99EE700BFF369FFCF00800040CB
:106E000000380140A1F1020800440040A4F1F60757
:106E10000024F400B2F10208FFFC0F00836ADA07D5
:106E200010B506D50168C46A4A6822F400322243CC
:106E30004A609C0706D50168046B4A6822F48032D8
:106E400022434A60590706D50168446B4A6822F418
:106E5000802222434A601A0706D50168846B4A687B
:106E600022F4004222434A60DC0606D50168C46B66
:106E70008A6822F4805222438A60990606D5016806
:106E8000046C8A6822F4005222438A605A060FD5A5
:106E90000168446C4A6822F480122243B4F5801FD2
:106EA0004A6005D14A68846C22F4C00222434A60D9
:106EB0001B0606D50268C16C536823F400230B43FC
:106EC000536010BD2DE9F041DDF8188004460E46F0
:106ED00015461F462268D36936EA03030CBF012317
:106EE0000023AB4201D0002027E0B8F1FF3FF2D0F1
:106EF000FBF7BCFCC01B4045206802D8B8F1000F6E
:106F00001DD150E8003F23F4D07340E80032002A3E
:106F1000F7D100F1080353E8003F23F0010300F12B
:106F2000080141E80032002AF3D12023C4F884305C
:106F3000C4F8883084F880200320BDE8F08103681D
:106F40005A07C7D5C3691B05C4D54FF40063036254
:106F500050E8003F23F4D07340E80032002AF7D114
:106F600000F1080353E8003F23F0010300F108019A
:106F700041E80032002AF3D12023C4F88430C4F859
:106F80008830C4F88C30D5E72DE9F7439846D0F81F
:106F90008430202B04460E4617464FD100294BD093
:106FA000002A49D090F88030012B47D0012380F887
:106FB000803000252123C0F88C50C0F88430FBF7C6
:106FC00055FCA368A4F85470B3F5805F8146A4F81B
:106FD000567003D123690BB935461E46002384F849
:106FE0008030B4F85620CDF8008092B24B4642B9BA
:106FF00040212046FFF766FF48B92023C4F88430BB
:1070000006E0002280212046FFF75CFF18B1032034
:1070100003B0BDE8F08322685EB935F8023BC3F3E4
:1070200008039362B4F85620013A92B2A4F85620AD
:10703000D7E716F8013BF4E70120E9E70220E7E78C
:1070400073B504460026C0F88C60FBF70FFC23687C
:107050001B681A07054618D423681B685B070AD506
:107060006FF07E43009300222B464FF480012046B0
:10707000FFF728FFA8B920230020C4F8843084F843
:107080008000C4F88830E0660CE06FF07E43009327
:10709000324603464FF400112046FFF713FF002845
:1070A000DAD0032002B070BD10B5044650B3D0F85A
:1070B00084301BB980F880300EF06AFB22682423EC
:1070C000C4F88430136823F0010313602046FFF7EF
:1070D0008BFD012816D0A36A13B12046FFF79EFE50
:1070E00023685A6822F490425A609A6822F02A0271
:1070F0009A601A6842F0010220461A60BDE810400A
:10710000FFF79EBF012010BD10B5044670B3D0F844
:1071100084301BB980F880300EF03AFB22682423BB
:10712000C4F88430136823F0010313602046FFF78E
:107130005BFD01281AD0A36A13B12046FFF76EFE4B
:1071400023685A6822F490425A609A6822F0220218
:107150009A609A6842F008029A601A6842F0010246
:1071600020461A60BDE81040FFF76ABF012010BD3D
:1071700070B51346A0F85C2000252222C0F88C5080
:1071800004468165C0F88820C06FB8B11E4A2668E1
:10719000C2621E4A02631E4AC0E90D250A4606F174
:1071A0002401FDF7ADF848B11023C4F88C3020233A
:1071B00084F88050C4F88830012070BD002384F822
:1071C0008030226852E8003F43F4807342E8003187
:1071D00022680029F5D102F1080353E8003F43F08B
:1071E000010302F1080040E800310029F3D102F167
:1071F000080353E8003F43F0400302F1080141E86F
:1072000000300028F3D1D8E7C16A0108A56A010857
:107210005F670108D0F88830202B30B41FD1D9B176
:10722000D2B190F88030012B19D0012380F8803042
:1072300000230468C3660B4B9C420AD063681B02A0
:1072400007D554E8003F43F0806344E80035002D43
:10725000F7D130BCFFF78CBF012030BC7047022053
:10726000FBE700BF00800040436E30B51BB94FF014
:107270000113836630BD03680A4D9A6899680A4C09
:10728000490FC2F342626B5C615CDB00B3FBF1F35C
:10729000A0F86A30AB5CA25CDB00B3FBF2F3A0F8B1
:1072A0006830E7E7D2F10208CAF102087047704778
:1072B0001FB504AB03E9060090F880300299012B5A
:1072C00004463AD0012380F880302423C0F884306B
:1072D00003681A6822F001021A609A6822F44012C8
:1072E0000A439A6071B95968BDF80C209DF80E00E8
:1072F00021F01001114359605A6822F07F4242EA9E
:1073000000625A601A6842F001021A60FBF7AEFA96
:107310006FF07E42034600924FF480010022204627
:10732000FFF7D0FD38B92023C4F88430002384F857
:10733000803004B010BD0320F8E70220F9E790F890
:107340008020012A03460ED0012280F8802019688F
:1073500051E8002F42F0020241E800200028F6D157
:1073600083F8800070470220704790F88020012A3F
:1073700003460ED0012280F88020196851E8002FC2
:1073800022F0020241E800200028F6D183F88000B4
:1073900070470220704790F88030012B14D00268AB
:1073A0002423C0F884301168136823F001031360AC
:1073B00021F000510023436611602022C0F8842090
:1073C00080F88030184670470220704738B590F832
:1073D0008030012B04461BD0012380F88030242309
:1073E000C0F8843003681D681A6822F001021A6030
:1073F0009A6822F0604211439960FFF735FF0368F5
:107400001D602023C0F88430002084F8800038BD3F
:107410000220FCE738B590F88030012B04461BD0E1
:10742000012380F880302423C0F8843003681D686D
:107430001A6822F001021A609A6822F06062114311
:107440009960FFF711FF03681D602023C0F88430A6
:10745000002084F8800038BD0220FCE7012070473E
:1074600001F0FCBA01F034BA08B501F030FD012199
:1074700001F017FDBDE8084001F012B938B5074B1F
:1074800004460D4693F85600002101F00AFD2946F6
:107490002046BDE8384001F0DBB800BF307E002058
:1074A000002001F093B8000008B501F089F8043815
:1074B000C0B2032896BF024B0020185C08BD00BF75
:1074C00010F2020873B5764AB2F854300025402B0A
:1074D0008DF803500195144600F0D6801CD8082B77
:1074E00000F0CA8005D8012B2CD0022B43D002B06B
:1074F00070BD202BFBD16B4801F084FF10B16948AF
:1075000001F0C8FF6078002800F0B380664B1B686C
:10751000002BECD0DB682AE0B3F5807F79D0B3F59F
:10752000007F00F08480802BE1D1284601F04EF8E6
:107530005D4B1B68002BDAD09B69002BD7D0284607
:107540009847D4E7594801F05DFF10B1574801F062
:10755000A1FF002001F03AF801F072FD012801D1ED
:1075600001F077FD504B1B68002BC0D01B68002B2F
:10757000BDD09847BBE74B4801F044FF10B14948E4
:1075800001F088FF657895B9284601F01FF8294673
:1075900040F6021001F09CF940F6441001F05EFA4A
:1075A00040F00201C9B240F6441001F091F9FF2207
:1075B0000DF103013E483C4D01F05AFC3D4801F0FD
:1075C0004BF92B68002B92D09E68002E8FD094F838
:1075D0002430012B08D194F9313094F930209DF8F2
:1075E00003103348B04782E7E06B01A901F0DCFCEF
:1075F000019B9DF803102E484FF47A7203F5FA733D
:1076000093FBF2F32A685BB2956894F92920A847A6
:107610006DE7284600F0DAFF234B1B68002B3FF490
:1076200066AF9B69002B3FF462AF012088E700F052
:10763000C7FF042810D11D4801F0E4FE10B11B481B
:1076400001F028FF002000F0C1FF174B1B68002B42
:107650003FF44DAF5B688AE700F0B2FF05287FF486
:1076600046AF104801F0CEFE10B10E4801F012FFF7
:10767000002000F0ABFF49E701F0E0FC01287FF4B7
:1076800036AF01F0E7FC32E7507808B900F09EFF12
:10769000054B1B68002B3FF42AAF1B6967E700BF4F
:1076A000307E0020A07E0020CC490020887E002073
:1076B000CC480020547E002008B501F01DFC0330AA
:1076C00008BD01F063BB01F0BFBA08B501F0B7F81F
:1076D00000B208BD38B50D46144601F085F82846BD
:1076E00001F0F5FB084D012101F0DBFB00F0D8FFB4
:1076F0004FF47A716143284601F056FF2846BDE8F1
:10770000384001F017BF00BF887E002001F06CB840
:1077100008B5084B002193F8560001F0C2FB002386
:107720004FF4C0711A46084601F034F8BDE808402D
:1077300000F0AABF307E002008B54FF0040001F031
:10774000E9F9BDE808400220FBF796B808B5064BFA
:107750001B6843B1DB6833B198470448FBF710F866
:10776000034B00221A7008BDCC490020F40300200E
:107770009C7D002008B5064B1B6843B15B6833B1A4
:1077800098470448FAF7FCFF034B00221A7008BD23
:10779000CC490020F40300209C7D002008B5064B56
:1077A000A3F854000548FAF7EBFF054B00221A70C6
:1077B000BDE80840FFF786BE307E0020F4030020BD
:1077C0009C7D0020F0B5BDF814509DF818E09DF8A0
:1077D0001CC09DF8204040B1012819D0012200238F
:1077E0001344581EB0FBF2F0F0BDBEF1000F0CBF09
:1077F00008230023002C03EBC50314BF022400243C
:107800001833644403EBC4044FF47A736343E7E72B
:107810001E1D531F012B02D80C2D38BF0C2500292B
:1078200038D1A2F10B07012F8CBF00270127002CB4
:1078300014BF1024002404EBCC04BEF1000F14BFCD
:1078400000201420A4EB8204062A04444FEA820399
:10785000A2F1020002D9083407B18300002CACBFAA
:107860001C191C1C062A104A515C04F1FF3494FBBD
:10787000F3F306FB03538CBF0C330E330A2912D8E3
:107880009B0001334FF47A7283405343074A52F806
:107890002120A5E7012904D1A2F10C035F425F4139
:1078A000C5E70027C3E7FFDEDAF10208E4F10208CA
:1078B0000128084805D1084BC17719700E3001F036
:1078C00001BA437D012B03D1034B81751970F5E794
:1078D000704700BF307E0020F003002010B5044642
:1078E00001F0ACFB012817D101F0B0FB34B1104816
:1078F000214601F059FE0E4801F01CFE0D4C0021FE
:1079000094F8560001F0CDFA63786BB16FF07F40C8
:10791000BDE8104000F0ECBF002340F262211A469F
:10792000084600F037FFE1E7A0688001F0E700BFFC
:10793000A07E0020307E002010B5044601F07EFBC2
:10794000012817D101F082FB34B11048214601F023
:107950002BFE0E4801F0EEFD0D4C002194F8560070
:1079600001F09FFA63786BB16FF07F40BDE8104083
:1079700000F058BE002340F262211A46084600F08B
:1079800009FFE1E7A0688001F0E700BFA07E0020CA
:10799000307E00200D4B10B504461873587301203B
:1079A00000F016F85CB134214FF4E86000F090FF6D
:1079B0004421BDE8104040F2417000F089BF14211D
:1079C0004FF4E86000F084FF2421F2E7307E0020CD
:1079D00038B50F4D0446287001F03DFB012C0AD04C
:1079E000023C012C4FF0000494BF0220204600F01E
:1079F000B3FF6C7338BD204600F0AEFF287B6B7B75
:107A00008342F7D06873BDE83840FFF7C3BF00BFBB
:107A1000307E00202DE9F043054687B00027CDE9F0
:107A200001770C469146984601F007FB012D78D06E
:107A3000022D00F0C480002D5CD1A368002B00F063
:107A4000D2802269002A00F0CE80227D082A00F22E
:107A5000CA8001A9AA425BDC644D002685F8386023
:107A6000EB63237885F84430606801F089FA85F883
:107A70004500E3682B64236994F82410AE73DB009F
:107A80002B820423AB74237D2E75DB000229EB745B
:107A90002E46E37F02D0A27F022A3ED103F10F02DD
:107AA000D2B2012A02D9012B40F09D80504B514A9D
:107AB00019680394012503A88DF8145001F0BAFA4F
:107AC000002840F090803076F5757075FFF7E8FC7F
:107AD0000020FFF77DFF484800F054FF474801F0C1
:107AE000F1F801A801F0C0F8A08B01F02DF8208C6E
:107AF00001F0D6F8484601F0EAF93C4C84F856000B
:107B000001F0A0FAC4F80480002007B0BDE8F083BB
:107B1000A069405D685401359CE7EB7529766A756C
:107B2000D4E7324E86F8385094F8283086F8503032
:107B300094F8292086F8512094F82A2086F85220BB
:107B400094F82B10012902D002292BD009B986F80C
:107B50005310A38DB38394F82E30B37794F82F305D
:107B600086F82030012594F8303086F82130B5733E
:107B7000FFF796FC2846FFF72BFF1F4800F002FF97
:107B80001E4801F09FF896F85130062B40F6890008
:107B90000FD100F063FF00F0FB0140F6890000F018
:107BA00097FEA7E70B3B012B88BF3D4686F8535055
:107BB000CFE700F053FF40F00401C9B2EDE7636B7B
:107BC000013BB3F57A7F0ED22846FFF701FF074845
:107BD00080F83850636B8364162380F84C3038305B
:107BE00000F0D0FE86E74FF0FF308EE7307E0020B9
:107BF000CC490020887E0020687E00203E7E002048
:107C00002DE9F041002686B098461446CDE901667C
